:020000040800F2
:100000000000012055460008D1270008D32700082A
:10001000D5270008D7270008D927000800000000CE
:10002000000000000000000000000000DB270008C6
:10003000DD27000800000000DF270008E127000896
:10004000A5460008A5460008E5270008A5460008C3
:10005000A5460008A5460008F1270008F727000874
:10006000A5460008A546000829280008A54600085E
:10007000FD270008FF270008012800080D280008B8
:100080001928000825280008A5460008A5460008EC
:1000900000000000A54600082B280008A54600081F
:1000A000A5460008A5460008A5460008A546000884
:1000B000A5460008A5460008A5460008A546000874
:1000C000A5460008A5460008A5460008A546000864
:1000D000A546000835280008A5460008A5460008E2
:1000E000A54600083128000841280008A546000858
:1000F000A54600080000000000000000A54600081A
:10010000A5460008A54600084D280008A546000899
:10011000A5460008A5460008A5460008A546000813
:10012000A5460008A5460008A5460008A546000803
:08013000A5460008A5460008E1
:1001380010B5054C237833B9044B13B10448AFF319
:1001480000800123237010BDCC08002000000000AF
:10015800C843010808B5034B1BB103490348AFF373
:10016800008008BD00000000D0080020C843010836
:1001780014214160704714207047406A704700009E
:10018800790100087F01000883010008990100082F
:1001980010B5044604F1100000F05CFCC4F8F80047
:1001A8000148C4F87C0110BD88010008F8B5E6B024
:1001B80004460D4616461F460A4906A800F0CAFE20
:1001C80070996F9A05910492009733466E996D9ACB
:1001D800039102922A466C990191214600F060F839
:1001E80067B0F0BD94010008F8B5E6B004460D46C6
:1001F80016461F46094906A800F0ACFE6F996E9A8C
:100208000491039200976D996C9A0291019233467A
:100218002A46214600F087F867B0F0BD940100082F
:1002280038B500281CBF01680029184A23D1184B8B
:100238001C684FF6F0710C404CF24025AC421FBFD1
:100248001B6819404CF27024A14212D1114D296843
:1002580079B911490B68C3F30B03B3F58A6F1FBF54
:100268000968C1F30B0140F28343994204BF01219D
:10027800117028B905E0094B994204BF012111709A
:100288004068BDE8324001F09FBE00BFE80800208A
:1002980000ED00E0002004E00010005C000037489A
:1002A8002DE9F04104460D46216816464A681F4666
:1002B80090478046B8F5403F2ED122680A99936846
:1002C800204698478046B8F5403F25D12368089ACC
:1002D8000799D3F80CC02046E0478046B8F5403F60
:1002E8001AD12368069A39461F692046B8478046BE
:1002F800B8F5403F10D1236829465D69324620464B
:10030800A8478046B8F5403F06D123680B9A09995B
:100318009D692046A847804621680A68204690477C
:100328004046BDE8F0812DE9F04104460D462168BC
:1003380016464A681F4690478046B8F5403F2ED17A
:1003480022680A999368204698478046B8F5403F46
:1003580025D12368089A0799D3F80CC02046E047AE
:100368008046B8F5403F1AD12368069A39461F6976
:100378002046B8478046B8F5403F10D12368294643
:100388005D6932462046A8478046B8F5403F06D109
:1003980023680999DD6900222046A847804621681C
:1003A8000A68204690474046BDE8F0814FF4403047
:1003B80070470000F0B50C4685B0114600281A4673
:1003C8001CBF0568002D0B4B11D082B104B971B95F
:1003D8000D9860B10F9E0E9F0A9B0290049603979A
:1003E8000B980C9E009001962046A8470346184695
:1003F80005B0F0BD020003002DE9F04F0646D0B06D
:100408000868F56DD6F860E0726EB76EF36E00BAE4
:1004180000906C46486800BA60600DF14008886832
:1004280000BAA060C86800BAE060086900BA206134
:10043800486900BA6061886900BAA061C86900BAF1
:10044800E061086A00BA2062486A00BA6062886A95
:1004580000BAA062C86A00BAE062086B00BA2063FA
:10046800486B00BA6063886B00BAA063C86B00BAB7
:10047800E063402058F80C1C58F820CC58F838ACE9
:100488008CEA010158F840CC8AEA01018CEA01099A
:100498004FEAF979401E48F8049BEBD187EA02003D
:1004A80000EA0E00784010EBF5610098DFF824C4EC
:1004B80041186144C81882EABE032B404FEAF06134
:1004C80053405918636859186144CF194FEAB50366
:1004D80083EABE01014081EABE0111EBF765A1681C
:1004E8004D196544A91883EAB0023A404FEAF1650C
:1004F8005A405519E26855194FEAB70282EAB0071F
:1005080065440F4005EBBE0E97EAB00717EBFE6592
:1005180027697D194FEAB10782EA0701654401EAB4
:100528000E01EB18514011EBF36561694D194FEA63
:10053800BE0187EA010E65440EEA030E15EBB00012
:100548008EEA070E0EEBF065D4F818E075446544A2
:10055800AA1881EAB30505404FEAF26E4D40AE4451
:10056800E569AE44E64477444FEAB00080EAB30E4A
:100578000EEA020E8EEAB30E0EEBF765D4F820E011
:1005880075446544691880EAB2053D404FEAF16E4A
:100598004540AE44656AAE44E6440EEBB3034FEA09
:1005A800B70787EAB20E0EEA010E8EEAB20E0EEB1C
:1005B800F365D4F828E075446544281887EAB1053E
:1005C8001D404FEAF06E7D40AE44E56AAE44E64415
:1005D8000EEBB2024FEAB30383EAB10E0EEA000E45
:1005E8008EEAB10E0EEBF265D4F830E0754465443E
:1005F800EF1983EAB00515404FEAF76E5D40AE4447
:10060800656BAE44E6440EEBB1014FEAB20282EAF2
:10061800B00E0EEA070E8EEAB00E0EEBF165D4F8B6
:1006280038E075446544EB1882EAB7050D404FEA97
:10063800F36E5540AE44E56BAE44E6440EEBB000B5
:100648004FEAB10181EAB70E0EEA030E8EEAB70E41
:100658000EEBF065D4F840E07544654481EAB30ECA
:10066800AA180EEA000E4FEAF2658EEA010E7544EA
:10067800DDF844E04FEAB000754480EAB30E654403
:100688000EEA020E15EBB7078EEAB30E0EEBF7650E
:10069800DDF848E04FEAB202754480EA020E65448C
:1006A8000EEA070E69188EEA000E0EEBF165DDF80A
:1006B8004CE07544654405EBB3034FEAB70E1427C5
:1006C8000DF1500CDFF810528EEA010B82EA0B0B89
:1006D8000BEBF36A5CF804BBDA44AA44504483EA9F
:1006E800B10B4FEAF06A8EEA0B0BDA445CF804BBF4
:1006F800DA44AA44524480EAB30B4FEAF26A8BEA1E
:10070800B10BDA445CF804BBDA444FEAB000AA44FF
:1007180080EA020BD6448BEAB30B0BEBFE6A5CF85B
:1007280004BBDA444FEAB202AA4482EA0E0B0AEB8F
:10073800B10180EA0B0B0BEBF16A5CF804BBDA44FD
:100748007F1DAA44282F0AEBB3034FEABE0EBBD382
:100758003C2F61D3502F4DD204EB870CC7F15407BF
:100768005E4CA7FB04A504465D4FA8088EEA010A63
:1007780082EA0A0A5CF804BB0AEBF3655D447D195A
:100788002C1983EAB10A4FEAF4658EEA0A0A55443D
:100798005CF804AB5CF804BB55447D19AA1884EADC
:1007A800B30A4FEAF2658AEAB10A55445D444FEA52
:1007B800B4047D1984EA020AAE448AEAB30A0AEB51
:1007C800FE655CF804AB55444FEAB2027D1982EA33
:1007D8000E0A15EBB10184EA0A0A5CF804BB0AEBBD
:1007E800F1655D447D1915EBB303401E4FEABE0E5B
:1007F800BCD12046F46D1B19F365336EC9183166F8
:10080800716E71447166B36ED218B266F16E40189B
:10081800F06650B0BDE8F08F4EEA010B0EEA010A0F
:100828000BEA020B4BEA0A0A0AEBF36554F827A015
:10083800DFF8B0C0554443EAB10B654403EAB10A96
:100848000BEA0E0B28184BEA0A0A7F1C0AEBF06524
:1008580054F827A0554440EAB30B654400EAB30AAC
:100868000BEAB10BAA184BEA0A0A7F1C0AEBF265DD
:1008780054F827A055444FEAB00040EA020B6544FB
:1008880000EA020A0BEAB30BAE444BEA0A0A7F1CE1
:100898000AEBFE6554F827A055444FEAB20242EA33
:1008A8000E0B654402EA0E0A0BEA000B15EBB101C8
:1008B8004BEA0A0A7F1C0AEBF16554F827A0554455
:1008C8007F1C65443C2F05EBB3034FEABE0EA3D350
:1008D80040E700BF9979825AA1EBD96ECDCCCCCC38
:1008E800D6C162CADCBC1B8F00B581B00168074A5B
:1008F800914200D110B9064801B000BD7C2113F027
:10090800C9FC4FF4003001B000BD00BFFC0900086D
:10091800030002002DE9F0410B4A92E8F85188B033
:10092800694681E8F8510268084B9A4200D118B923
:10093800074808B0BDE8F0811422083000F04FFBEA
:1009480008B0BDE8F08100BFDC090008FC09000818
:1009580003000200152904D20268044B9A4200D110
:1009680008B903487047083000F048BBFC09000884
:100978000300020010B481B013460268074CA2427B
:1009880000D118B901B010BC0548704701B000F19A
:10099800240210BC083000F035BB00BFFC09000879
:1009A8000300020010B481B013460268074CA2424B
:1009B80000D118B901B010BC054870470A4601B00B
:1009C80000F1240110BC083000F070BBFC090008DD
:1009D800030002000123456789ABCDEFFEDCBA981E
:1009E80076543210F0E1D2C300000000000000008D
:1009F80000000000F10800081D0900085D09000852
:100A08007D090008AD09000801040008790F0008F5
:100A1800C50F0008810F0008F0B5A3B004460B48C5
:100A280002900D4616461F46094B0822402104A88D
:100A380000F0D1FA28980190009733462A462146BB
:100A480002A800F01BF823B0F0BD00BFFC090008A5
:100A5800100A000810B5040008BF002408D0054893
:100A6800054B20600822402104F1080000F0B3FA89
:100A7800204610BDFC090008100A00082DE9F041C5
:100A880004460E46216817464A681D469047804628
:100A9800B8F5003F19D1226806999368204698470F
:100AA8008046B8F5003F10D123683146DE683A46E3
:100AB8002046B0478046B8F5003F06D12368079A1C
:100AC80029461D692046A847804621680A682046AD
:100AD80090474046BDE8F08110B500F033FA4FF476
:100AE800403400280EBF034C4FF4C07113F0D2FB02
:100AF800204610BD0200030010B5044600F022FA9B
:100B080008B9054810BD0021A160D0F87C21116802
:100B180088474FF4403010BD0200030070B504460A
:100B28000D4600F00FFA064E40B1D0F87C0141683E
:100B38008847A84224BF65604FF44036304670BDF0
:100B4800020003002DE9FF4715000C4600D02CB128
:100B5800064600F0F7F95FEA000801D16448C3E0EF
:100B6800D8F8F80001684A689047B0F5003F17D1F7
:100B7800D8F87C118A68404690478146B9F1810FC0
:100B880080F09E80A94508F1FC0A17D2D8F8F80031
:100B98000368D3F80CC02A462146E047B0F5003F69
:100BA80040F08E80D8F8F8000368D3F810C06A4681
:100BB8005146E047B0F5003F76D10AE0002004E056
:100BC800215C0AF800100098401C00900098A84288
:100BD800F6D34FF0000C4749474A484B01AC009800
:100BE800844558D2D3E9007001ADC5E9007010788A
:100BF80000281ABF042086464FF0000E085854F803
:100C08000E5028443E4D05600127D0F800E087606B
:100C1800019D4F681AF80C007D408EEA050585F0A5
:100C2800040E65680F687D4085F0FC05754485F005
:100C3800A30568400AF80C000CF1010CCFE7D3E9D2
:100C4800004501A8C0E9004510782E4D002814BFC2
:100C58004FF0040E4FF0000E01A8744651F80EE054
:100C68000459A6440127CEF80050DEF80040CEF81B
:100C780008704D68019F40687D406C400D68684071
:100C880084F0040480F0FC00041984F057040AF886
:100C98000C400CF1010CCC45D1D3D8F8F800016810
:100CA8004A689047B0F5003F0AD1D8F8F8000368C1
:100CB800D3F80C804A465146C047B0F5003F01D0F2
:100CC800114811E0002006E05AF8201081F06A313E
:100CD8004AF82010401CB0EB990FF5D3B06840F0EB
:100CE8000100B0604FF4403004B0BDE8F08700BFA9
:100CF8000200030034440108E8080020240F00081B
:100D0800ADBE4ED70DBE75A10100030038B50C4627
:100D1800017A1546CA0702D500F014F908B908483F
:100D280032BDD0F8F80003682146DC682A46A0479F
:100D3800B0F5003F01D0034832BD4FF4403032BD1A
:100D480002000300010003002DE9F84191B00546B7
:100D58000E461746402101A813F09CFA297AC807C5
:100D680004D5284600F0EEF8040002D1DFF8A4808C
:100D78004BE0D4F8F800DFF8A0800368D3F810C07F
:100D88006A4601A9E047B0F5003F3ED1D4F8F80023
:100D980001684A689047B0F5003F36D1D4F87C1115
:100DA8008A6820469047D4F8F830024618461B68EF
:100DB800D3F80CC004F1FC01E047B0F5003F24D1A2
:100DC800D4F87C0141688847D4F8F83002461846C0
:100DD8001B68D3F80CC001A9E047B0F5003F14D157
:100DE800D4F8F8000268696893689847B0F5003F3E
:100DF8000BD1D4F8F80003681C693A463146A0477D
:100E0800B0F5003F08BF4FF44038404612B0BDE887
:100E1800F08100BF02000300010003002DE9F84142
:100E2800A5B0074688461646402115A813F032FAA1
:100E380000220492402105A813F02CFA387AC10741
:100E48005ED5384600F07EF8050059D0D5F8F80090
:100E58002D4C0368D3F810C06A4605A9E047B0F5E1
:100E6800003F3CD1D5F8F80001684A689047B0F5D2
:100E7800003F34D1D5F87C118A6828469047D5F8C8
:100E8800F830024618461B68D3F80CC005F1FC017F
:100E9800E047B0F5003F22D1D5F87C01416888478A
:100EA800D5F8F830024618461B68D3F80CC005A9D7
:100EB800E047B0F5003F12D1D5F8F800026879682C
:100EC80093689847B0F5003F09D1D5F8F800036852
:100ED8001D6904AA15A9A847B0F5003F01D020460E
:100EE8000FE00A4B0A490B4A0396029101924046C9
:100EF8001C68049B009415AA796800F0E5F900E0E5
:100F0800054826B0BDE8F081010003003C44010813
:100F1800936E030026C703000200030004B001011A
:100F280000170145E10A0008010B0008250B00081D
:100F3800B50300084D0B0008150D0008510D0008F9
:100F4800250E00080168024A914218BF0020704728
:100F58002C0F000810B5040008BF002404D0034873
:100F68002060204609688847204610BD2C0F0008DD
:100F780020225C3013F08CB9F0B58468A3080022F5
:100F880004F0030407E000F15C0555F8226035BA67
:100F980041F82250521C9A42F5D300220BE000F18E
:100FA8005C0502EB830755F82360D500C5F11805E9
:100FB800EE40CE55521CA242F1D3F0BD30B5C46804
:100FC80003690022E31AD5188C5C0544521C082AD0
:100FD8002C77F8D330BD0360C1600261704738B523
:100FE800044615460022626023685A68904700202C
:100FF8006061A061A5604FF4003032BD81604FF49C
:10100800003070472DE9F84304462079D4F80C8065
:10101800450748BF244845D466691D46A8F1010024
:1010280000EAD60306EBC506B6EBC50F666102D229
:10103800A669761CA6611746A66906EB5576A661D1
:101048000E46E918884225D2A8EB03094A463146DC
:10105800F81813F01DF92268136839460FE0424664
:10106800384613F015F923681A6839462046904720
:1010780007E0311811F00300F1D122681368204607
:101088009847484600EB0809A9F10101A942F0D3A5
:10109800002300E000202A1A3118F81813F0F8F895
:1010A8004FF40030BDE8F283040002002DE9FC4F44
:1010B800024685B0D0681369DFF86CC1DFF86C812F
:1010C800A0EB030A506840F004005060002703A812
:1010D80002900DF10C0ED8E9003403A8544DC0E974
:1010E80000342878534D00280CBF00230423994668
:1010F8005CF803305EF80940234401261D601C6833
:101108009E60DCF80430039DDCF80090DEF8046093
:101118005D406540484C654089EA0606474C664094
:101128007519474C6540D8E9006B03AC0028C4E941
:10113800006B0EBF002404200424029E5CF800000B
:10114800345920183F4C04600126046886600398CF
:10115800029E43406340384C7068634089EA00004F
:10116800364C6040034438484340280018BF0120EB
:101178005B1E9B41042F2CBFC0B2D80F02F1140391
:1011880053F8200007F00303C3F10303DB00D84042
:101198000DF807007F1C082F9DD315460C466A6979
:1011A800AB69E868D20842EA4372401E00EA0207C7
:1011B800002302409B420AD8524508D28020E055BD
:1011C8007F1C574516D2AAEB0701E01910E08020D2
:1011D800E05500E0E355E8687F1C8742FAD32A68A7
:1011E800136828469847BAF1000F03D051462046A5
:1011F80013F050F82A68069E059F936869462846AA
:1012080098472A68D2F8009021462846C8472B6894
:10121800DA683946284690470EB1A86830604FF41E
:10122800003007B0BDE8F08F3444010854120008BC
:10123800E80800205FC5109304850012FC68017A55
:10124800C0F524FF24AF33D426AF698B04B0010165
:1012580000170145F8B501240094002300240DE08F
:10126800009D065D0F5D7E40F643761CF60F86F006
:10127800010635400095641C009DEB189442EFD39D
:101288001846F2BDF8B5002301240094002A11E0A5
:10129800009C85188F1815F8016C17F8015C6E40D2
:1012A800F643761CF60F86F0010634400094009C45
:1012B800E318521EECD11846F2BD00005D1200087A
:1012C8008D120008010000002DE9F84F1D46DDF8D9
:1012D80028900B9F0D9C4FF0FF3300930E469246CB
:1012E800D9F800B0804632465146D847834664B3A1
:1012F800D9F8043032465146404698476FEA0B0207
:10130800521C42EA0B0200996FEAD2735B1C194027
:10131800C2430091521C024300996FEAD2735B1CCE
:101328001940009186F05531484087EA000181F064
:101338005531216080F05531C943491C0843009A52
:101348006FEAD070401C82430092D9F80800012847
:1013580009D17540E943491C0D4300986FEAD572DD
:10136800521C90430AE0F11C85EA9102D243521CB8
:10137800154300986FEAD5735B1C984386F0AA362C
:10138800009086EA0B0686F0AA33F243DB430C98FA
:10139800C2F3C0725B1C42EAD3720099D243521C5A
:1013A80091430091774000998843009987F0AA37C4
:1013B8000F403843BDE8F28F034613F8012B002A8B
:1013C800FBD1181A0138704781F0004102E000BFD4
:1013D80083F0004330B54FEA41044FEA430594EAED
:1013E800050F08BF90EA020F1FBF54EA000C55EA28
:1013F800020C7FEA645C7FEA655C00F0E2804FEAF9
:101408005454D4EB5555B8BF6D420CDD2C4480EADA
:10141800020281EA030382EA000083EA010180EA0A
:10142800020281EA0303362D88BF30BD11F0004F58
:101438004FEA01314FF4801C4CEA113102D040428E
:1014480061EB410113F0004F4FEA03334CEA1333C9
:1014580002D0524263EB430394EA050F00F0A780E1
:10146800A4F10104D5F1200E0DDB02FA0EFC22FADC
:1014780005F2801841F1000103FA0EF2801843FAD0
:1014880005F359410EE0A5F120050EF1200E012AC1
:1014980003FA0EFC28BF4CF0020C43FA05F3C018FF
:1014A80051EBE37101F0004507D54FF0000EDCF178
:1014B800000C7EEB00006EEB0101B1F5801F1BD321
:1014C800B1F5001F0CD349085FEA30004FEA3C0C25
:1014D80004F101044FEA445212F5800F80F09A801B
:1014E800BCF1004F08BF5FEA500C50F1000041EB1F
:1014F800045141EA050130BD5FEA4C0C404141EB23
:101508000101013C28BFB1F5801FE9D291F0000F1D
:1015180004BF01460020B1FA81F308BF2033A3F1CC
:101528000B03B3F120020CDA0C3208DD02F1140CC3
:10153800C2F10C0201FA0CF021FA02F10CE002F1FE
:101548001402D8BFC2F1200C01FA02F120FA0CFCF7
:10155800DCBF41EA0C019040E41AA2BF01EB045140
:10156800294330BD6FEA04041F3C1CDA0C340EDC3E
:1015780004F11404C4F1200220FA04F001FA02F381
:1015880040EA030021FA04F345EA030130BDC4F13F
:101598000C04C4F1200220FA02F001FA04F340EA34
:1015A8000300294630BD21FA04F0294630BD94F0E5
:1015B800000F83F4801306BF81F480110134013DCC
:1015C8004EE77FEA645C18BF7FEA655C29D094EA3D
:1015D800050F08BF90EA020F05D054EA000C04BFBB
:1015E8001946104630BD91EA030F1EBF00210020A6
:1015F80030BD5FEA545C05D14000494128BF41F045
:10160800004130BD14F580043CBF01F5801130BDA8
:1016180001F0004545F0FE4141F470014FF0000033
:1016280030BD7FEA645C1ABF194610467FEA655CE4
:101638001CBF0B46024650EA013406BF52EA033586
:1016480091EA030F41F4002130BD00BF90F0000F74
:1016580004BF0021704730B54FF4806404F13204B0
:101668004FF000054FF0000150E700BF90F0000F69
:1016780004BF0021704730B54FF4806404F1320490
:1016880010F0004548BF40424FF000013EE700BF60
:1016980042004FEAE2014FEA31014FEA02701FBFF0
:1016A80012F07F4393F07F4F81F06051704732F022
:1016B8007F4208BF704793F07F4F04BF41F4002179
:1016C800704730B54FF4607401F0004521F00041D7
:1016D8001CE700BF50EA010208BF704730B54FF061
:1016E80000050AE050EA010208BF704730B511F062
:1016F800004502D5404261EB41014FF4806404F19A
:1017080032045FEA915C3FF4D8AE4FF003025FEA1F
:10171800DC0C18BF03325FEADC0C18BF033202EBA3
:10172800DC02C2F1200300FA03FC20FA02F001FAFD
:1017380003FE40EA0E0021FA02F11444BDE600BFA0
:101748004FF0FF3C06E000BF4FF0010C02E000BF85
:101758004FF0010C4DF804CD4FEA410C7FEA6C5C68
:101768004FEA430C18BF7FEA6C5C1BD001B050EA0B
:10177800410C0CBF52EA430C91EA030F02BF90EAF6
:10178800020F0020704710F1000F91EA030F58BFB5
:10179800994208BF90422CBFD8176FEAE37040F017
:1017A800010070474FEA410C7FEA6C5C02D150EAB5
:1017B800013C07D14FEA430C7FEA6C5CD6D152EA70
:1017C800033CD3D05DF8040B704700BF8446104635
:1017D80062468C461946634600E000BF01B5FFF734
:1017E800B7FF002848BF10F1000F01BD4DF808ED04
:1017F800FFF7F4FF0CBF012000205DF808FB00BFD5
:101808004DF808EDFFF7EAFF34BF012000205DF82E
:1018180008FB00BF4DF808EDFFF7E0FF94BF01207B
:1018280000205DF808FB00BF4DF808EDFFF7CEFF7C
:1018380094BF012000205DF808FB00BF4DF808EDBB
:10184800FFF7C4FF34BF012000205DF808FB00BF8C
:101858004FEA410212F5001215D211D56FF47873D0
:10186800B3EB625212D94FEAC12343F0004343EA73
:10187800505311F0004F23FA02F018BF404270474E
:101888004FF00000704750EA013005D111F00040D8
:1018980008BF6FF0004070474FF00000704700BF6E
:1018A80080F0004002E000BF81F0004142001FBF0D
:1018B8005FEA410392EA030F7FEA226C7FEA236C16
:1018C8006AD04FEA1262D2EB1363C1BFD21841400B
:1018D80048404140B8BF5B42192B88BF704710F0A1
:1018E800004F40F4000020F07F4018BF404211F044
:1018F800004F41F4000121F07F4118BF494292EAAC
:10190800030F3FD0A2F1010241FA03FC10EB0C00D7
:10191800C3F1200301FA03F100F0004302D5494264
:1019280060EB4000B0F5000F13D3B0F1807F06D311
:1019380040084FEA310102F10102FE2A51D2B1F109
:10194800004F40EBC25008BF20F0010040EA0300FE
:101958007047490040EB0000013A28BFB0F5000F7E
:10196800EDD2B0FA80FCACF1080CB2EB0C0200FA34
:101978000CF0AABF00EBC25052421843BCBFD04083
:101988001843704792F0000F81F4000106BF80F4FD
:1019980000000132013BB5E74FEA41037FEA226CC0
:1019A80018BF7FEA236C21D092EA030F04D092F08B
:1019B800000F08BF0846704790EA010F1CBF0020BF
:1019C800704712F07F4F04D1400028BF40F000401C
:1019D800704712F100723CBF00F50000704700F03C
:1019E800004343F0FE4040F4000070477FEA226263
:1019F80016BF08467FEA23630146420206BF5FEA34
:101A0800412390EA010F40F4800070474FF0000333
:101A180004E000BF10F0004348BF40425FEA000CFA
:101A280008BF704743F0964301464FF000001CE0A2
:101A380050EA010208BF70474FF000030AE000BFF8
:101A480050EA010208BF704711F0004302D5404236
:101A580061EB41015FEA010C02BF844601460020A8
:101A680043F0B64308BFA3F18053A3F50003BCFAC3
:101A78008CF2083AA3EBC25310DB01FA02FC634470
:101A880000FA02FCC2F12002BCF1004F20FA02F277
:101A980043EB020008BF20F00100704702F120026A
:101AA80001FA02FCC2F1200250EA4C0021FA02F2CB
:101AB80043EB020008BF20EADC7070474FEA40029F
:101AC800B2F1FE4F0FD34FF09E03B3EB12620DD964
:101AD8004FEA002343F0004310F0004F23FA02F0CE
:101AE80018BF404270474FF00000704712F1610F75
:101AF80001D1420205D110F0004008BF6FF000404C
:101B080070474FF00000704753B94AB9002908BF21
:101B180000281CBF4FF0FF314FF0FF3000F070B9C4
:101B2800ADF1080C6DE904CE00F006F8DDF804E02C
:101B3800DDE9022304B070472DE9F047089E0D4601
:101B480004460F46002B4AD18A42944665D9B2FA18
:101B580082F343B102FA03FCC3F120029F4020FA4A
:101B680002F217439C404FEA1C4E1FFA8CF5B7FB54
:101B7800FEF1220C0EFB117742EA074201FB05F049
:101B880090420AD91CEB020201F1FF3780F01B8159
:101B9800904240F2188102396244121AA4B2B2FB90
:101BA800FEF00EFB102244EA024400FB05F5A542B4
:101BB8000AD91CEB040400F1FF3280F00681A5422B
:101BC80040F203816444023840EA0140641B00216A
:101BD8001EB1DC400023C6E90043BDE8F0878B4214
:101BE80008D9002E00F0EC800021C6E9000508465F
:101BF800BDE8F087B3FA83F1002949D1AB4202D39B
:101C0800824200F2F780841A65EB0302012017462E
:101C1800002EE2D0C6E90047DFE702B9FFDEB2FADC
:101C280082F3002B40F08F808A1A4FEA1C471FFA74
:101C38008CFE0121B2FBF7F507FB1520220C42EAC6
:101C480000420EFB05F0904208D91CEB020205F198
:101C5800FF3802D2904200F2CA804546121AA4B256
:101C6800B2FBF7F007FB102244EA02440EFB00FE29
:101C7800A64508D91CEB040400F1FF3202D2A645A0
:101C880000F2BA801046A4EB0E0440EA05409FE734
:101C9800C1F120078B4022FA07FC4CEA030C05FA35
:101CA80001F420FA07F3FD40234300FA01F94FEA53
:101CB8001C401FFA8CFEB5FBF0F81C0C00FB1855F5
:101CC80044EA054408FB0EF5A54202FA01F20BD9D5
:101CD8001CEB040408F1FF3A80F08780A54240F22B
:101CE8008480A8F102086444641B9DB2B4FBF0F33D
:101CF80000FB134445EA044403FB0EFEA64508D93D
:101D08001CEB040403F1FF306BD2A64569D9023BF2
:101D1800644443EA0840A0FB0283A4EB0E049C42FF
:101D2800C6461D4655D352D056B1B9EB0E0364EBE7
:101D3800050404FA07F7CB40CC401F43C6E90074FA
:101D48000021BDE8F087C3F1200102FA03FC20FA64
:101D580001F225FA01F19D402A434FEA1C471FFA78
:101D68008CFEB1FBF7F007FB1015110C41EA054199
:101D780000FB0EF58D4204FA03F408D91CEB0101AF
:101D880000F1FF382FD28D422DD902386144491B0A
:101D980092B2B1FBF7F507FB151142EA014205FBC8
:101DA8000EF1914208D91CEB020205F1FF3816D258
:101DB800914214D9023D6244521A45EA004139E77A
:101DC8003146304609E73946E7E61046FCE6C145A4
:101DD800AAD2B8EB020E63EB0C050138A4E745461E
:101DE800EAE7034695E74046D1E7D0467CE7023D5F
:101DF800624433E708460BE76444023843E700BF10
:101E0800704700BF1348144A08B54FF00043C0E9B3
:101E180000230422002342610122C2614FF4805151
:101E280007220383C0E90233C0E90933C0E90C1271
:101E38000361837680F8203080F82C30826380F844
:101E48003C30C36405F00AFB18B1BDE8084000F057
:101E580017BC08BDEC080020002401400268084BAC
:101E68009A4282B00AD14FF0B0431A6E42F400721F
:101E78001A661B6E03F400730193019B02B070474E
:101E8800002401400268054B9A4201BF4FF0B0425E
:101E9800136E23F400731366704700BF00240140DB
:101EA80030B585B000240546CDE901440394FFF719
:101EB800A9FF144805F06AFE08B100F0E1FB1148DB
:101EC800039401A9CDE9015405F026FC08B100F0FE
:101ED800D7FB0C4805F084FD08B100F0D1FB4FF0AA
:101EE800FF31084805F0BAFB064805F031FE054801
:101EF80005F00EFC0446034805F0D4FD204605B065
:101F080030BD00BFEC080020014B024A1A60704740
:101F1800EC0800200024014008B50948FFF7C0FF7D
:101F280068B1084BB3F8AA304FF6FF72934216BF58
:101F380040F6E442044B5343B3FBF0F398B208BDB8
:101F4800002000B40075FF1FD8084C0013B500230B
:101F5800ADF80630FFF7E0FF04461948FFF7A0FF89
:101F6800184BB3F8C820B3F8A8108A4204FB00F055
:101F780018D040F6E443B0FBF3F364205B1A434304
:101F8800521A93FBF2F31E331BB2ADF80630BDF8BC
:101F980006305BB21B02ADF80630BDF8060000B291
:101FA80002B010BD4FF47A7240F6FF73B0FBF3F342
:101FB8005343A3F53923A3F50C6340F6C412E0E7B5
:101FC800001000B00075FF1F4FF0B04382B09A6A4E
:101FD80022F480529A629A6C42F480529A649B6C02
:101FE80003F480530193019B002002B070474FF027
:101FF800B04382B09A6C02439A649B6C034001938D
:10200800019B02B0704708B50420FFF7F0FF0120DC
:10201800FFF7EDFF0220FFF7EAFF002211460B2031
:1020280005F052FE0B2005F081FE002211460C201F
:1020380005F04AFE0C2005F079FE002211460D201D
:1020480005F042FE0D2005F071FE002211460E201B
:1020580005F03AFE0E2005F069FE002211460F2019
:1020680005F032FE0F2005F061FE00221146102017
:1020780005F02AFE102005F059FE00221146112015
:1020880005F022FE112005F051FE002236201146EF
:1020980005F01AFEBDE80840362005F047BE0000EE
:1020A80008B506F08BF810B16FF0040008BD064BB8
:1020B8009A6942F040429A614CF2FA321A6106F08B
:1020C8008FF80028F2D0EFE700400058F0B585B04F
:1020D80000230C4600930646A8B3FFF7E1FF054628
:1020E80070BB06F06BF888BB1A481B4A02230193A1
:1020F800D0F8E01506F1784302EA8121B3FBF1F745
:1021080001FB1733DB0A0293D0F8E00504F17841AC
:102118000139314402EA8022B1FBF2F002FB1011CE
:10212800C3EBD1230133694601A8039306F0D8F81D
:1021380020B102280CBF01256FF0010506F050F808
:10214800284605B0F0BD6FF00505F9E76FF0040506
:10215800F6E700BF0070FF1F00FCFF03014B18608B
:1021680000207047500900202DE9F04F89B0B0F1E8
:10217800006F06460F460092C0F0C580DFF89881D0
:10218800664DD8F8E03505EA832303F10063013B87
:10219800984200F2B880002800F0B880002900F0CA
:1021A800B58040EA02035B0740F0B080FFF778FF94
:1021B8000446A0BB06F002F8002840F0AA80D8F830
:1021C800E01506F1784205EA8121B2FBF1F301FB43
:1021D8001322009B03F17843013B3344B3FBF1F036
:1021E80001FB1033DB0A01334FEAD22AA3EBD222D8
:1021F800012A039388BFC6F30A050AF58038C6F199
:10220800080398BF009D069388BFC5F500654FEA8F
:10221800C828B346039B9A4505D305F0E1FF20463D
:1022280009B0BDE8F08FA6F10803069A1A44954252
:1022380019D804950197CDF814B04FF00009059B03
:1022480009EB0301049B99453ED3009BAB442F4403
:102258005D1BB5F5006F28BF4FF400650AF1010A50
:1022680008F50068D6E753F8081F5A68B2F1FF3F2F
:1022780008BFB1F1FF3FD8D0294B186810B96FF0EB
:102288000504CAE7B8F1000F04D04FF400624146D4
:1022980011F092FBDFF88890D9F80030CBF30A00F0
:1022A80039461844AAB211F087FB4FF40061404642
:1022B800FFF70CFF08BBD9F8003001934FF4006317
:1022C800CDF814800493B8E7019B07914B4402931F
:1022D8000120D3E9002305F0BDFF88B90799019BC8
:1022E800D1E9000259F80310029B5B689A4208BFC3
:1022F800884205D109F10809A1E76FF001048CE7CC
:102308006FF0030489E74FF0FF3488E76FF00504A6
:1023180085E76FF0040482E70070FF1F00FCFF03ED
:1023280050090020B1F1006F70B511D30B4BD3F8F1
:10233800E0650B4B03EA862303F10063013B9942F6
:1023480006D840B139B192B211F036FB002070BD09
:102358004FF0FF30FBE76FF00500F8E70070FF1F54
:1023680000FCFF03B0F1006F10B40DD3084BD3F895
:10237800E045084B03EA842303F10063013B9842DC
:1023880002D810BCFFF7A2BE4FF0FF3010BC704758
:102398000070FF1F00FCFF034FF0B04382B0DA6CFF
:1023A8000243DA64DB6C03400193019B02B070477F
:1023B80070B586B01422002101A811F035FF012064
:1023C800FFF7EAFF0220FFF7E7FF0420FFF7E4FF2B
:1023D8004FF4007101224FF0904006F0F5F8012506
:1023E80002234FF4041401A94FF09040CDE90134C1
:1023F800224E039505F0C2FF4FF4441301A94FF094
:102408009040CDE90235019505F0B8FF2023CDE9CC
:10241800013401A900243046039405F0AFFF4FF4BE
:10242800007301A94FF09040CDE90135CDE903547F
:1024380005F0A4FF04230DEB03013046CDE9013577
:10244800CDE9034405F09AFF22462146062005F00F
:102458003BFC062005F06AFC22462146072005F0D1
:1024680033FC072005F062FC22462146162005F0C1
:102478002BFC162005F05AFC06B070BD000400487D
:1024880008B51248124A134BC0E900230023012261
:10249800C0E90232C0E90433C0E90633036206F03A
:1024A80007FA08B100F0ECF80848002106F080FBB4
:1024B80008B100F0E5F80548002106F09FFB18B1C7
:1024C800BDE8084000F0DCB808BD00BF140A0020D1
:1024D800005800405D3E302070B596B00546142285
:1024E800002103A811F0A0FE3822002108A811F04D
:1024F8009BFE2A68304B9A425BD18023089308A838
:102508004FF440230E9307F0D5F808B100F0B8F85F
:102518004FF0B0444FF4C050E36C43F00103E36460
:10252800E36C03F001030293029B12230026CDE91A
:1025380003030323CDE905634FF09040042303A967
:10254800079305F01BFFA36DDFF870C043F4800309
:10255800A365A36D1A4C03F480030193019B2662C3
:102568000D23C4E900C320468023C4E90266C4E9F8
:102578000436C4E9066605F039FC08B100F080F8B5
:10258800104AEC63A562104C0E23C4E90023102105
:10259800002380222046C4E90213C4E90423C4E9C5
:1025A8000633236205F022FC08B100F069F8AC6339
:1025B800A56216B070BD00BF00580040440002403C
:1025C8005409002058000240B409002000B59BB00F
:1025D8004822002108A811F027FE1822002102A88D
:1025E80011F022FE06F030FB4FF0B0420120D2F885
:1025F800903023F01803C2F89030D2F8003423F456
:10260800C06343F40073C2F80034D2F8003403F412
:10261800C0630193019B2423089381230B93002318
:10262800CDE91003B02208A8CDE9122306F084FCF6
:1026380008B172B6FEE74F23CDE90230CDE90400B8
:10264800CDE90600022102A806F010FF08B172B613
:10265800FEE71BB05DF804FB08B504F0ADFEFFF71C
:10266800B5FFFFF7A5FEFFF7CEFCFFF709FF00F067
:10267800F8FD40F6B83000F049FA00F0F9FDFCE743
:1026880072B6FEE700B58DB02C22002101A811F02A
:10269800CBFD1748174B03601F2383604FF0804220
:1026A8000023C0E90433C0E9072383614FF4807332
:1026B800436207F085F908B1FFF7E2FF0C4807F01D
:1026C800ABFA08B1FFF7DCFF4FF000530022079385
:1026D800074808924FF4807301A9029206920B935F
:1026E80007F0CEF908B1FFF7CBFF0DB05DF804FB9A
:1026F800680A00200028004010B5044690B038222F
:10270800002102A811F090FD2268194B9A422CD1A1
:102718004FF48033029302A84FF480730F9306F0AE
:10272800C9FF08B1FFF7ACFF4FF0B0430220D3F860
:10273800902042F40042C3F890209A6D42F48062DF
:102748009A659B6D002203F4806311460193019BF7
:1027580005F0BAFA022005F0E9FA00222A2011460B
:1027680005F0B2FA2A2005F0E1FA10B010BD00BF5A
:10277800002800407047000008B504F033FE044B01
:102788000120C3F88800BDE8084006F0B5BA00BFCC
:102798000004005804F02DBE08B504F02AFE00F02D
:1027A80063FCFFF705FEFFF72EFCBDE80840FFF7C6
:1027B80067BE08B504F016FEBDE8084001210020F8
:1027C80006F04ABA70477047FEE7FEE7FEE7FEE705
:1027D800FEE770477047704770470000014807F0F0
:1027E80041BA00BF680A0020012005F0F3BE0220AC
:1027F80005F0F0BE70477047014805F071BC00BF96
:1028080054090020014805F06BBC00BF400B0020B4
:10281800014805F065BC00BFE00A0020FFF7F2BFE1
:102828007047202005F0D6BE70470000014807F029
:10283800DDBD00BFA00B0020014807F045B800BF70
:10284800680A0020014807F038BC00BFCC0A002005
:102858002DE9F04389B080460020109E07908946F4
:1028680015461F46FDF7DCFCF0B9104CCDE9009089
:10287800CDE9020407AB0E480593142304933A46A6
:10288800434629460068FDF795FD2346324604F184
:10289800140153F8044B42F8044B8B42F9D1079BBF
:1028A800337509B0BDE8F0830120FAE7A00A0020DB
:1028B800304401087FB5124C00253C2302A86375FB
:1028C800CDE90255257500F0C3F8042303AA009446
:1028D80012210C48FFF7BCFF0B491422204611F0C7
:1028E80093FC0646B0FA80F0400960750090074BEB
:1028F8002A462946022010F057FF304604B070BD22
:10290800B40A0020764401084E0E002058440108FD
:10291800054808B50823036007F0EAF918B1BDE8CF
:102928000840FFF7ADBE08BDCC0A00204FF0B04309
:1029380007B55A6E42F001025A665B6E002203F038
:102948000103019311463220019B05F0BDF93220A5
:1029580003B05DF804EB05F0E9B900000CB407B565
:10296800054A05AB1021019311F030FB03B05DF867
:1029780004EB02B0704700BF8844010830B585B049
:10298800044602A80D4611F04DF9BDF90C30064A6F
:1029980000931021029B2046FFF7E0FF2046FEF738
:1029A8000BFD288005B030BD884401084FF0B042C7
:1029B80010B5936823F40043936011F0BBF90E4BF4
:1029C80001241C7000F0B6F810F084FE0B4810F0DB
:1029D8009BFE0B4B4FF400421A61204610F09AFE02
:1029E800FFF792FA00F012F910F090FF2146204606
:1029F800BDE8104010F0AABFD80A002085290008B9
:102A08000040005810F0B8BF08B5FFF785FA40F647
:102A1800B83398420CD8B0F5E16F0BD3FE23A0F57C
:102A2800E16058434FF49663B0FBF3F0C0B208BDC1
:102A3800FE20FCE70020FAE77FB5684600F0CAF8F8
:102A48000198FFF73BF800B207B05DF804FB0000FF
:102A5800194A38B5D2F88035591C044619D104F002
:102A6800CFFC054604F0D8FC054404F0CFFC2B0E3F
:102A7800E3712B0CA3712B0A6371030EE370C0F38F
:102A88000742C0F307232571C0B2A270637020709B
:102A980038BD190AC3718171190C1B0E417103717C
:102AA800D2F88435C370D2F88405C0F30722C0F386
:102AB8000743000EE9E700BF0070FF1F38B5094B58
:102AC800D3F8803503600133054609D104F098FC3A
:102AD800044604F09BFC444004F09EFC44402C60F7
:102AE80038BD00BF0070FF1F0121022010F018BF81
:102AF8000021022010F014BF00207047024B187804
:102B080008B100F0BBB87047D80A002082B0019025
:102B1800019802B000F04EB94FF0B04382B0DA6CC1
:102B280042F00202DA64DB6C03F002030193019BBA
:102B380002B070472DE9F043254C87B004F072FCD1
:102B480004F078FC04F07EFC0123002502934FF486
:102B58008059032301A9204604934FF40058039594
:102B68000595FFF7D9FFFFF7D7FFFFF7D5FFFFF769
:102B7800D3FFCDF8049005F001FC01A920464FF4DD
:102B88000067CDF8048005F0F9FB01A920464FF451
:102B98000046019705F0F2FB01A92046019605F0D1
:102BA800EDFB2A464946204605F00EFD2A464146D9
:102BB800204605F009FD2A463946204605F004FD61
:102BC8002A463146204605F0FFFC07B0BDE8F083F1
:102BD8000004004810B50446FFF7B8F9074BA36096
:102BE80040F30F20FEF716FF054B064A2360064BFD
:102BF8006060C4E90323002010BD00BF0000484204
:102C080000007A440D093E00AB0305000020704720
:102C1800014B1868704700BFDC0A0020032070478A
:102C280008B501464FF47A7200238002890DFEF739
:102C38006BFF08BD4FF47A73A0FB0303800A40EAD8
:102C480083507047034B98689A689042FBD1C04301
:102C5800704700BF0028004008B5FFF7F3FF014B9D
:102C6800186008BDDC0A002008B5FFF7EBFF024B2F
:102C78001B68C01A08BD00BFDC0A0020024B187888
:102C880008B1FFF7DFBF7047D90A002010B5074B1E
:102C9800074C0122DA654FF48071204606F0DAFD10
:102CA8004FF0FF332363002010BD00BF0028004011
:102CB800680A002002460021014806F0E4BF00BF70
:102CC800680A002002460121014806F0DCBF00BF67
:102CD800680A002010B58CB02C220021044601A8F7
:102CE80011F0A2FAFFF7D2FF0C4B0D481B681C44E9
:102CF8000023089306934FF00053E44307930122FF
:102D08004FF4807301A902940B9306F0B9FE08B141
:102D1800FFF7B6FC00200CB010BD00BFDC0A002095
:102D2800680A002038B50546FFF78CFF02210446E3
:102D3800074806F0AFFFC4F309024FF47A71A2FB0B
:102D48000121920AA30A2A8043EA805038BD00BFB5
:102D5800680A00200148002106F09CBF680A00208C
:102D68000148012106F096BF680A0020F8B50F4D0A
:102D78002E78CEB90E4C4FF0FF372763FFF782FC51
:102D8800FFF784FF4FF48071204606F063FD20466C
:102D9800276306F023FF32462046022106F073FF20
:102DA800FFF75AFF01232B700020F8BDD90A002035
:102DB800680A0020014610B54FF47A720023800299
:102DC800890DFEF7A1FE0146FFF73CFF0446FFF719
:102DD80039FF031B8B4200D310BD00BFF7E711F08A
:102DE800B1B8000010B5064C0221204606F052FF8B
:102DF8000221421C2046BDE8104006F044BF00BF37
:102E0800680A00201648174A08B54FF4E133C0E9AC
:102E1800002300230C22C0E90233C0E90523C0E9DE
:102E28000733C0E90933036108F0C1F808B1FFF7B7
:102E380027FC0B48002108F036FA08B1FFF720FC00
:102E48000748002108F04FFA08B1FFF719FC0448B9
:102E580008F009FA18B1BDE80840FFF711BC08BD31
:102E6800A00B00200044004070B596B0054614221F
:102E7800002103A811F0D8F93822002108A811F080
:102E8800D3F92A68334B9A4261D10223089308A8E0
:102E9800314B0A9306F00EFC08B1FFF7F1FB4FF037
:102EA800B0430C219A6D2D4C42F400329A659A6D0C
:102EB80002F400320292029ADA6C42F00102DA64F9
:102EC800DB6C03F001030193019B02230026CDE98B
:102ED80003130323CDE905634FF09040072303A9AB
:102EE800079305F04BFA1E4826621423C4E9000331
:102EF8001023C4E9023620468023C4E90436C4E915
:102F0800066604F073FF08B1FFF7BAFB154AEC67D1
:102F1800A562154C1323C4E9002320460023802210
:102F2800C4E90233C4E90423C4E90633236204F084
:102F38005DFF08B1FFF7A4FB2520C5F880400022FB
:102F48000221A56204F0C0FE252004F0EFFE16B0B1
:102F580070BD00BF0044004004000C00400B00207E
:102F6800800002406C000240E00A002002680E4B1C
:102F78009A4210B5044616D14FF0B0420C21936D19
:102F880023F4003393654FF0904005F0A3FAE06F07
:102F980004F0A0FFD4F8800004F09CFFBDE81040C6
:102FA800252004F0D1BE10BD0044004008B50A46F3
:102FB8000146024807F07EF9002008BDA00B00205A
:102FC80013B5114B114C18604FF40013009302AB6A
:102FD80013E90600204608F0EAF82368DA69D10305
:102FE800FCD4DA695202FCD59A68084842F4800297
:102FF8009A6008F022F906490448012208F090F87E
:10300800002002B010BD00BF340C0020A00B00202F
:103018003C0C002008B5074B1860FEF7F4FFFFF7DB
:10302800F1FE054AD2F8803043F00063C2F88030E0
:10303800002008BD380C00200008005808B54FF0E3
:10304800B04308489A6B42F400329A639A6B22F4B0
:1030580000329A63FFF78AFF0F2004F075FE002004
:1030680008BD00BFA00B002008B5074807F09FFF68
:1030780008B1FFF705FB054804F0B8FE18B1BDE834
:103088000840FFF7FDBA08BDA00B0020400B002048
:103098000268044B9A4203D1034B00201B6818476F
:1030A800704700BF00440040380C002002680B4BFA
:1030B8009A4210B504460FD1094B1B682BB1D0F8C2
:1030C800902012B907480121984720460549BDE8D4
:1030D8001040012208F024B810BD00BF0044004091
:1030E800340C00203C0C002002480122102105F07D
:1030F8006BBA00BF0004004802480022102105F006
:1031080063BA00BF0004004813B5134C23785BB9B9
:10311800E37C03F0FF023BB9104B1146022002B0DA
:10312800BDE8104010F040BBFFF7C4FB00380C4B63
:1031380018BF0120400018701A78022A02BF002226
:103148002270E2741B7800930022064B114603207C
:1031580010F02AFB02B010BD4E0E0020E444010816
:10316800440C00200045010838B5184C23785BBB97
:10317800E37C03F0FF023BBB154D2B68012B0CD9F8
:103188002B68042B09D81146124B022010F00CFBB7
:10319800114A0421012000F075FB2B68042B13D978
:1031A80000220E4B1146022010F0FEFAFFF782FBB8
:1031B80000380B4B18BF0120400018701B78022BF9
:1031C80002BF00232370E37438BD00BF4E0E0020F9
:1031D800400C0020174501083C45010841450108FD
:1031E800440C002008B5FFF77FFF0022054B11466D
:1031F800032010F0D9FA01F011FDBDE80840FFF7EF
:103208007BBF00BF74450108022801D8FFF76CBFD7
:103218007047022801D8FFF76FBF7047022808B52A
:103228001BD8012210210D4805F0CEF93220FFF7F6
:103238006DFC0A480022102105F0C6F90122102170
:10324800064805F0C1F93220FFF760FCBDE80840E8
:1032580002480022102105F0B7B908BD0004004853
:10326800704708B5FFF7A2FBBDE8084000F0D4BCE2
:103278004FF0FF3010F0E4BB70477047014BD87037
:10328800704700BF5C000020014B1874704700BFF6
:103298005C00002007B5064B00221B5C009311461A
:1032A800044B022010F080FA03B05DF804FB00BF65
:1032B800B04501089645010808B50220002110F024
:1032C80087FBBDE80840014810F0EABD9C0D0020CE
:1032D8000021012010F07CBB13B50D4CA0B120607B
:1032E8000C4810F08FFD21680A4810F013FE0948B9
:1032F80010F0D6FD236800930022074B11460320E7
:1033080010F052FA02B010BD42F210732360E7E7E2
:10331800740000209C0D0020B445010813B50D4C25
:10332800206023680BB90C4B23600C4810F06AFD31
:1033380021680A4810F0EEFD084810F0B1FD236836
:1033480000930022064B1146032010F02DFA02B01C
:1033580010BD00BF0C000020A0860100B40D0020A5
:10336800DD45010837B5044600283AD090F90650E3
:10337800002D38D11F4810F045FD2A4629461E4B1E
:10338800022010F011FAE379012B0CBF1B4B1C4BE8
:103398002A46294602201B4D10F006FAE3792B70C5
:1033A800194B1868FFF7BAFF184B1868FFF794FF16
:1033B8002978174A174B012918BF13460022009392
:1033C8001146154B032010F0EFF994F905300193DD
:1033D80094F9043000930022104B1146022010F09B
:1033E800E3F903B030BD00220D4B1146022010F066
:1033F800DBF9EAE7380D00202246010837460108C4
:1034080054460108680D00200C00002074000020BC
:103418001D4601081946010871460108A946010818
:103428009046010838B504460D4607484FF4006138
:10343800FEF798FF30B92A4621460348BDE83840D0
:10344800FEF792BE38BD00BF00F003080A460149E6
:10345800FEF768BF00F0030870B5164810F0D2FCFC
:1034680008F09AFB044650B10022134B1146022083
:1034780010F09AF9BDE87040104810F011BD104DD9
:10348800104B02460146022010F08EF901260E4B21
:103498002E7022462146022010F086F90B4808F0CB
:1034A8001FFA2878314608F049F8024810F0F8FC6D
:1034B800E0E700BF9C0D0020D24601086C0D0020FB
:1034C80000000020F0460108044701085C000020C5
:1034D80030B587B0FFF798FA002104464FF48070A2
:1034E80010F076FA02A801F0AFF923B203EB430318
:1034F800FE2203EB4313B3FBF2F33C4A0B2111709A
:103508003B4950680978DBB28DF814300170546873
:103518000020607054681A25A57054680125E5706C
:1035280054682371334B1C7844B118700C23137002
:10353800536861F07F011970052314E02E4B2F4862
:10354800197811B901780029F6D000210170197095
:10355800536802215971BDF808305168180A8871FA
:103568005168CB7108232649264C0978012988BF60
:1035780000235370637A33B107F082FF012802D128
:10358800204610F03FFC204B1848D978002208F05C
:1035980063F80446A8B901461C4B0122032010F029
:1035A80003F91B4810F02EFC1A4B19481968A14260
:1035B80038BF214610F0AEFC154810F071FC07B07A
:1035C80030BD063410D107F055FF04460028E8D076
:1035D80001224FF47A730021B0FBF3F310460093F5
:1035E8000D4B10F0E1F8DCE70024DAE704000020D6
:1035F800370D0020CC0D0020630E00204D0E00205A
:10360800440C0020380D00205C00002023470108EE
:103618009C0D0020740000203247010800B50346C5
:103628008DB000282CD0407802280AD003282AD050
:10363800164B0022114602200DB05DF804EB10F085
:10364800B3B8DA7E0B929A7E0A925A7E09921A7E53
:103658000892DA7D07929A7D06925A7D05925A68F9
:103668000492DA68039293F914200292B3F91220B3
:1036780001921B7C00930022054B114610F094F830
:103688000DB05DF804FB034BD3E700BF50470108BA
:1036980067470108D947010801284FF000020CBF0D
:1036A800024B034B1146022010F07EB8F847010880
:1036B8000A4801081FB50446002831D00378002BBA
:1036C8002ED01D4810F0ECFB002211461B4B0220A7
:1036D80010F06AF894F91830039394F90A300293B9
:1036E800237C0193E368009300221146144B0320C6
:1036F80010F05AF80022134B1146032010F054F82A
:10370800237A012B0ED1617A0F4A104B002908BF8A
:1037180013460022009311460D4B032010F044F885
:1037280004B010BD00220B4B1146032004B0BDE8C5
:10373800104010F039B800BF840D0020234801085C
:1037480054480108854801081E4801081F48010817
:1037580092480108A348010808B5104B012200212E
:1037680002201A7010F034F90D4810F099FB0D4B37
:103778001B788BB10C4B1A7872B9DB7C63B90B4B95
:103788001A68042A9EBF1A6801321A600021BDE82F
:103798000840102010F01CB908BD00BFCC0D002057
:1037A800B40D0020680D00204E0E0020400C0020B3
:1037B800044B1B78022B03D10021082010F008B914
:1037C800704700BF0000002008B508F0EEF980B986
:1037D80007F056FE01280CD1BFF34F8F0549064B61
:1037E800CA6802F4E0621343CB60BFF34F8F00BF97
:1037F800FDE708BD00ED00E00400FA0510B508F08B
:1038080069FA10F1080F07D1064B0022BDE81040F5
:10381800114602200FF0C8BF013001D1024BF4E776
:1038280010BD00BFB1480108C7480108704770477C
:10383800022813B5014618D0202819D001281AD11A
:103848004FF0904004F0BAFE0022044600900B4B63
:10385800114603200FF0A8FF012C0CD100210220F3
:1038680002B0BDE8104010F0B3B800210820F7E717
:10387800034B01221A7002B010BD00BFDF480108D7
:10388800C80E002073B505460C46164607F0C6FE5E
:103898000346002838D00024264810F0B3FA264BF7
:1038A80024481968A14238BF214610F033FB21484B
:1038B80002B0BDE8704010F0F3BA4A68F05CD0542A
:1038C8000133DAB2A242F8D31C4B0D701B78012BDE
:1038D80088BF00244C701A4C637A33B107F0D0FDCE
:1038E800012802D1204610F08DFA164B1648D978D7
:1038F800002207F0B1FE044640B90146134B0122ED
:1039080003200FF051FFC7E70F49DAE70634C2D1A9
:1039180007F0B0FD04460028BED04FF47A730122A8
:10392800B0FBF3F3002100930320094B0FF03CFF99
:10393800B2E700BF9C0D002074000020440C00205A
:10394800380D00205C0000200400002023470108F7
:1039580032470108044B1B7823B9044A052101208A
:10396800FFF790BF704700BF440C0020FD480108D6
:1039780010B5002490B03C22214601A8009410F014
:1039880053FC2F4B2022DA7219788DF800105978E1
:103998008DF8011099788DF80210D9788DF80310F8
:1039A80019798DF8041059798DF8051099798DF8E1
:1039B8000610D9798DF80710197A8DF80810597AF8
:1039C8008DF80910997A8DF80A108DF80B20214688
:1039D8000DF10B0258180131007B02F8010F1C2968
:1039E800F8D193F828208DF8282093F829208DF80D
:1039F800292093F82A208DF82A2093F82B208DF877
:103A08002B2093F82C206AB193F83F2052B10DF186
:103A18002B0100229818013290F82C0001F8010FB0
:103A2800142AF7D107484FF40061FEF79BFC20B930
:103A3800044840226946FEF797FB10B010BD00BF4E
:103A48007800002000F80308014940220FF0B4BFB5
:103A580000F8030870B52A4D28796B794D2BC0B250
:103A680033D1C0EB001080000A2838BF0A204FF479
:103A78007A735843234BAC791860EB794D2BE4B239
:103A88002BD1C4EB0414A40095F82C301E4E63BB54
:103A980095F83F304BBB42F21070FFF71DFC3068C1
:103AA800FFF73CFC2B7A194A1949DBB213706B7A81
:103AB800184ADBB213700023EA1892F82C20D2B20D
:103AC800CA540133142BF7D170BD6B79482B0ABF48
:103AD8004FF461636B795843C6E7EB79482B0ABF0B
:103AE8004FF46163EB795C43CEE7FFF7F5FB012CFC
:103AF80038BF01244FF47A735C433460CFE700BFCA
:103B080078000020740000200C000020620E0020C5
:103B18004E0E0020440C002010B590B000213C222D
:103B280001A8009110F080FB4022374968460FF049
:103B380043FF9DF800203AB99DF801001A2803D1E7
:103B48009DF80210012914D0002211462F4B0320A2
:103B58000FF02AFEFFF70CFF2D48142200210FF06A
:103B680035FF4FF47A70FEF7D1FFFFF773FF10B0FF
:103B780010BD284B1A70587099709DF80310D970B1
:103B88009DF8041019719DF8051059719DF80610DB
:103B980099719DF80710D9719DF8081019729DF850
:103BA800091059729DF80A1099729DF80B1001F0CE
:103BB8003F01D972D87AD1B288421BD89DF8282003
:103BC80083F828209DF8292083F829209DF82A20A9
:103BD80083F82A209DF82B2083F82B200DF12B0148
:103BE80000229818013211F8014F80F82C40142A4D
:103BF800F7D1BAE701F140006844194410F8340CD1
:103C080008730132D6E700BF00F80308034901082A
:103C18004E0E002078000020F0B50B238BB00A224E
:103C280000240125CDE9063203271A231721CDE9FF
:103C3800043122465F4B03942146CDE90155009794
:103C4800284609940FF0B0FD5B4B009522462146AB
:103C5800CDE9017402200FF0A7FD02260523CDE966
:103C680000632246554B0294214630460FF09CFDD6
:103C7800534B009522462146CDE9017430460FF09A
:103C880093FD09A9204607F073FF099BC3F3072298
:103C98000292C3F307421B0E019200932246494B3E
:103CA800214630460FF080FD09A9284607F060FF3D
:103CB800099BDAB20392C3F307220292C3F30742C5
:103CC8001B0E0192009322463F4B214630460FF0CF
:103CD8006BFD3E4B3E48009422464FF4FA7110F0BB
:103CE80033F83C4B3C48009422464FF4FA7110F0EC
:103CF8002BF83A4B3A4800942A464FF4FA7110F0E0
:103D080023F82046FEF72AFA08B1FEF7B9FC354B2E
:103D1800009400224FF4FA61334810F015F8334A42
:103D2800002101200FF010FF314A002102200FF07E
:103D38000BFF304A002104200FF006FF2E4A002115
:103D480008200FF001FF00F005FC2C492C4807F073
:103D5800D1FE2C4807F0C4FD214810F0A1F82A4BE9
:103D68000021187807F0EAFB28490094284B0968D5
:103D7800284800220FF0E8FF264810F091F8FFF7D6
:103D8800CBFE254A002110200FF0DEFE234A002139
:103D98004FF480700FF0D8FE214B22481968224B4F
:103DA800009400220FF0D0FF1E4810F079F80BB0F5
:103DB800F0BD00BF454901088C490108AD4901081B
:103DC800CE490108EF490108104A0108813200086C
:103DD800840D002037380008500D002035380008C1
:103DE800380D0020B93700086C0D002041B40008D8
:103DF800D9340008053800086134000800000301C0
:103E0800100000205C00002000000020740000204A
:103E1800C13200089C0D002071310008ED31000806
:103E28000C000020B40D00206137000830B50024D4
:103E3800A5B021467C2205A8049410F0F5F9532377
:103E48008DF810304FF48D73ADF812300123ADF8B2
:103E58000C408DF81430FEF7D7FD00B200EB40009F
:103E6800FE2300EB4010B0FBF3F08DF8150003A81B
:103E780000F0FAFC2246009021461C4B0546032020
:103E88000FF092FC07249DB958238DF81630302284
:103E98008021174810F0C8F9224604A9144810F0E8
:103EA800FCF9134A21460120FFF7ECFC25B030BD90
:103EB8008DF816408DF8175000F0B0FE0D4B1A68BB
:103EC80012128DF818201A688DF819205A681212E3
:103ED8008DF81A205A688DF81B209A689B688DF80F
:103EE8001D3012128DF81C200E24D0E7344A010828
:103EF800CD0D0020F40E0020F0B50378592B95B0B5
:103F0800044640F0108205295FD84378443B162BBD
:103F18005BD8DFE813F034015A0024015A002C0161
:103F28005A005A005A005A008E005A000F015A00CF
:103F38005A005A00AB015A005A00B2005A005A00FF
:103F48005A0017008578482D17D1BC4A1421012042
:103F5800FFF798FC41F28830FEF7D8FD0022B84BF5
:103F6800114603200FF020FC40F6B830FEF7CEFDD6
:103F780015B0BDE8F040FFF727BC532D0ED1302215
:103F88008021B04810F050F9FFF750FF41F2883017
:103F9800FEF7BCFDAB4A1521012083E0432D16D165
:103FA800002404A88DF8104007F0FEFBA54A4C2316
:103FB80013701A2393709DF8103054700120413308
:103FC800D07013710521FFF75DFC15B0F0BD442DCD
:103FD800FBD19C4C592323705A236370A57000F0C1
:103FE80024FC2C228021201D10F01EF900232570AE
:103FF800637001251A23A370E5702571FEF704FD8F
:104008009149FE23B0FBF3F04B6864229BB2B3FBEB
:10401800F2F3A3714B6800EB40009BB200EB401039
:10402800B3FBF2F102FB11336071E3712246082100
:10403800B2E78378303BDBB2092BC6D8834C844A7D
:1040480023702378DBB253727E4A592313704D23B1
:10405800537023783033937003210120FFF712FC4B
:104068002378009300227B4B114601200FF09CFB24
:1040780015B0BDE8F040FFF77BBC8578482D16D118
:10408800704A56231370002353701A239370032326
:104098001371172353710B23012093710A23D070D6
:1040A800D371082115B0BDE8F040FFF7EBBB432DF5
:1040B8008BD1644C00213C2205A8049110F0B4F87F
:1040C80004A8FFF7C1FC2422802104F10C0010F0A1
:1040D800ABF89DF8103063709DF81130A3709DF80F
:1040E8001230E3709DF8133023719DF8143063711A
:1040F8009DF81530A3719DF81630E3719DF81730BF
:1041080023729DF81830257063729DF81B509DF836
:104118001930A3729DF81A30E3722A4607A925734D
:1041280004F10D0010F0B9F805F10D012246C9B2ED
:10413800012048E7807839280CD83038C0B2FFF71A
:1041480063F8404A2378137063785370A3789370A8
:10415800032121E715B0BDE8F040FFF7FBBB8078ED
:104168003928F7D83038C0B2FFF753F8E9E7807834
:104178003928EFD83038C0B2FFF750F8E1E7837834
:10418800303BDAB2092AE5D8C578303DEAB2092AC7
:10419800E0D80179A1F14802D2B20B2ADAD82E4828
:1041A80040FA02F2D007D5D40A224D2902FB035562
:1041B8003FD13C235D43294B4FF47A706843186024
:1041C800274B1860FFF788F81E4A23781370637826
:1041D8005370A3789370E378D37023791371052112
:1041E8000120FFF74FFB1A4B1A2200261E705A7047
:1041F80001229A70DA70A178303901EB8100E178F8
:10420800303901EB4001C9B2197122795A71154A46
:104218001278D2B21A720D4A1278D2B25A72FFF7D5
:10422800A7FB114B00953246314603200FF0BCFA2C
:10423800CBE64829BFD14FF46163BBE7414A010887
:10424800564A0108CD0D0020F40E0020440C002031
:1042580078000020784A0108DEF7FFFF740000208C
:104268000C000020620E0020A14A01088378303B30
:10427800DAB2092A3FF66EAFC578303DEAB2092AAC
:104288003FF668AF0179A1F14802D2B20B2A3FF696
:1042980061AF734840FA02F2D2073FF55BAF0A22DA
:1042A8004D2902FB035539D13C235D436D4A4FF438
:1042B8007A736B4313601068FFF730F86A4A237803
:1042C800137063785370A3789370E378D37023796D
:1042D800137105210120FFF7D5FA644B1A22002635
:1042E8001E705A7001229A70DA70A178303901EB89
:1042F8008100E178303901EB4001C9B29971227926
:10430800DA715B4A1278D2B21A725A4A1278D2B269
:104318005A72FFF72DFB584B009584E74829C5D101
:104328004FF46163C1E7502B5DD102297FF64DAE92
:104338004378303B012B3FF648AE8378312B7FF42E
:1043480044AE0B2904D8FFF705FB0021464A23E6B3
:10435800464D4A4F0234002614F8012FA919303A65
:10436800D2B20A730B7BCDE9026323780022CDE930
:10437800006311463B46032001360FF015FA0C2E58
:10438800EAD1FEF76DFF384B50221A701A229A7044
:10439800002401225C70DA7003F8042F2A19013412
:1043A800127B0C2C02F1300203F8012FF6D1002207
:1043B8005023114600930320314B0FF0F5F90023E9
:1043C8002B701A236B700123AB70EB70284B1B7892
:1043D800DBB22B72274B1B78DBB26B72EC72FFF7E8
:1043E800C7FA1121B2E7412B7FF4EFAD4378432B95
:1043F8007FF4EBAD16297FF4E8AD224D421C002373
:1044080012F8011FE9540133142BF9D1FEF77CFE91
:104418001D4B5B7D012B19D114490023EA5CC81898
:104428000133D2B2142B80F82C20F7D1114B002283
:104438001A701B78DBB24B72FFF79AFA0A4A631EAE
:1044480015349C4206D1084A1621A5E5094B0222DB
:104458001A70F3E713F8011F02F8011BF1E700BF18
:10446800DEF7FFFF0C000020CD0D002078000020B3
:10447800620E0020440C0020D84A0108234B010892
:104488004B4B01084E0E0020B40A002070B50546BB
:1044980086B00C4600293BD028480FF001FD26784D
:1044A800EEB1002D48D068682E78C0B1032E0BD02D
:1044B8000B2E2FD0022E12D1697801290FD00B06AE
:1044C8000DD4FFF719FD0AE06B78012B07D10078AE
:1044D800012802D0022800D008B906F0E5FF237CA5
:1044E800052B15D894F90A20059294F9092004920D
:1044F800134A52F82330039394F90830CDE9016345
:104508000022E368009311460E4B03200FF04CF98C
:1045180006B070BD6B78012BE1D102780A4B02F02E
:1045280001021A702AB9094B114603200FF03CF911
:10453800D5E7074B0022F7E72E46D0E7500D0020BD
:10454800D04B0108794B0108370D0020664B010854
:10455800704B0108034B0022C3E902220122C3E980
:1045680000227047640E002000487047640E002047
:104578004FF0B04382B0DA6C0243DA64DB6C03407C
:104588000193019B02B070472DE9F04186B00024E9
:104598000220154D0594FFF7EBFF0420FFF7E8FF15
:1045A800124F03944FF4807601230DEB0001CDE9FF
:1045B80001632846032304934FF4005803F0DEFEFA
:1045C80001A93846CDF8048003F0D8FE22464146BA
:1045D800384603F0F9FF28462246314603F0F4FF37
:1045E800204606B0BDE8F0810004004800080048F5
:1045F800032810B50ED8012810D868B902460B4810
:104608004FF4807103F0E0FF002209484FF4005195
:1046180003F0DAFF002010BD0122F0E70022034872
:104628004FF4807103F0D0FF0122EEE70004004848
:10463800000800480220704700207047012070479A
:1046480000280CBF0F201620704700000D48854633
:1046580002F0B0FE0C480D490D4A002302E0D45880
:10466800C4500433C4188C42F9D30A4A0A4C0023B4
:1046780001E013600432A242FBD30FF0DDFDFDF729
:10468800EBFFFEE70000012000000020CC0800201E
:1046980084590108CC080020382E0020FEE74FF08E
:1046A800B04382B0DA6C42F00102DA64DB6C03F0EA
:1046B80001030193019B02B07047000030B587B039
:1046C800FFF7EDFF4FF4805101224FF0904003F0C7
:1046D8007BFF01224FF400614FF0904003F074FF1C
:1046E8004FF4C0551123CDE9015301A901234FF01F
:1046F8009040039303F042FE08240A2500224FF459
:1047080080514FF0904003F05FFF0120FEF7FEF963
:1047180001224FF480514FF0904003F055FF0120E3
:10472800FEF7F4F9013DE9D14FF400614FF09040F4
:1047380003F044FF08B9013CDFD14FF400614FF0AA
:10474800904003F03BFF68BBFFF7A9FF0424012357
:10475800039001A92A48CDE9014303F00FFE284C34
:1047680001220421204603F02FFF2120FEF7CEF975
:1047780000220421204603F027FF2120FEF7C6F976
:1047880001220421204603F01FFF2120FEF7BEF975
:1047980020460022042103F017FF4FF42570FEF78E
:1047A800B5F9DDE7FFF77BFF4FF0B04300249A6DC2
:1047B80042F480029A659B6D03F4800300934FF4E2
:1047C800C052009B1223CDE901230323CDE9034303
:1047D80004230DEB03014FF09040059303F0CEFD49
:1047E80008480949094B8460C0E900130123C0E95E
:1047F8000334C0E90744446104F05AF807B030BDF7
:1048080000040048740E0020005800401A091020C7
:10481800FFF754BF40B94B1E5A425A414FF400713A
:104828004FF0904003F0D0BE704708B50120FEF766
:10483800EBFC6420FEF76AF900F0F0F9BDE80840E7
:104848000120FEF7E6BC0000054B1A6802805A6892
:104858009B684381034B028101221A70704700BF95
:10486800F40E00204D0E002030B585B0044600F04F
:1048780017F810F0FF051FBFEE232370AA236370FB
:104888006378029323780022CDE900531146034B45
:1048980003200EF089FF284605B030BDE84B01081B
:1048A8002DE9F04F0025484E484C356089B029461F
:1048B8002846FFF7AFFF29460120FFF7ABFF29463F
:1048C8000220FFF7A7FFDFF80881DFF80891424FC1
:1048D80094F86401522301214FF0000A84F86031F2
:1048E800C4F868A1FFF796FF0320FEF70FF95246B8
:1048F8008821204602F0C4FC0DF11E02C02120468A
:1049080002F00CFD024650B1344B524611460320CA
:104918000EF04AFF0021E8B2FFF77CFF3DE0BDF84A
:104928001E304EF6AA618B424AD14FEA450A0AF177
:10493800540A5FFA8AFA05905146204600F006FAB2
:10494800834610B1264B059AE0E70DF11E02C021FF
:10495800204684F860A102F0E1FC824610B1214BA8
:104968005A46D3E7204600F0B5FB0246F0B9316855
:104978000123194431603968C4F86831AB400B43EE
:104988003B60029394F860310193D4F8643100934A
:104998000146154B03200EF007FF0135032D04F5E2
:1049A800C87495D1306809B0BDE8F08FBDF81E30E5
:1049B800009352464B46114603200EF0F5FEA9E738
:1049C80000934346F7E700BFEC0E0020BC00002030
:1049D800BD4C0108A24C0108E80E00200B4C010850
:1049E8001D4C0108404C0108594C01082DE9F04FB5
:1049F8004FF4804387B04FF49012CDE90232684CEF
:104A0800DFF8A0A1DFF8A0B105464FF00A094FF082
:104A18000E0848F2E8070026D4F86831002B00F0A9
:104A2800AE800022614B0096114603200EF0BCFEBA
:104A3800204600F043FE28B100225D4B11460320BA
:104A48000EF0B2FE0DF112020DF11101204600F038
:104A5800EFFB28B100225346114603200EF0A4FEB6
:104A68000DF1130205A9204600F02DFF28B1002200
:104A7800504B114603200EF097FE0021204600F00F
:104A880069F928B100224C4B114603200EF08CFE28
:104A980001220021204600F021FA28B10022474BCC
:104AA800114603200EF080FE01221146204600F038
:104AB80015FA28B10022414B114603200EF074FE6E
:104AC800022D65D83E4B33F8153002933D4B53F811
:104AD800253003933C4B53F825703C4B13F8058065
:104AE8003B4B13F80590029A0121204600F041FA49
:104AF80028B10022374B114603200EF055FE039AC9
:104B08000021204600F035FA28B10022314B114629
:104B180003200EF049FE3946204600F035F928B149
:104B280000222D4B114603200EF03EFE4246002186
:104B3800204600F02BF928B100225B4611460320DD
:104B48000EF032FE4A460121204600F01FF928B136
:104B580000225B46114603200EF026FE0DF11202DC
:104B68000DF11101204600F063FB28B100225346E5
:104B7800114603200EF018FE0123C4F87C310136DB
:104B8800032E04F5C8747FF447AF07B0BDE8F08F73
:104B98000022124B114603200EF006FEA3E700BFC9
:104BA800BC000020144D01080D4E0108CF4C01082F
:104BB800F94C01083A4D0108634D0108814D01087F
:104BC800E84E0108F04E0108FC4E0108084F0108A4
:104BD8000B4F0108B34D0108D64D0108A54D01083A
:104BE80010B50B7E9BB9D0F87C21098912B1C0E9B8
:104BF8005E1310BD084BD0F878411A68C2F580736F
:104C08004B4304FB02331B12C0F87831F1E7012350
:104C1800C0F87C31EDE700BFB80000202DE9F04F67
:104C2800DFF80491414E87B0FFF7F2FDD9F8003064
:104C38000BB133684BB9FFF733FE002230603C4BB1
:104C48000090114603200EF0AFFD3368394D002463
:104C5800A3422C606C60AC605BDDDFF8DC80374E13
:104C6800DFF8DCA02046FFF7C1FE88F80040D6F840
:104C780068B1BBF1010F35D10BFA04F304930A278D
:104C88002F49304600F07AFCC8B9059051463046A5
:104C9800FFF7A6FF9AF81830059A002B3CD1D6F8F2
:104CA800783145F82430049AD9F800301343C9F80C
:104CB800003098F8003043F0010388F800300120F4
:104CC800FDF724FF9AF818301BB1013F17F0FF07D2
:104CD800D6D1D6F8783140F6C412002B08BF134657
:104CE80045F8243005200134FDF710FF032C06F5A4
:104CF800C876BCD198F800305BB12B686A68A9689F
:104D08000093CDE9012100220E4B114601200EF03F
:104D18004BFD07B0BDE8F08FCDE9004B0A4B1146BB
:104D280003200EF041FDCAE7E80E0020F00E002037
:104D3800A94E0108F40E00204D0E0020BC000020F2
:104D4800CC0E00205A4E0108C74E01084A088A2195
:104D580002F096BA152906D8044BCB40DB0702D5DA
:104D68000174002070476FF0070070470B00300097
:104D780010B50A460C46092102F0A4FA18B923789E
:104D880003F00103237010BD01F06BBE01F053BDA9
:104D980001F04DBEF7B500230C46174601210DF171
:104DA800070206468DF8073002F08CFA0546D8B996
:104DB800012F9DF8073026D1042C3AD8DFE804F0FB
:104DC80003171A1D200043F01004A3420CD02246FA
:104DD8000121304602F054FA054628B9716986F86F
:104DE80030413046FFF7D0FF284603B0F0BD43F00E
:104DF8002804EAE743F00404E7E743F04004E4E763
:104E080043F08004E1E7042C13D8DFE804F003063C
:104E1800090C0F0003F0EF04D7E703F0D704D4E739
:104E280003F0FB04D1E703F0BF04CEE703F07F04EF
:104E3800CBE76FF00305D7E713B500230C460DF158
:104E4800070201218DF8073002F03CFA78B99DF885
:104E58000730C3F300122270C3F3C002A270C3F379
:104E680080026270C3F38012DB09E270237102B022
:104E780010BD37B50D460DF10202F821044602F0C7
:104E88004DFA70B901AA0421204602F067FA40B928
:104E9800BDF802201AB1019BB3FBF2F32B602B681B
:104EA800A36103B030BD037F0B700020704737B596
:104EB8000D460DF106022021044602F02FFA28B90A
:104EC800BDF8063023B9236A2B60207703B030BDC4
:104ED800DB002B60236201232377F7E70529F8B568
:104EE80004460E46154635D862B100EB8103012110
:104EF8005A6B0023701E042807D8DFE800F00E174D
:104F08001A1D240011460123F4E784F828103444BC
:104F1800E5B984F82850002007E0C2F34F22442165
:104F2800204602F0BDF90028F1D0F8BD84F82A1017
:104F3800EDE784F82B10EAE75B00FE2260212046AB
:104F480002F0D5F9EFE71B01EF22F7E7012384F818
:104F58002830E0E76FF00300E7E7052996BF40181F
:104F6800002390F82830137094BF00206FF00300DE
:104F7800704770B54318044693F828000E46154646
:104F880018B904EB8106726370BD05291BD8DFE8E8
:104F980001F0030912141616626304EB860400205C
:104FA8006563F1E7C2F34F224421204602F078F905
:104FB8000028E9D1F1E7E263EFE72264EDE7C2F305
:104FC8004F226421F1E76FF00300DDE737B50446AF
:104FD800154605292CD8DFE801F0030717191B1B14
:104FE800436B2B60002021E00DF10602442102F002
:104FF80095F9D8B9BDF8062053029AB12B60A3637E
:10500800012384F8293011E0C36BEAE7036CE8E771
:105018000DF10602642102F081F938B9BDF80630B5
:105028005B02DEE7A36B2B6084F8290003B030BD78
:105038006FF00300FAE737B50D460DF107020121BD
:10504800044602F03FF938B99DF8073084F830314A
:10505800DB092B7084F84C3003B030BD2DE9F843E0
:10506800037C0C4601F8083B0546FFF702FF40BBEE
:10507800207304F110012846FFF719FF08BB04F15B
:105088001401284600F021FCD8B904F1240705F1E1
:10509800270904F1170806463A46B1B22846FFF731
:1050A80095FF70B9013619F8013F08F8013F062E3F
:1050B80007F10407F0D104F13C012846FFF7BBFFD4
:1050C80008B1BDE8F883211D2846BDE8F84301F082
:1050D80030BD0000F0B50022054693B0882102F0EB
:1050E800CFF84FF47A72A5F852214FF4C872A5F898
:1050F80054214C4AC5F8582100234B4A85F8F03012
:10510800C5F8D4202B6202A92846FFF7A7FF04465A
:1051180070B9ADF8080002AE0FCE05F110070FC741
:105128000FCE0FC70FCE0FC796E80F0087E80F0006
:105138003E4BC5F834314FF4FA730126A5F83831DF
:105148004FF42063A5F83C313246802185F8506140
:10515800284602F095F832460746FF21284602F015
:105168008FF8002211460743284602F089F83C438D
:1051780064B204430DF107029121284602F0A2F817
:1051880064B29DF8073085F83A310443324600216D
:10519800284602F075F864B204430022FF2128462D
:1051A80002F06EF864B2044300228021284602F01F
:1051B80067F864B2204340B2002488BBA1B2012240
:1051C80028460134FFF78AFE062CF6D140BB044678
:1051D8006885024604212846FFF780FE00BB024688
:1051E80005212846FFF77AFED0B94FF490136B6378
:1051F8004FF4804201212846FFF7BBFE80B94FF4E7
:105208000C13FF22C5E90F3085F83021012128460B
:1052180002F036F8012385F8323108B985F81541CE
:1052280013B0F0BD856B0100A4700900640084030D
:10523800012300F079BD2DE9F0428EB00C460C2315
:1052480004AA1421054602F005F8844600286CD10A
:105258009DF81A309DF81B609DF817209DF81810CE
:10526800A07506EB03269DF81630206002EB03229A
:105278009DF81930606003EB01239BB25B029DF837
:10528800121023619DF81330B5F8520103EB012386
:1052980092B252029BB2E260A382B0F57A7F9DF887
:1052A800101095F83171B6B20AD0704300F5FA7053
:1052B8004FF47A76B0FBF6F02E7F002E39D186B205
:1052C800002F40D0B001C0B2B608E0750DF10F0054
:1052D8002681CDE90040284601F086FE844620BBA1
:1052E8009DF80FE084F818E005F150060FCE07AFDF
:1052F8000FC796E80700E37D87E80700D4E90301B4
:10530800A28AADF83020D4E90149CDE90A01CDE9F6
:10531800084907AC8DF833308DF834E00FCC5035A0
:105328000FC597E8070086E8070060460EB0BDE89D
:10533800F0822E8C5E43B2EB262F4FEA262C04D146
:1053480057B948F6E0260020BFE780B25043A2EBE9
:105358000C06B0FBF6F0B2E742F2B826B2E700005E
:10536800F7B517460E210DF106021D460B4C0646F1
:1053780001F0D4FFBDF8063004EA43433B6050B95E
:105388000DF106020C21304601F0C8FFBDF80630C9
:1053980004EA43442C6003B0F0BD00BF0000FE1FC8
:1053A80073B590F8DA30013B022B06460C4634D828
:1053B80001AB6A460121FFF7D3FF009BB3F57F0FCE
:1053C800054603D8019BB3F57F0F23D915BB34B12C
:1053D8001349304602B0BDE8704001F00FBC04220A
:1053E800FF21304601F04CFF2A4604467021304622
:1053F80001F046FF2A460443FF21304601F040FFF2
:1054080064B204432A468021304601F039FF64B271
:10541800044365B2284602B070BD0025FAE700BF14
:105428005F06002037B5044601228021057C01F083
:1054380027FF0122FF21204601F022FF002211460A
:10544800204601F01DFF94F83A219121204601F0F1
:1054580017FF01220021204601F012FF0022FF2140
:10546800204601F00DFF00228021204601F008FFB0
:10547800012D29D0032D37D0002D3CD101222946FA
:10548800204601F0FDFE01238DF80730A0B103B0DE
:1054980030BD01460DF10702204601F013FF9DF8CB
:1054A8000730DB0705F1010508D538B9B5F5FA6FFE
:1054B800EFD16FF00600EAE70546F0E7B5F5FA6FB9
:1054C80008BF6FF00600E2E718B929462046FFF743
:1054D80067FF02220021204601F0D2FE0028D6D123
:1054E800042384F83231D2E718B901212046FFF7A6
:1054F80057FF0422EEE76FF00700C8E738B5057CD0
:10550800044625B1204600F054FD28B138BDFFF708
:1055180089FF0028F6D0F9E7002DF7D1032384F896
:105528003231F3E773B50646002501220B213046D8
:1055380001F0A6FE002204460B21304601F0A0FE31
:105548000DF1070204431321304601F0BBFE9DF81C
:10555800073064B2044301355B0760B2EDB205D091
:10556800032D08D00028E0D002B070BD032D08BF7D
:105578006FF00B00F8E76FF00B00F5E738B5002384
:10558800037404460D46FFF7B9FF50B92946204673
:10559800FFF751FE28B901462046BDE83840FFF71D
:1055A800C1BF38BD152970B5054616461C4667D1DA
:1055B8000122FF2101F064FE00221146044628461C
:1055C80001F05EFE00220443FF21284601F058FE48
:1055D80064B2044301228021284601F051FE64B2DE
:1055E800044302228521284601F04AFE64B204439E
:1055F8000422FF21284601F043FE64B2044300223E
:10560800CD21284601F03CFE64B204431122CC218E
:10561800284601F035FE64B204430722FF212846DC
:1056280001F02EFE64B204430022BE21284601F098
:1056380027FE64B204430622FF21284601F020FE1B
:1056480064B204430922CC21284601F019FE64B251
:1056580004430022FF21284601F012FE64B20443ED
:105668000122FF21284601F00BFE64B20022044308
:105678001146284601F004FE64B2204340B270BDD2
:10568800042A17D80A2101F0FBFD0028F7D1231EB0
:1056980018BF01231B01EF228421284601F027FEB1
:1056A8000028ECD185F8DA6001462846BDE870404C
:1056B800FFF738BF6FF00A00E1E7000070B594B05B
:1056C80005464022002104A80EF0AEFD002301216A
:1056D8002846ADF806308DF803308DF80430029373
:1056E80000F0B8FC95F8142195F81311012A04D894
:1056F80040F0AD80202940F2AC8001AA02A92846DA
:1057080000F02DFB0446002840F09E8095F85031AB
:10571800002B40F0A280D5F84C11284601F06EFA13
:105728000446002840F0908023462146042228465B
:10573800FFF738FF0446002840F086800122FF2149
:10574800284601F09DFD0DF10602064684212846F3
:1057580001F0E4FD22460643FF21284601F090FDB2
:1057680076B2064374B2002C6ED1BDF806301B0128
:10577800C5F8D43004A92846FFF770FC0446002871
:1057880062D10DF103012846FFF7F2FA044600281A
:105798005AD19DF8033085F8313104AE0FCE05F1AA
:1057A80010040FC40FCE0FC40FCE0FC496E80F001D
:1057B80084E80F000DF103020121284601F082FD63
:1057C8000446002840D19DF8033085F83031024660
:1057D80001462846FFF7DEFA0446A8BB0246022126
:1057E8002846FFF7D7FA044670BB0323014685F81D
:1057F80032310DF10502284601F019F9044618BBAB
:105808009DF8053085F8E8300DF10502012128469C
:1058180001F00DF90446B8B99DF8053085F8E03077
:1058280003AA0321284600F001FF044660B9039B40
:10583800C5F8E43003AA0421284600F0F7FE044620
:1058480010B9039BC5F8DC30204614B070BD0C2994
:1058580051E7284600F010F954E701495DE700BF19
:105868006C05002013B50C460DF10702132101F059
:1058780029FD9DF8073013F0180F03F0070218BF31
:105888006FF00500226002B010BD13B590F8DA3051
:10589800042B0C460BD101A9FFF7E4FF019B042B55
:1058A80001D1012300E00023237002B010BD01AA3A
:1058B800142101F007FD0028F7D19DF80430DB071B
:1058C800EFD42070F1E700F04ABA13B50C460DF199
:1058D8000602282101F022FD78B9BDF80620C2F39E
:1058E8000B0312F4006F18BFA3F580534FF0FA02B0
:1058F80014BF13FB02F35343236002B010BDF0B58D
:105908004FEAD20C4FF0FF341C6002F007026646E3
:1059180000278E4200D207B1F0BD845D664503BF03
:105928001441E4B215463D4614F0010704D005EBD6
:10593800C6051D600136ECE70135082D4FEA540411
:10594800F2D1F7E7034B800953F82000003818BF5D
:10595800012070471808002010B5B1EBD20F4FEAAC
:10596800D20402F0070381BF01229A40035D13436A
:105978008ABF03556FF03100002010BD0A46062388
:10598800B02101F049BC0A460623B02101F062BCEF
:105998002DE9F04F85B08046109E0E9D01968A46EF
:1059A80093461C464FF00009119B994508D10023E6
:1059B800129A1660F3B16FF0310005B0BDE8F08FB0
:1059C80001AB324629465846FFF799FF019F7B1CD9
:1059D8000DD00F9BF818FFF7B5FF504507D13A4691
:1059E8002046FFF7B9FF7E1C09F10109DCE76FF0DB
:1059F8003103DDE721464046FFF7C0FF0028DCD130
:105A080002A94046FFF7BFFF2544234602AAAB423E
:105A1800D3D013F8014B12F8011B8C42F7D0CAE718
:105A280070B5C02288B00E46012190F83041054675
:105A380001F026FCF0B901A92846FFF79FFDC8B977
:105A48000122FF21284601F01BFC98B93246B621F5
:105A5800284601F063FC68B90246FF21284601F098
:105A68000FFC38B922460121284601F009FC08B983
:105A780085F8304108B070BDF0B50F4689B01646BC
:105A8800FF210122044601F0FBFB0246A8B94F2181
:105A9800204601F0F5FB80B92C224E21204601F06A
:105AA800EFFB024648B9FF21204601F0E9FB20B987
:105AB800B422B621204601F0E3FB0025C4F82451A6
:105AC800A4F82851DEB9354607ABB422CDE90373F3
:105AD8000623CDE90032029504F5927304F5957218
:105AE80031462046FFF754FF30B9012384F81531B9
:105AF80084F8137184F8146109B0F0BD013505F11B
:105B0800B400FFF71FFF0028DED12C2DF6D1DBE70C
:105B180010B541F001020021044601F0B1FB78B94B
:105B2800204600F046FA58B901462046FFF7FAFC2D
:105B380030B9024601462046BDE8104001F0A0BB3E
:105B480010BD2DE9F74F4FF0000B88461746FF218F
:105B5800012205461E469DF838A09DF83C908DF818
:105B680007B001F08DFB5A4604465946284601F015
:105B780087FB5A460443FF21284601F081FB64B2A3
:105B8800044364B2B8F1000F32D0BAF1000F06D066
:105B98000C9ACB21284601F095FB204344B2B9F179
:105BA800000F07D00DF10702EE21284601F08AFB0D
:105BB800204344B20122FF21284601F061FB012263
:105BC80004430021284601F05BFB64B20443002231
:105BD800FF21284601F054FB64B29DF807300D9A66
:105BE800204323F0100340B2137003B0BDE8F08FD8
:105BF800BAF1000F06D03A46CB21284601F040FB07
:105C0800204344B2B9F1000FD4D033468022EE21AC
:105C1800284601F06CFBCBE72DE9F04387B09146AD
:105C28000022054688468DF817201E461BB390F8BB
:105C3800307101221146284601F022FB044658BB68
:105C480040212846FFF764FF044628BBB9F1010F3D
:105C580013D10DF11703CDE90290CDE90083024677
:105C6800034649462846FFF76CFF40B104462046E4
:105C780007B0BDE8F0831F46DBE788F80000002E78
:105C8800F5D03A460121284601F0FAFA04460028E0
:105C9800EDD185F83071EAE7002388F80030204616
:105CA800E4E72DE9F043054687B0884691461E464D
:105CB80023B390F8307102220121284601F0E0FA5E
:105CC800044660BB01462846FFF722FF044630BB66
:105CD800B9F1010F14D10DF11703CDE902090093B1
:105CE80002460346CDF8048049462846FFF729FFB7
:105CF80040B10446204607B0BDE8F0831F46DAE706
:105D080088F80000002EF5D03A460121284601F017
:105D1800B7FA04460028EDD185F83071EAE7002388
:105D280088F800302046E4E7F8B51D4616460023FB
:105D38002A4690F830710446FFF76EFF70B90346A3
:105D48002A4631462046FFF7ACFF38B93A460121CA
:105D5800204601F095FA08B984F83071F8BD2DE9AC
:105D6800F04F002393B0CDE90A12C0F82431A0F80F
:105D780028310122FF21CDE90E33B0F83C818DF89E
:105D8800343005468DF8353001F07AFA044600289B
:105D980040F0E38002464F21284601F071FA04469C
:105DA800002840F0DA802C224E21284601F068FABB
:105DB8000446002840F0D1800246FF21284601F021
:105DC8005FFA0446002840F0C880B422B62128466D
:105DD80001F056FA0446002840F0BF8002468021B0
:105DE800284601F04DFA0446002840F0B6800346E4
:105DF8000DF135020DA92846FFF796FF0446002845
:105E080040F0AB800323CDE90203B421062305F556
:105E1800957A05F592790EAECDE9003104960146E2
:105E28004B4652462846FFF7B3FD0446002840F08B
:105E380094800DF1360128460E9FFFF7F1FD0446C8
:105E4800002840F08A80BDF83630434540F2AA80E9
:105E5800C5F82401A5F8280107F1B400FFF772FD81
:105E680008B92B2F7DD90623B4224FF0030BCDE9B7
:105E78000032CDE9027B04964B4652460121284662
:105E8800FFF786FD002840F08B800DF1360128468B
:105E98000E9FFFF7C5FD064600287CD1BDF83630B9
:105EA800434540F2828001260696BDF836304345C8
:105EB80060D2A3EB080383EAE372A2EBE3729DF8D6
:105EC8001860099205F592734FF0030B0793079B2F
:105ED80018689B881090ADF844303A460FAB0621FD
:105EE8005046FFF70CFD0F9F7B1C56D007F1B400FE
:105EF800FFF728FD069B98423CD10BF101033A4677
:105F080048460893FFF728FD002849D14946284606
:105F1800FFF734FD002843D10DF136012846FFF77D
:105F28007FFD00283CD1BDF83620A2EB0803002BEA
:105F3800B8BF5B42424516D9099A934218D910A9AD
:105F48002846FFF71BFD079A07990346109810602B
:105F5800BDF844208A806BB11C46204613B0BDE8CA
:105F6800F08F013778E7DDF820B009930137AEE705
:105F7800DDF820B00A9BC3F800B00B9B1E7001230C
:105F880085F815310A9B1B6885F813310B9B1B7824
:105F980085F81431E1E70446DFE76FF03104DCE708
:105FA8000446DAE70026B3467EE7012383460693D4
:105FB8007BE737B5002304468DF807304FF4FA65C0
:105FC8000DF107012046FFF760FC58B99DF807302E
:105FD800012B07D0013D03D0204601F0E5F9EFE79A
:105FE8006FF0060003B030BD02464FF08043934285
:105FF80002D8002013B970479B08F8E7C1189142EE
:106008004FEA50009CBFC018521A9B08F2E773B5BC
:1060180000228321054601F033F9044688B94FF47C
:10602800FA660DF107028321284601F04BF99DF825
:1060380007300343DBB204461BB9013EF1D16FF0D0
:10604800060401228321284601F01AF9204340B2B0
:1060580002B070BD2DE9F04F90F8F06091B04FF0AC
:106068000009072ECDE9079904460F4600F0A282E1
:106078000122802101F004F901228046FF212046F7
:1060880001F0FEF84A4648EA00084946204601F071
:10609800F7F84FFA88F848EA00080622FF21204658
:1060A80001F0EEF84FFA88F848EA00080DF11502F9
:1060B8008321204601F006F99DF815204FFA88F84B
:1060C80048EA000842F004028321204601F0D8F88B
:1060D8004FFA88F848EA00080722FF21204601F015
:1060E800CFF84FFA88F80122812148EA00082046B3
:1060F80001F0C6F84FFA88F848EA0008204601F08F
:1061080053F94FFA88F848EA00080122802120460E
:1061180001F0B6F84FFA88F848EA000517F0010BC5
:106128006DB200F01E82F20700F11E826B229421EC
:10613800204601F0A5F880462046FFF768FF06AA2A
:1061480048EA00089021204601F008F945EA0805C8
:10615800069B6DB22422942105432046C3F3062AE8
:10616800C3F3C03901F08CF86DB205432046FFF740
:106178004EFF6DB2054306AA9021204601F0EEF8C5
:10618800069B6DB21BBA252294210543204609932C
:1061980001F076F86DB205432046FFF738FF6DB27F
:1061A800054306AA9021204601F0D8F8069B6DB257
:1061B8001A0E05431B0C6DB28DF828208DF8293076
:1061C80017F00203029300F0DB8016F0020840F09B
:1061D800D78002229421204601F052F801902046EF
:1061E800FFF715FF019B0DF116020343902120468E
:1061F8001D4301F067F86DB27B22942105432046C8
:1062080001F03EF86DB205432046FFF700FF6DB27E
:1062180005430DF117029021204601F053F86DB2A5
:10622800772294210543204601F02AF86DB20543F0
:106238002046FFF7ECFE6DB2054306AA90212046E2
:1062480001F08CF8069B5A0E8DF82C20C3F3864279
:106258008DF82D20C3F3C6228DF82E206DB2C3F31E
:106268000612DB0003F07803942105438DF82F20F4
:10627800204678228DF8153001F002F86DB20543FA
:106288002046FFF7C4FE6DB2054306AA90212046BA
:1062980001F064F8069B9DF8152002EB53728DF807
:1062A8003020C3F386528DF83120C3F3C6328DF8FF
:1062B8003220C3F306228DF833206DB2C3F34602B1
:1062C8009B0103F04003942105438DF834202046B8
:1062D80079228DF8153000F0D3FF6DB205432046C2
:1062E800FFF795FE6DB2054306AA9021204601F0FE
:1062F80035F8069B9DF8152002EB93628DF8352042
:10630800C3F3C6428DF83620C3F306328DF8372022
:106318006DB2C3F346129B0003F07C03942105433E
:106328008DF8382020467A228DF8153000F0A8FF25
:106338006DB205432046FFF76AFE6DB2054306AA13
:106348009021204601F00AF8069B9DF815208DF84B
:106358003E8002EB93728DF83920C3F3C6526DB2BA
:106368008DF83A20C3F3064205438DF83B20C3F36A
:106378004622C3F386036DB28DF83C208DF83D307C
:1063880017F00403019300F0F180730700F1EE8029
:106398007B229421204600F073FF80462046FFF7B9
:1063A80036FE07AA48EA00089021204600F0D6FFEA
:1063B80045EA08084FFA88F848EA00057C22942143
:1063C800204600F05DFF6DB205432046FFF71FFE33
:1063D8006DB2054308AA9021204600F0BFFF6DB2B8
:1063E800732294210543204600F04AFF6DB205430D
:1063F8002046FFF70CFE6DB2054306AA9021204601
:1064080000F0ACFF069B6DB21B0274229421054379
:1064180020461FFA83F800F033FF6DB2054320468B
:10642800FFF7F5FD6DB2054306AA9021204600F05E
:1064380095FF6DB29DF81B307522942105432046C7
:1064480043EA080800F01CFF6DB205432046FFF739
:10645800DEFD6DB2054306AA9021204600F07EFFBE
:10646800069B6DB21B029BB27622942105432046FF
:10647800039300F005FF6DB205432046FFF7C7FD03
:106488006DB2054306AA9021204600F067FF6DB261
:106498009DF81B20039B05436DB213430022812105
:1064A8002046039300F0ECFE06220543FF21204618
:1064B80000F0E6FE6DB205430DF11502832120467A
:1064C80000F000FF9DF815206DB2054302F0FB02B5
:1064D8008321204600F0D4FE6DB205430122FF213E
:1064E800204600F0CDFE6DB2054301220021204672
:1064F80000F0C6FE6DB205430022FF21204600F0E1
:10650800BFFE6DB2054300228021204600F0B8FE90
:106518006DB205436DB2039BFDB9BBF1000F29D1E4
:10652800029AAABB019AAAB1720713D4079AC4F8AF
:106538001821089AC4F81C214FEA4822C4F82021DF
:106548003BB1A3F5C8534FF47A7253431B095B421E
:106558001BB2E3603E4384F8F060284611B0BDE802
:10656800F08FD946DA462BE6CA4629E64FF00008EE
:10657800434693E7F007D3D40998BDF8282084F858
:1065880013A184F81491C4F82A01A4F82E21C7E7AE
:10659800B107C7D49DF8162084F8F1209DF817207C
:1065A80084F8F2200BA904F1F30002930DF068FEC1
:1065B800029BB7E74D46D0E750B10138002330F0D1
:1065C800FF019AB203F1010303D100EB022080B26C
:1065D80070474008F3E7C3B2000A03FA00F001303D
:1065E80070470000084B5A434FF47A7302F5FA7269
:1065F8004FF4FA60B2FBF0F0B2FBF3F203FB0100D8
:10660800B0FBF2F0704700BF002F3A00064B5A4328
:106618004FF47A7002F5FA72B2FBF0F24A4302F5CF
:10662800FA72B2FBF0F07047002F3A002DE9FF41F3
:1066380002294FF00005074616468DF80350ADF8BD
:1066480004501CD80DF102022946FEF7A1FB0446AE
:1066580030B90DF103024621384600F033FE0446F6
:106668009DF80300FFF7B7FF81B29DF80220384676
:10667800FFF7CCFF3060204604B0BDE8F081032965
:1066880018D10DF102022946FEF782FB04460028C4
:1066980046D101460DF102023846FEF779FB044661
:1066A80028B901AA5121384600F038FE0446BDF841
:1066B8000400D7E7042935D102A9FEF7BDFB9DF8F0
:1066C8000B30ABB10DF1020229463846FEF760FBEC
:1066D800044658B901AA5121384600F01FFE044665
:1066E800BDF80400FFF777FF85B214B1002015E06C
:1066F8001D460DF1020201213846FEF749FB04460A
:106708000028F3D10DF106027121384600F006FE8B
:106718000446BDF80600FFF75EFF80B2401BA3E702
:106728002846A7E728462C46A4E7F0B5022985B0F5
:10673800054616461ED80DF105020021FEF728FB76
:106748000446A0B99DF8052031462846FFF74AFFC0
:1067580083B2B3F5807F9ABF00F1FF32D2B2FF2235
:10676800A5F8D8204621284600F08AFD0446204690
:1067780005B0F0BD03291FD10DF105020021FEF778
:1067880007FB9DF80520314604462846FFF72AFFF7
:1067980080B2FFF711FF0246ADF80600A5F8D80051
:1067A800002CE4D15121284600F07AFD0446002847
:1067B800DDD1C5F8E460DAE7042939D102A9FEF78A
:1067C8003BFB9DF80B70B7B10DF10502002128467F
:1067D800FEF7DEFA04460028C9D10DF10602512160
:1067E800284600F09BFD0446BDF80600FFF7F3FEBF
:1067F80087B2002CBBD10DF1050201212846FEF716
:10680800C7FA04460028B2D19DF80520314628462B
:10681800FFF7E8FE3844FFF7CFFE7121024628460D
:1068280000F03EFD04460028A1D1C5F8DC609EE7D3
:106838006FF003049BE7F0B585B000238DF80330B3
:10684800D30705460F46164605D439B9A2F10C03FD
:10685800DAB2062A11D96FF00300E6E0012921D146
:10686800A2F10803DAB2062AF5D8062B1AD8DFE80F
:1068780003F03B1969198A199D00062B12D8DFE825
:1068880003F004112D112F11310018225721284629
:1068980000F0F6FC08225621284600F0F1FC0028FA
:1068A80040F0C3807408013CE4B2002F00F09180EE
:1068B800012FD0D101AA04212846FFF7B7FE50B90D
:1068C80022467021284600F0DBFC20B9019A0421F9
:1068D8002846FFF72AFF85F8E06099E03022D5E7DF
:1068E8004022D3E75022D1E71022482100F0C8FC0B
:1068F80008224721284600F0C3FC02220446322120
:10690800284600F0BDFC0C2204433021284600F044
:10691800B7FC64B204430122FF21284600F0B0FC12
:1069280064B2044364B230223021284600F0A8FC47
:1069380000220443FF21284600F0A2FC64B2204351
:1069480040B2ACE72822482100F09AFC08224721EF
:10695800284600F095FC032204463221284600F020
:106968008FFC044364B209223021284600F088FCD9
:1069780001220443FF21284600F082FC64B204434C
:1069880064B22022D0E73822482100F079FC08229E
:106998004721284600F074FC032204463221284689
:1069A80000F06EFC044364B20822DDE74822114679
:1069B80000F066FC08224721284600F061FC03220B
:1069C80004463221284600F05BFC044364B20722E7
:1069D800CAE702AA03212846FFF728FEB0B903AA8E
:1069E80002212846FFF722FE80B922465021284678
:1069F80000F046FC50B9029A03212846FFF795FE9D
:106A080020B9039A02212846FFF78FFE85F8E8602F
:106A180058B969692846FEF7B7F930B90246012323
:106A28000DF103012846FFF73CF905B0F0BD13B599
:106A3800144629B1012910D06FF0030002B010BD2F
:106A48000DF10702502100F03DFC0028F6D19DF819
:106A5800073001335B002370F0E70DF10702702166
:106A6800F1E7F0B5002385B04FF4FA62CDE90023D1
:106A780044F61F63994206460F4604D86FF0030593
:106A8800284605B0F0BD02A9FEF7D6F9054600284C
:106A9800F6D19DF809209DF8083013439DF80A2087
:106AA8001343A7F636341BD06A4602213046FFF757
:106AB800BDFD00283BD19DF808302BB1009B03F2A7
:106AC8004E239C42DAD9E41A9DF80A3023B3009B7E
:106AD80003F2B223B4EB430F4FEA4302CED9A41A10
:106AE8009DF80B305BB101AA03213046FFF79EFDEC
:106AF800019B03F52573A342C0D2C0B9E41A9DF8DF
:106B08000C30002BBCD0A4F2262204213046FFF71B
:106B18000CFE77610546B3E79DF80930002BDFD0FE
:106B2800009B03F525739C42A8D9E41AD8E70546CB
:106B3800A6E770B54FF4FA6286B00023CDE90223C8
:106B480040F636330B600C4604A90646FEF774F986
:106B58000546002836D19DF811209DF810301343C2
:106B68009DF81220134319D002AA02213046FFF7DC
:106B78005DFD002840D19DF810302BB1029B03F237
:106B88004E222368134423609DF81230EBB1029B18
:106B980003F2B222236803EB420323609DF813300B
:106BA800EBB99DF814305BB101AA04213046FFF718
:106BB8003DFD019B03F22622236813442360D8B9C4
:106BC80023687361284606B070BD9DF81130002B0C
:106BD800E4D0029B03F5257223681344DDE703AA7A
:106BE80003213046FFF722FD039B03F52572236836
:106BF800134423600028D4D00546E3E72DE9F74382
:106C0800002406460D46204615F80480B8F1000F0A
:106C180000D010B103B0BDE8F083671CB8F1FF0FD6
:106C280015F8079029D1A71CEB5DB9F1030F36D8E9
:106C3800DFE809F0020B131B271D2C44E27802EB56
:106C48000323A6F834313C46DEE7271D2C44E278BE
:106C580002EB0323A6F83631F5E7271D2C44E2782A
:106C680002EB0323A6F83831EDE7271D2C44E27820
:106C780002EB0323A6F83C31E5E7B8F1040F0ED880
:106C880002344246291901A80DF007FB434601AA20
:106C98004946304604EB080700F0BEFAD3E76FF028
:106CA8000300D0E773B500230E4613600DF107010A
:106CB80005461446FEF7F7F840B99DF807302BB1A2
:106CC800B38A2A6A534380331B0A236002B070BD1B
:106CD80013B5CB681360144601AAFFF7E3FF18B990
:106CE8002368019A1344236002B010BDF8B5B0F8C8
:106CF8005451D0F8580168438030000A0E46454385
:106D0800DDE90717144652B1B60206EB5202B2FB90
:106D1800F4F202EB4202524302F50042140C069AC6
:106D2800534301F50042120C06200332B2FBF0F285
:106D3800C2EBC202B2F5803F38BF033103F500430E
:106D48003EBFB1FBF0F1C1EBC10101F500414FEAD3
:106D5800134334BF090C1B4903FB03F338BF4943F2
:106D680003EB57030B44B3FBF7F39B03FE2205F138
:106D780020007F33B3FBF2F35C434FF47A7704F5DA
:106D8800FA748009B4FBF7F42401FFF72DF904F530
:106D9800FA74BC4228BF4FF4FA63064629BFB4FB15
:106DA800F3F300205B19B4FBF7F428BFB3FBF4F04E
:106DB800FFF71AF9099B864294BF1E6018600020ED
:106DC800F8BD00BF0000F0FF2DE9F04F91B0CDE90C
:106DD8000723036A0E930B6909930546CB680B9347
:106DE8000F460FAAFFF774FF0EAA39462846FFF789
:106DF80059FF58BB0F9C95F8E0B0D5F8DC300593E7
:106E08004FF47A7606FB04F101F5004104910E99DE
:106E18000A910499D5F8E4300693BBF1080F04F100
:106E280080040CBF0223032324F0FF0A090C95F801
:106E3800E820DFF8A081CDF83CA00C9109D1079B90
:106E4800C3F80080089BC5F84081186011B0BDE800
:106E5800F08F06990D932846FFF7C4FB5A4605990B
:106E680081462846FFF7BEFB0D9B5B490C9A81447F
:106E780003FB09F94FEAC92940F2776309F5FA7962
:106E8800240AB9FBF6F903FB09F909F5FA79B9FB04
:106E9800F6F909FB04F404F18003099C74430C40DF
:106EA800B4FBF2F44D4A1B0A944228BF1446012B46
:106EB80038BF01230C204FF4167258435443FFF790
:106EC80093F83B7E3A894FEA400B002B7FD1424929
:106ED800049B0B4003F5FA71414B5A4341F25C2382
:106EE800B2FBF3F20A9B7343B3F5481F28BF4FF474
:106EF8004813A1EB4303B1FBF6F1B3FBF6F31B0216
:106F0800B3FBF1F63602C6F58036564306F5004661
:106F1800360C06F5803676087643B60B4FF4487083
:106F2800704304F5004300F500401B0C5B43000C64
:106F380000FB0030FFF758F803046422323341F2B3
:106F48008837B3FBF2F340F6B532B3FBFBF302FB31
:106F58000377244B9F429CBF42F21073B7FBF3F7B1
:106F6800DDE90532134403F5FA734FF47A7B4FF4E5
:106F7800FA62B3FBFBF0B3FBF2F202F5C812B2FB04
:106F8800F0F088BF4FF47047FFF72EF8000200F5C5
:106F9800FA70B0FBFBF0404307FB0700FFF724F84B
:106FA8000BFB00F0079B0B9A404528BF4046186032
:106FB800089BC5F84001CDE902934FF4487300934C
:106FC8000194334651462846FFF790FE3EE74FF4BA
:106FD8008036A3E7AE878F020000FFFF6666660073
:106FE8009A9906000F279F242DE9F04F8BB00027B0
:106FF80011F0780FDDE914B80446019299468DF82E
:107008000E708DF80F708DF810708DF81170ADF846
:1070180012700997C1F3C30A00F0AF80AAF1050303
:10702800DBB20A2B01D86B4AD75C0DF10E020021A6
:107038002046FDF792FF9DF80E500646D5B1002870
:1070480040F09D8009AB05AA59462046FFF7BCFED3
:10705800002840F09680099BABF80A30014606AA42
:107068002046FDF7B3FF069D25B1059B9D422CBF29
:107078000025012520B904AA02212046FDF76DFF4D
:107088009DF8106026B300287DD107AA022120466A
:10709800FDF79CFF88B90122FF21204600F0F0F897
:1070A80058B90DF11202B621204600F037F920B97F
:1070B8000246FF21204600F0E3F8BDF81230079E93
:1070C8005B02C4F848311EB19E422CBF002601263F
:1070D80028B90DF1110203212046FDF73EFF9DF866
:1070E800113093B1002873D1B9F1000F03D0019B7F
:1070F8001B02B3FBF9F908AA03212046FDF766FF36
:10710800089B4B4594BF0023012320B9012F3CD194
:10711800FF2288F8002098F800200AB9ABF80A2066
:107128000DF10F02012120460193FDF716FF08BB60
:107138009DF80E20019B002A08BF0125BAF1040F13
:1071480018BF9DF80F2084F82E501ABFB2FA82F2A9
:107158005209012284F82F209DF81020002A9DF85A
:10716800112008BF0126002A08BF012384F83060D7
:1071780084F831300BB0BDE8F08F012755E70025C2
:107188007EE735467CE70026A9E70AF1FF32092A9F
:107198000AD8DFE802F0050505090907090B070BFE
:1071A8000522B6E70422B4E7012E01D10322B0E795
:1071B800BAF1040F01D0012B01D10222A9E7012D58
:1071C8001BBF002388F8003088F800502B46A2E740
:1071D8000023A0E70E4F010807B502F10A03009348
:1071E80093B20A4690F86011D0F85C0101F0B2FB46
:1071F80003B05DF804FB13B502F10A0390F860418F
:107208000093D0F85C0193B20A4644F0010101F002
:1072180037FC02B010BD00003F2BF8B50E460546FE
:1072280011461C4611D80A4F38461A4600F8016B19
:107238000DF033F8621C39462846FFF7CDFF0028C9
:107248000CBF00206FF01300F8BD6FF00300FBE7E0
:10725800000F002073B515468DF8071001220DF1B7
:10726800070104461E46FFF7B7FF28B932462946EC
:107278002046FFF7C0FF08B16FF0130002B070BDE1
:1072880008B5064B19705A7019460222FFF7A4FF79
:10729800002814BF6FF01300002008BD000F002065
:1072A80008B5074B1970110A59709A7019460322CC
:1072B800FFF792FF002814BF6FF01300002008BDED
:1072C800000F002037B515468DF8071001220DF183
:1072D80007010446FFF780FF28B901222946204606
:1072E800FFF789FF08B16FF0130003B030BDF7B5A1
:1072F80015460DF1070206460F461C46FFF7E2FF4A
:1073080050B99DF807301D4044EA05023946304619
:107318008DF80720FFF7B4FF03B0F0BD73B514462E
:107328008DF8071001220DF107010646FFF754FFFB
:1073380018B16FF0130002B070BD074D0222294644
:107348003046FFF758FF0028F3D12A786B7803EB13
:1073580002232380EFE700BF000F002073B5144617
:107368008DF8071001220DF107010646FFF734FFDB
:1073780018B16FF0130002B070BD0A4D04222946FF
:107388003046FFF738FF0028F3D16B782A781B04C2
:1073980003EB0263EA781344AA7803EB0223236021
:1073A800E9E700BF000F002008B50220FBF7AEFB9D
:1073B800002008BD7047000010B5032000F072FCE3
:1073C80001F0AAFD064B18600F20FBF795FB044659
:1073D80018B9FBF7F8F9204610BD0124FBE700BFF8
:1073E800280800204FF0E022136923F002031361FC
:1073F80070474FF0E022136943F0020313617047AE
:10740800014BD3F8900570470070FF1F014BD3F86C
:10741800940570470070FF1F014BD3F8980570471B
:107428000070FF1F024A536823F00103536070473E
:10743800002004E0024A536823F0020353607047B7
:10744800002004E0024A536823F0040353607047A5
:10745800002004E08068C0F380007047F7B500237F
:1074680001930446002800F0E980856D25B9FAF7F4
:10747800F5FCE56584F8545023689A68D00040F11B
:10748800A1809A68D10000F1B480A26D42F0100288
:10749800A265E26D42F00102E26501251846FFF798
:1074A800D9FFA26D02F01002024340F0C980A26D1C
:1074B800206922F4817242F00202A2659A68D2071A
:1074C8005DD4226BA67E94F82CC0003A18BF012226
:1074D8001703D4E902120A43217E42EA8132617E0F
:1074E80042EAC13242EA4632002842EA4C02B4BFBC
:1074F80020F000414FF400113A430A4394F8201059
:10750800012903D1002E76D142F48032616A21B17B
:10751800A66A01F4E07131430A43D968E66C21F4A4
:10752800FE3121F4FF711143D96094F83C20616861
:10753800012A01F0404C4CEA060609D1D4E910278B
:107548003A433243A66C324342EA0C0242F0010647
:107558001F693E4A3A4032431A6121F00042B2F1B3
:10756800804F0CD0B1F1004F09D0394ED6F808271A
:1075780001F4701122F470120A43C6F808275A69F8
:10758800666BA16B22F0070232435A615A6922F0F6
:10759800700242EA01125A61002835D19A6A62F0F3
:1075A8000F029A625B6903F007039E423CD10023F5
:1075B800E365A36D23F0030343F00103A3652846A5
:1075C80003B0F0BD9A68234922F0104222F0170256
:1075D80042F080529A60204A1268B2FBF1F20132FE
:1075E80052000192019A002A3FF44BAF019A013AE6
:1075F800F7E7002552E7A16D41F02001A165E16D93
:1076080041F00101E16581E7B0F5001FCAD19A6A2E
:10761800E269013A92006FF00F0102F01C0201FAD0
:1076280002F2216E0A43BCE7A36D23F0120343F074
:107638001003A365E36D43F00103E3650125BEE78D
:10764800A36D43F01003A365F8E700BF02FCFF1F1A
:1076580000200140400D030028080020F8B54569C6
:10766800082D04460E460AD00368DB68D80705D5FE
:10767800A36D43F02003A3650120F8BD0425FBF7A3
:107688003DFA074623681A682A4221D0A26D42F4BF
:107698000072A265DA6812F4406F14D1A27E92B922
:1076A8001A6812070FD51846FFF7D4FE28BB5A6888
:1076B80022F00C025A60A26D22F4807222F00102BC
:1076C80042F00102A265207E00BB0C221A60D4E7BA
:1076D800711CD8D0FBF712FAC01BB04201D8002E9B
:1076E800D0D123681B682B40CCD1A26D84F85430CC
:1076F80042F00402A2650320BFE7A26D42F0200217
:10770800A265E26D42F00102E265DCE70020B4E721
:107718000368186C70470000F7B50023019390F8D0
:107728005430012B044600F0C58005680669012322
:1077380080F854302846FFF78DFE002840F0B480CA
:10774800D1E90020022826F0040300F08280B3F17A
:10775800004FC2F3110E13D1AB6A43EA0E03AB62BA
:107768008B68686903EA022323F07C4323F0FF0354
:1077780020EA02210B43002A6B6126DB002055E03A
:10778800236E00F01F074FF00F0C0CFA07FC6FEA8E
:107798000C0623EA0C0CBEF1000F11D1C2F384636E
:1077A800BB4043EA0C0323668008E3690130984232
:1077B800D6D8A86AC2F38363BB4006403343CEE7FA
:1077C80092FAA2F3B3FA83F3EAE73B493B48D1F8CC
:1077D8000837824203F0E07519D11B02CED4D1F8E4
:1077E800083723F0E0732B4343F40003C1F808374C
:1077F800334B1A68334BB2FBF3F20C2302FB03330F
:107808000193019B002BB9D0019B013BF8E72E485F
:10781800824210D113F08070B0D1D1F8083723F02C
:10782800E0732B4343F08073C1F80837002384F8D2
:10783800543003B0F0BD254882429FD113F4800034
:107848009CD1D1F8083723F0E0732B4343F480032D
:10785800EAE7B3F1004F01BFAB6AC2F311018B43F2
:10786800AB62002A8ADA154813498242D1F80837F0
:1078780009D1D1F8082703F0A07322F0E07213436E
:10788800C1F808377AE71048824204D1D1F80827AE
:1078980003F44003F1E70D4882427FF46FAFD1F85B
:1078A800082703F0C073E8E7A26D42F02002A26542
:1078B8001846BBE70220BCE700200140001000B0DA
:1078C80028080020400D0300004000B8002000B444
:1078D800026838B504461046FFF7BCFD08B9002019
:1078E80038BD9368990707D4936823F0004323F0C1
:1078F800170343F010039360FBF700F9054623686C
:107908009B685B07EBD5FBF7F9F8401B0228F6D913
:1079180023689B685A07F2D5A36D43F01003A3654B
:10792800E36D43F00103E3650120D9E773B5002354
:10793800026801939368DD07044602D5002002B06F
:1079480070BD9168214B194209D0A36D43F0100313
:10795800A365E36D43F00103E3650120EFE7936856
:1079680023F0004323F0170343F001039360184BFF
:10797800D3F8083718021CD4637E012BDED0FBF73E
:10798800BDF8144E054622681368DB07D6D4936801
:10799800D9075FBF9368334043F001039360FBF757
:1079A800ADF8401B0228EED923681B68DA07EAD431
:1079B800CBE7094B094A1B68B3FBF2F30133019388
:1079C800019B002BD8D0019B013BF8E717000080F2
:1079D80000200140E8FFFF7F28080020400D030039
:1079E80038B504460068FFF735FD054620BB94F816
:1079F8005430012B20D0012384F854302046FFF75F
:107A080095FFB0B9A36D226823F4706323F00103D6
:107A180043F48073A3651C23E065136084F8540065
:107A2800936823F0004323F0170343F004039360A3
:107A380038BD84F85450FBE70220F9E7026838B5EE
:107A4800936891680446C80701D4002038BD990797
:107A5800FBD4936803F00503012B19D1936823F035
:107A6800004323F0170343F00203936003231360DA
:107A7800FBF744F8054623689B68DB07E5D5FBF769
:107A88003DF8401B0228F6D923689B68DA07F2D52F
:107A9800A36D43F01003A365E36D43F00103E365B1
:107AA8000120D3E770B5044600284BD0836D43F01E
:107AB80002038365FFF70CFF054668B92046FFF708
:107AC800BDFF054608B90123A3652268936823F022
:107AD800104323F01703936023685A6822F46772EF
:107AE80022F003025A6040F29F321A60D968164A9F
:107AF8000A40DA601A6922F040421A615A6922F093
:107B080007025A611A6A02F0F0221A625A6A02F0EF
:107B1800F0225A62DA6A02F0F022DA629A6A0B4AB2
:107B280000269E62D2F8083723F0FE73C2F80837A1
:107B38002046FAF7A7F9E6652666A66584F8546034
:107B4800284670BD0125FBE700023E830020014066
:107B580010B590F85430012B044615D0012380F855
:107B68005430FFF7B5FE58B92046FFF767FF38B91C
:107B7800A36D23F4807323F0010343F00103A3658D
:107B8800002384F8543010BD0220FCE7F7B5002329
:107B9800019390F85430012B04467FD0012380F8DC
:107BA8005430FFF74BFF23689A6812F0010205462C
:107BB80007D0A36D43F01003A365002384F8543065
:107BC8002DE0A16D364F21F4817141F00201A165CC
:107BD800DE68D96826F4FF4626F07C0621F40041C9
:107BE800360421F00301360CD96008209968394021
:107BF80041F0004199609968002913DA019901312F
:107C080001910199B1F52E3FF5D3A36D23F012032D
:107C180043F01003A365002384F854300125284657
:107C280003B0F0BDD3F8B410013801F07F010A4465
:107C3800DCD199681A48014041F001019960D3F8F4
:107C4800B41021F07F0141EAD202C3F8B4209A6847
:107C5800024042F002029A60FAF750FF0746236892
:107C68009A68D20708D4DA683243DA60A36D23F041
:107C7800030343F001039FE7FAF740FFC01B022804
:107C8800EDD923689B68D907E9D5A36D43F01003A4
:107C9800A365E36D43F00103E365BFE70225BEE793
:107CA800E8FFFF7F0749CA6822F4E0620302120472
:107CB80003F4E063120C134343F0BF6343F400334F
:107CC800CB60704700ED00E0164B30B5DC68C4F3BC
:107CD8000224C4F10703251D042B28BF0423062D05
:107CE8004FF0FF358CBF033C002405FA03F321EA6B
:107CF8000303A54022EA0502A340002843EA020341
:107D0800ACBF00F16040084A4FEA0313B8BF00F067
:107D18000F00DBB2AABF00F56140135480F80033AE
:107D280030BD00BF00ED00E014ED00E0002807DBE7
:107D3800044A4109012300F01F00834042F8213022
:107D4800704700BF00E100E000280CDB430906494A
:107D580000F01F0020330122824041F82320BFF3A6
:107D68004F8FBFF36F8F704700E100E070B5D0E927
:107D780013456560446D14B1D0E916456560D0E9D6
:107D8800105404F01C060124B4406C60046863605D
:107D98008368102B0BBFA260A160E160E26070BD38
:107DA8000268416CD3B210B5083B1424B3FBF4F35A
:107DB8000B4CA24288BF0B4A21F0030199BF01F185
:107DC800804202F50232521807338264064AC264BE
:107DD80003F01F03012202FA03F3036510BD00BF7D
:107DE800070402401C0802408008024038B50028F9
:107DF8005ED002682F4B9A424FF014014CD82E4B9C
:107E08001344B3FBF1F32D499B00C0E9101302237F
:107E180080F825301368056923F4FF4323F07003C5
:107E28001360D0E9024323432B43456911682B4370
:107E380085692B43C5692B43056A2B430B431360A4
:107E4800FFF7AEFFB4F5804F04BF002343604268DC
:107E5800816C02F07F030B60D0E91314013A032A06
:107E68004C6020D8164A174981651A44013B920094
:107E7800012103F0030301FA03F300214265C365FE
:107E88001160114A536400230122C36380F824302F
:107E980080F82520184638BD0C4B1344B3FBF1F38A
:107EA8000B499B00B1E70023C0E91533C365EAE736
:107EB8000120F0E707040240F8FFFDBF0000024080
:107EC8003F8200104009024000090240F8FBFDBF54
:107ED8000004024038B5002841D00268136823F036
:107EE800010313601F4B9A424FF0140130D81E4B08
:107EF8001344B3FBF1F31D499B00C0E9101301249F
:107F080003F01C0304FA03F3002515604B60FFF728
:107F180047FF836C41681D60D0E913325A604A1EDE
:107F2800032A06D8124B0B449B0094401D60114B4A
:107F38005C640023C363C0E91533C0E90B33C0E9AF
:107F48000D33C36580F8253080F82430184638BDD5
:107F5800094B1344B3FBF1F308499B00CDE701201B
:107F6800F5E700BF07040240F8FFFDBF000002402C
:107F78003F82001000090240F8FBFDBF00040240E8
:107F880070B590F82450012D04463BD090F8256038
:107F98000125AE4280F824504FF000062CD102256E
:107FA80080F825500568C6632E6826F001062E6005
:107FB800FFF7DCFE036BBBB12B6843F00E032B60AD
:107FC800A36C1A68D20342BF1A6842F480721A601E
:107FD800636D1BB11A6842F480721A602B6843F013
:107FE80001032B60002070BD2B6823F004032B6075
:107FF8002B6843F00A03E2E78023C36380F8246018
:108008002846F0E70220EEE7034640B190F8252025
:10801800022A06D00422C263002280F8242001200C
:1080280070470268806C116821F00E0111600168C8
:1080380021F480710160116821F001011160D3E918
:10804800100202F01C0101228A404260D3E9132188
:1080580051605A6D32B1116821F480711160D3E911
:10806800162151600122002083F8252083F824007E
:10807800704710B590F82530022B03D00423C36352
:10808800012010BD03681A6822F00E021A601A68EF
:1080980022F001021A60826C136823F48073136063
:1080A800D0E9101303F01C02012393404B60D0E980
:1080B80013325A60436D33B11A6822F480721A6021
:1080C800D0E916325A60012380F82530836B0024EA
:1080D80080F8244013B198472046D2E71846D0E7E5
:1080E80070B4426C046C036826681D6802F01C02B8
:1080F8000421914031420FD015F0040F0CD01A68BA
:1081080092065EBF1A6822F004021A60036B61606F
:10811800002B33D070BC184702219140314217D050
:1081280015F0020F14D01A68940606D41A6822F0C3
:108138000A021A60012280F82520114A93428CBF56
:10814800104B114B5960002380F82430C36ADFE7D5
:1081580008219140314211D029070FD5196821F023
:108168000E011960012303FA02F26260C36380F80A
:108178002530002380F82430436BC9E770BC704772
:108188008000024000040240000002400A4A53698D
:1081980043F4802330B55361EFF3108472B60023A3
:1081A800CD58C5500433B3F5807FF9D11369DB038B
:1081B800FCD484F3108830BD00400058064B5A693F
:1081C800002ABFBF054A9A6002F188329A60BABF96
:1081D8005869C00F002070470040005823016745C8
:1081E800044B5A6942F000425A615869C043C00FB3
:1081F800704700BF0040005870B50546FAF77EFC8E
:10820800124E04463369D90313D43369DA0744BFDD
:10821800012232614CF2FA32134011D10B4E30690F
:1082280010F480200BD0FAF769FC001BA842F6D3A3
:1082380004E0FAF763FC001BA842E3D3032070BDF7
:10824800024A1361024A01205360F8E700400058CF
:10825800400F00202DE9F041184D98462B78012B4E
:1082680006460C46174626D001232B704FF47A7029
:1082780000236B60FFF7C0FFA0B9012E16D1104A8A
:10828800536943F0010353612760BFF36F8FC4F84C
:1082980004804FF47A70FFF7AFFF094A536923EA65
:1082A8000603536100232B70BDE8F0813946204650
:1082B800FFF76CFFEDE70220F6E700BF400F002054
:1082C80000400058054A536923F47E7343EAC0000E
:1082D80040F4803040F00200506170470040005880
:1082E8002DE9F041234F3B78012B054688463FD0C6
:1082F80001233B704FF47A7000237B60FFF77CFF0B
:10830800044688B92B68042B13D11B4A536943F4DC
:10831800803343F0040353614FF47A70FFF76CFF26
:108328000446154B1A681B6800233B702046BDE8BD
:10833800F0814FF0FF33C8F800306E68D5E901329C
:108348001344B3420AD93046FFF7BCFF4FF47A70A2
:10835800FFF752FF50B1C8F800600446064A536957
:1083680023F47E7323F002035361DAE70136E5E76D
:108378000224DBE7400F0020004000582DE9F04FB1
:10838800524C00234FF00F090A6832FA03F501D165
:10839800BDE8F08F012505FA03F818EA020200F09B
:1083A8008E804E68032706F003054FEA430E07FA4E
:1083B8000EFC6F1E012F6FEA0C0C32D8876807EA93
:1083C8000C0ACF6807FA0EF747EA0A07876047687A
:1083D80027EA0808C6F300179F4047EA08074760DE
:1083E800C76807EA0C088F6807FA0EF747EA080714
:1083F800022DC76017D14FEAD30800EB880803F0B5
:10840800070AD8F820704FEA8A0A09FA0AFB27EA0D
:108418000B0B0F6907FA0AF747EA0B07C8F8207031
:1084280001E0032DDCD1076805FA0EF507EA0C0711
:108438003D4316F4403F056041D023F0030707F1A0
:10844800804707F5803703F0030CBD684FEA8C0CB2
:108458004FF0070E0EFA0CFEB0F1904F25EA0E0E03
:108468002FD01B4DA8422ED005F58065A8420CBF21
:108478000225072505FA0CF545EA0E05BD602568B5
:10848800D74316F4801F0CBF3D401543256065682F
:1084980016F4001F0CBF3D4015436560D4F88050AA
:1084A80016F4803F0CBF3D401543C4F88050D4F803
:1084B8008450B60354BF3D401543C4F8845001337B
:1084C80062E70025D6E70125D4E700BF0008005879
:1084D80000040048374A2DE9F04F00234FF0010A05
:1084E8004FF0070B4FF00F0931FA03F401D1BDE843
:1084F800F08F0AFA03FC1CEA010654D023F00304A7
:1085080004F1804404F5803403F00307A568BF0034
:108518000BFA07F8B0F1904F08EA050E45D0264D42
:10852800A84244D005F58065A8420CBF022507255E
:10853800BD40754517D1D2F8805025EA0605C2F826
:108548008050D2F8845025EA0605C2F88450156890
:1085580025EA06051560556825EA06055560A568EB
:1085680025EA0805A560056803265C0006FA04F4F8
:1085780023FA06F6254300EB8606056003F0070597
:10858800376AAD0009FA05F527EA050737628568F5
:1085980025EA04058560456825EA0C054560C56837
:1085A80025EA0404C46001339EE70025C0E70125DD
:1085B800BEE700BF000800580004004803691942DC
:1085C80014BF0120002070470AB1816170478162A1
:1085D80070470000044AD168014208B502D0D06053
:1085E800FBF726F908BD00BF0008005803689A6920
:1085F800910744BF00229A629A69D2075EBF9A69BE
:1086080042F001029A61704730B5039D04682B431C
:1086180043EA0243064A6068C1F309010B4342EA90
:10862800555223F0004320EA02000343636030BD43
:10863800FF63FF0303682DE9F0419C6914F01004FF
:1086480005460F4616466FD010220024DA61A04670
:108658002B689A69900661D4B8F1000F35D044F0C0
:10866800040401202E68B369D90541BF4FF4807214
:10867800F26144F0010401205A0541BF4FF48062C1
:1086880044F00804F26101209B054FD54FF40073B4
:1086980044F00204F3612846FFF7A8FF736823F04B
:1086A800FF7323F48B3323F4FF7323F00103736008
:1086B8006B6C23436B64202385F84130002385F8D5
:1086C800423085F84030012032E07A1CC1D0FAF7F8
:1086D80015FA801BB84201D8002FB9D12B68596808
:1086E80095F8422098690004D2B20AD5490408D402
:1086F800202A06D05A6842F480425A60FAF7FEF9F6
:1087080006462B689B699B06A2D4FAF7F7F9801BEB
:108718001928F6D920244FF0010899E7B8F1000F7D
:108728009DD12022DA619AE720469BE70028B2D142
:10873800BDE8F08170B504460D46164623689B696E
:108748009B0701D5002070BD324629462046FFF719
:1087580071FFA0B96A1CF1D0FAF7D0F9801BA842C2
:1087680001D8002DEAD1636C43F020036364202311
:1087780084F84130002384F8423084F840300120E6
:10878800E1E770B504460D46164623689B695B070A
:108798000ED4324629462046FFF74CFF38BB2368E3
:1087A8009A69910625D59A69520703D5228D0AB18F
:1087B800002070BD9A6912F010021CBF1022DA6105
:1087C8004FF0200118BF04226264D9615A6822F070
:1087D800FF7222F48B3222F4FF7222F001025A60F7
:1087E800002384F8411084F8423084F84030012096
:1087F800DFE7FAF783F9801BA84201D8002DC4D11E
:10880800636C43F020036364202384F84130002321
:10881800EBE72DE9F041069F0446884616461D46BB
:108828002268936938EA03030CBF01230023B3428B
:1088380001D0002015E06B1CF3D0FAF75FF9C01BDC
:10884800A84201D8002DEBD1636C43F02003636488
:10885800202384F84130002384F8423084F84030E3
:108868000120BDE8F08170B504460D461646236820
:108878009B699B0601D5002070BD324629462046DB
:10888800FFF7D8FE90B9FAF739F9801BA84201D84A
:10889800002DECD1636C43F020036364202384F83B
:1088A8004130002384F8423084F840300120E3E767
:1088B80010B5044600284AD090F8413003F0FF0272
:1088C8001BB980F84020F9F707FE242384F84130CB
:1088D80023681A6822F001021A60626822F0706246
:1088E8001A619A6822F400429A60D4E902210129A7
:1088F80024D142F400429A605A6842F0007242F46D
:1089080000425A60DA6822F40042DA60D4E90421AD
:108918000A43A16942EA0122DA60D4E907210A433D
:108928001A601A6842F001021A600020202360646D
:1089380084F84130206384F8420010BD42F40442B8
:1089480002299A6004BF4FF400625A60D4E70120FC
:10895800F3E700002DE9F347984690F841300A9F65
:10896800202B04460E46914640F0868090F8403011
:10897800012B00F081804FF0010A80F840A0FAF73F
:10898800BDF819230546009052464FF40041204691
:10899800FFF73FFF18B1012002B0BDE8F08721239F
:1089A80084F84130102384F842306064A4F82A80A7
:1089B800638DC4F824909BB2FF2B60632F4B26D99C
:1089C800FF22228500934FF0807331462046FFF73F
:1089D8001BFE638D9BB22A4639462046FBB9FFF73A
:1089E80042FF0028D7D123682021D9615A6822F094
:1089F800FF7222F48B3222F4FF7222F001025A60D5
:108A080084F8411084F8400084F84200C4E7628D7D
:108A1800009392B222854FF00073D2B2D5E7FFF7E8
:108A280089FE0028B7D1636A226813F8011B916296
:108A38006362638D228D013B9BB26385638D013A2E
:108A480092B29BB22285002BC3D0002AC1D10095D7
:108A58003B4680212046FFF7DCFE00289BD1638D32
:108A68009BB2FF2B03D9FF2222850090ABE7628DD2
:108A7800009092B22285CEE702208DE70020008088
:108A88002DE9F347984690F841300A9F202B044679
:108A98000E46914640F0878090F84030012B00F058
:108AA80082804FF0010A80F840A0FAF727F81923CE
:108AB8000546009052464FF400412046FFF7A9FEB4
:108AC80018B1012002B0BDE8F087222384F84130B4
:108AD800102384F842306064A4F82A80638DC4F8B7
:108AE80024909BB2FF2B6063304B26D9FF2222854E
:108AF80000934FF0807331462046FFF785FD638D64
:108B08009BB22A4639462046FBB9FFF7ACFE00283F
:108B1800D7D123682021D9615A6822F0FF7222F444
:108B28008B3222F4FF7222F001025A6084F841105D
:108B380084F8400084F84200C4E7628D009392B242
:108B480022854FF00073D2B2D5E7FFF71AFE00284E
:108B5800B7D123685A6A636A1A70636A228D01332F
:108B68006362638D013B9BB26385638D013A92B268
:108B78009BB22285002BC2D0002AC0D100953B466B
:108B880080212046FFF745FE00289AD1638D9BB2CD
:108B9800FF2B03D9FF2222850090AAE7628D00905F
:108BA80092B22285CDE702208CE700BF0024008026
:108BB80010B590F84120202A0346D4B21CD190F871
:108BC8004020012A18D0242280F841200268106829
:108BD80020F001001060106820F4805010601068C8
:108BE800014311601168002041F00101116083F810
:108BF800414083F8400010BD0220FCE710B590F812
:108C08004120202A0346D4B21BD190F84020012AE3
:108C180017D0242280F841200268106820F0010053
:108C28001060106820F4706040EA0121116011683A
:108C3800002041F00101116083F8414083F84000B1
:108C480010BD0220FCE70000024A136843F4807359
:108C580013607047000400580D4B10B55B690C4653
:108C680028B99A0507D500F027F820B110BD9B0553
:108C780001D400F019F8074A1369012C23F0040302
:108C8800136101D130BFF1E740BF20BF20BFEDE73E
:108C98000004005800ED00E0024B186800F4C060C2
:108CA800704700BF00040058024A136843F4804329
:108CB80013607047000400580C4A136823F480437B
:108CC80013600B4B1B6832214B430A49B3FBF1F38A
:108CD8005169890500D533B9536913F4007F14BF6E
:108CE800032000207047013BF2E700BF0004005852
:108CF8002808002040420F000B4A136823F007039E
:108D080043F002031360094B1A69012842F0040278
:108D18001A6105D130BF1A6922F004021A6170473E
:108D280040BF20BF20BFF6E70004005800ED00E078
:108D38004FF0B0431868C0F3404070474FF0B0435D
:108D48001868C0F3400070474FF0B042536823F4EE
:108D58007F4343EA0023536070474FF0B0431868DD
:108D6800C0F34060704700007FB54FF0B0432C4A15
:108D7800D3F80831C0F3031003F00F0352F8204072
:108D8800284A52F82330B4FBF3F4FFF785FF264B4B
:108D9800054693E80700B5F5007F04AB03E9070033
:108DA80010D0224B9C4218D303F5B70303F67F5328
:108DB8009C4229D903F5741303F510639C4225D806
:108DC80002230BE01A4B9C4207D91A4B9C421BD931
:108DD80003F5370303F5D853F0E7002304AA02EBA1
:108DE800830353F80C4C144D2B6823F007032343DB
:108DF8002B60F9F783FE06462B6803F007039C42B5
:108E080006D1002004B070BD0123E7E70024EAE79B
:108E1800F9F774FE801B0228EED90320F2E700BFA1
:108E28007C4F01081C4F0108E0430108C0CF6A00CD
:108E3800BFEA21013F933402004000584FF0B0438D
:108E480010B59A68D96812F00C0205D00C2A4AD1DC
:108E580001F00303012B50D14FF0B0412B480B68B0
:108E680013F0080306D00B6813F0080337D1D1F8C4
:108E7800941007E00C68240756BFD1F894300968AD
:108E8800C3F3032350F82330002A0CBF18460020F0
:108E98004FF0B0418A6802F00C020C2A1ED1CA6851
:108EA80002F00302022A2ED0032A06D10B68184AC0
:108EB80013F4801F174B18BF13464FF0B042D06809
:108EC800D168D268C0F306205843C1F302130133B6
:108ED800B0FBF3F0530F0133B0FBF3F010BD0B6898
:108EE800C3F30313CEE7042A0AD0082A05D11B6866
:108EF80013F4801304D10748CAE700231846C7E7CC
:108F080003480023C4E7024BD7E700BF7C4F0108A2
:108F18000024F4000048E80108B5FFF78FFF4FF080
:108F2800B043044A9B68C3F3031352F82330B0FBE1
:108F3800F3F008BD1C4F01082DE9F0410446002854
:108F480053D04FF0B0439D68DE6803689B0605F078
:108F58000C0506F0030668D5026A1DB10C2D46D132
:108F6800012E44D1002A40D04FF0B043A16A1A68BC
:108F7800170756BFD3F894301B681B0903F0F0039A
:108F880099421FD90846FFF7EFFE00282DD14FF070
:108F9800B042136843F0080313601368A16A23F012
:108FA800F0030B431360606AFFF7CEFEFFF7B4FFD0
:108FB800AB4B1860AB4B1868F9F79EFD002834D00E
:108FC800BDE8F0814FF0B042136843F00803136026
:108FD800136823F0F0030B431360606AFFF7B4FED5
:108FE8000846FFF7C1FE0028E0D00120E8E74FF06F
:108FF800B043002A54D01A6842F001021A60F9F707
:109008007DFD0746FFF79AFE002842D04FF0B04298
:10901800136843F0080313601368A16A23F0F00390
:109028000B431360606AFFF78FFE2368D80748D4A4
:109038002368990700F18C8023681E0740F1FA80A5
:10904800A3694FF0B046002B00F0E180D6F89430C9
:10905800E16903F01002914200F0C48003F00302BA
:10906800022AC2D0D80740F1B380D6F8943023F052
:109078000103C6F89430F9F741FD0746D6F8943055
:10908800990740F1A580F9F739FDC31B112BF5D9D4
:1090980004E0F9F733FDC01B0228B3D903208FE79A
:1090A8001A6822F001021A60F9F728FD0746FFF74F
:1090B80045FE0028B9D0F9F721FDC01B0228F6D9D2
:1090C800ECE7082D03D00C2D05D1032E03D16368DE
:1090D800002BADD189E74FF0B043A1681A6822F49C
:1090E80080120A431A606268B2F5803F10D11A688C
:1090F80042F480321A60F9F701FD0746FFF718FEBF
:10910800002895D1F9F7FAFCC01B6428F6D9C5E701
:10911800B2F5041F04D11A6842F400121A60E6E797
:10912800196821F480311960196821F40011196057
:10913800002AE0D1F9F7E2FC0746FFF7F9FD00281D
:109148003FF476AFF9F7DAFCC01B6428F5D9A5E738
:10915800042D236903D00C2D0ED1022E0CD1002B27
:109168003FF443AF4FF0B0426169536823F0FE43C8
:1091780043EA016353605FE74FF0B046BBB1336821
:1091880043F480733360F9F7B9FC074633685A052E
:1091980007D57368626923F0FE4343EA026373608C
:1091A8004AE7F9F7ABFCC31B022BEFD976E7336824
:1091B80023F480733360F9F7A1FC074633685B0535
:1091C8007FF53AAFF9F79AFCC31B022BF6D965E78E
:1091D8004FF0B042E169D2F8943023F010030B430A
:1091E800C2F894304FF0B047D7F8943043F00103F9
:1091F800C7F89430F9F782FC0646D7F894309A07F6
:1092080018D4F9F77BFC831B112BF6D946E7D6F85F
:10921800943023F00103C6F89430F9F76FFC074641
:10922800D6F894309B0705D5F9F768FCC31B112BBA
:10923800F6D933E72368580754D50B4F3B68D9054F
:1092480014D4FFF701FDF9F759FC06463B68DA0527
:109258000CD4F9F753FC831B022BF7D91EE700BF88
:10926800280800202C08002000040058E3684FF06C
:10927800B046002B58D023F08003052B02BFD6F848
:10928800903043F00403C6F890304FF0B046F9F739
:1092980035FCD6F8903043F001030746C6F8903005
:1092A80041F28838D6F890309B0705D4F9F726FCA8
:1092B800C31B4345F6D9F1E6E36823F00403812B89
:1092C8001BD1F9F71BFCD6F8903043F08003C6F8A1
:1092D800903007464FF0B04641F28838D6F89030C3
:1092E800180504D5E06A00284AD1002068E6F9F795
:1092F80005FCC01B4045F1D9D0E6F9F7FFFBD6F8CD
:10930800903023F08003C6F8903007464FF0B046FF
:1093180041F28838D6F890301905E3D5F9F7EEFB15
:10932800C01B4045F6D9B9E6F9F7E8FBD6F8903006
:1093380023F080030746C6F8903041F28838D6F803
:1093480090301A0516D4F9F7D9FBD6F8903023F0E7
:109358000103C6F8903007464FF0B04841F288360E
:10936800D8F890309B07BDD5F9F7C8FBC31BB342AB
:10937800F6D993E6F9F7C2FBC01B4045DFD98DE665
:109388000C2D4ED04FF0B04302281A6822F080729C
:109398001A6033D1F9F7B2FB0546FFF7DEFC38BB9C
:1093A800D4E90C314FF0B0420B43D0682D4901404D
:1093B8000B43E16B0B43216C0B43616C0B43A16BBB
:1093C80043EA0123D360136843F080731360D368C2
:1093D80043F08053D360F9F791FB0446FFF7BDFCD7
:1093E800002882D1F9F78AFB001B0A28F6D955E62E
:1093F800F9F784FB401B0A28CFD94FE6F9F77EFB23
:109408000446FFF7AAFC30B94FF0B042164BD168BA
:109418000B40D360D4E5F9F771FB001B0A28F0D99B
:109428003CE601283FF4CCAD4FF0B043226BDB683B
:1094380003F0030191427FF4D8AD616B03F0700231
:109448008A427FF4D2ADA16B03F4FE42B2EB012F46
:109458007FF4CBAD626C03F0604393423FF445AFB9
:10946800C3E500BF8C80C111FCFFFEEE2DE9F04181
:109478000D46044610B90120BDE8F081684E3368F6
:1094880003F007038B4216D323689A0727D54FF0BA
:10949800B047A268BB6823F0F0031343BB60F9F739
:1094A8002DFB0646BB68DB0319D4F9F727FB831BA2
:1094B800022BF7D911E0336823F007030B4333601D
:1094C800F9F71CFB0746336803F00703AB42DBD010
:1094D800F9F714FBC01B0228F5D90320CCE7236851
:1094E800580617D54FF0B0476269D7F8083123F00E
:1094F8000F0343EA1213C7F80831F9F7FFFA0646D3
:10950800D7F80831D90305D4F9F7F8FA831B022BE9
:10951800F6D9E2E723685A0713D54FF0B047E26857
:10952800BB6823F4E0631343BB60F9F7E7FA064628
:10953800BB689B0305D4F9F7E1FA831B022BF7D923
:10954800CBE72368180714D54FF0B0472269BB68EA
:1095580023F4605343EAC203BB60F9F7CFFA064627
:10956800BB68590305D4F9F7C9FA831B022BF7D94D
:10957800B3E72368DA070FD4294C236803F00703FD
:10958800AB4239D8FFF7C8FC264B1860264BBDE81C
:10959800F0411868F9F7B0BA6268022A1DD1FFF7DE
:1095A800C7FB00283FF467AF4FF0B04641F2883858
:1095B800B36823F003031343B360F9F79FFA074630
:1095C800B368626803F00C03B3EB820FD4D0F9F7E9
:1095D80095FAC01B4045F3D97FE7032A02D1FFF76C
:1095E800BCFBDEE712B9FFF7A9FBDAE74FF0B0439F
:1095F8001B685B05D8D43EE7236823F007032B4399
:109608002360F9F77BFA0646236803F00703AB42A9
:10961800B8D0F9F773FA801B0228F5D95DE700BFC7
:1096280000400058280800202C08002008B5FFF743
:1096380073FC4FF0B043044A9B68C3F3022352F80B
:109648002330D84008BD00BF5C4F010808B5FFF7BC
:1096580063FC4FF0B043044A9B68C3F3C22352F83B
:109668002330D84008BD00BF5C4F01084FF0B0431D
:10967800D3F89000C0F3400070474FF0B0410209A2
:10968800D1F8883002F47F22000123EA020300F4B3
:109698007F200343C1F8883070474FF0B041020C77
:1096A800D1F88830120423EA020343EA0040C1F8E3
:1096B8008800704770B5066816F48036044638D0BE
:1096C800FFF7C2FAF9F71AFA614E05463368DB0567
:1096D80029D54FF0B043616BD3F8902002F4407263
:1096E800914214D0D3F89010D3F8902042F48032ED
:1096F800C3F89020D3F8902021F4407022F48032EF
:109708008D07C3F89020C3F8900000F190804FF0C7
:10971800B042616BD2F8903023F440730B43C2F827
:109728009030002605E0F9F7E9F9401B0228CDD969
:1097380003262568E8070AD54FF0B0416268D1F8DA
:10974800883023EA124392B21343C1F88830A9073C
:109758000AD54FF0B041A268D1F8883023EA124305
:1097680092B21343C1F88830AA0609D54FF0B04227
:109778002169D2F8883023F440630B43C2F888305B
:10978800AB0502D5206AFFF788FF680502D5606A35
:10979800FFF783FF290502D5A06AFFF77EFF6A0657
:1097A80002D56069FFF769FF2B0602D5A069FFF7AC
:1097B80064FFE80502D5E069FFF75FFFE90610D509
:1097C8004FF0B042E168D2F8883023F440730B437D
:1097D800C2F88830B1F5807F02BFD36843F0807348
:1097E800D3602A040ED54FF0B042216BD2F88830EE
:1097F80023F040430B43C2F8883019B9D36843F0CB
:109808008073D3606B0410D54FF0B042E16AD2F890
:10981800883023F040530B43B1F1005FC2F8883021
:1098280003D1D36843F48033D360304670BDF9F771
:1098380065F941F288360546FFF718FF01283FF41D
:1098480066AFF9F75BF9401BB042F5D970E700BF86
:109858000004005830B590F82C30012B02464FF028
:10986800020022D0174B82F82D00CA24012582F865
:109878002C505C6253245C62B1F5807F146B99694B
:1098880014D121F488519961596C24F0010421F014
:10989800004159641463DD650A4BFF2159620020B9
:1098A800012382F82D3082F82C0030BD21F40851B4
:1098B8009961D96C24F0020421F00041D964146341
:1098C800D865E9E70028004070B50B4E036B756D4D
:1098D8001D40EA07044603D50123F365F9F77FFA2B
:1098E800AB0704D50223F365204600F0CBF901232A
:1098F80084F82D3070BD00BF0028004038B50A4CF0
:10990800E36823F02003E360F9F7F8F80546E36815
:109918009B0601D5002038BDF9F7F0F8401BB0F5DB
:109928007A7FF4D90320F6E7002800402DE9F041BA
:10993800114DEC6814F0400407461AD1EB6843F067
:109948008003EB60F9F7DAF84FF003080646EB6896
:109958005B0601D4032C02D12046BDE8F081F9F75B
:10996800CDF8801BB0F57A7F84BF87F82D8003245B
:10997800EDE70024F0E700BF0028004038B50F4CA1
:10998800E36823F08003E360A3699B06054606D4D9
:10999800FFF7B4FF10B1032085F82D0038BDA36987
:1099A80023F02003A361FFF7A9FF10B1032085F876
:1099B8002D00A36943F02003A361EFE700280040CE
:1099C80038B5044600284BD090F82D3003F0FF023C
:1099D8001BB980F82C20F8F78FFE0223214D84F85C
:1099E8002D30EB68DB0632D4CA236B6253236B62DB
:1099F8002046FFF79BFF78BBAB6923F08E6323F00B
:109A08004003AB6121696368AA690B431343A269E8
:109A18001343AB61D4E9022343EA02432B61D4E93F
:109A28000931EA680B4322F4F8521343EB602046ED
:109A3800FFF7A4FF80B9D4E90713AA690B4322F002
:109A48006042134362691343AB61FF236B620123D6
:109A580084F82D30002002E0024BFF225A6238BD04
:109A68000120FCE7002800400023092803D840EA29
:109A78000310C0B270470A380133C0B2F5E70000DE
:109A88002DE9F04790F82C30012B05464FF00200E5
:109A980069D0012385F82C304E4B85F82D00DE68FF
:109AA80006F44076B6F5807F78D04C69087891F84E
:109AB800019091F802A091F82470002A55D19B6971
:109AC80013F0400308BFCB70FFF7CEFF804648462F
:109AD800FFF7CAFF02465046FFF7C6FF81463846E1
:109AE800FFF7C2FF0B6ACF78234343EA875343EA61
:109AF800090343EA084343EA022343EA0063354A79
:109B0800CA205062532050628C6A8869B4F5807FFD
:109B1800946945D124F4885494610124D465B6F538
:109B2800807F09BFCB6913640343536418BF506433
:109B3800284B4A681A672A6B42F001022A639A691D
:109B480042F488529A61244AD2F8803043F40033B0
:109B5800C2F880301F4BFF225A620020012385F88B
:109B68002D3085F82C00BDE8F087B4F1803F07D090
:109B7800B4F5000F04D09B6913F0400308BFCB7005
:109B88000B6ACA781C4344EA0A0444EA004343EADD
:109B9800092343EA825343EA0763B0E70023AEE7A9
:109BA80024F4085494610224D465B6F5807F09BF73
:109BB800CB6993640343D36418BFD064054B4A68E8
:109BC8005A672A6B42F002022A639A6942F40852E1
:109BD800B8E700BF002800400008005890F82C2083
:109BE800012A03464FF0020012D00A4A83F82D00DA
:109BF800CA21516253215162916941F0200191615A
:109C0800FF2151620020012283F82D2083F82C00C7
:109C1800704700BF0028004090F82C20012A034616
:109C28004FF0020019D00D4A83F82D00CA21516265
:109C38005321516291690A4841F080019161D0F83D
:109C4800801041F48021C0F88010FF21516200206B
:109C5800012283F82D2083F82C007047002800404B
:109C680000080058064B5A6D520610B5044603D535
:109C78004022DA65F9F7B6F8012384F82D3010BDD3
:109C8800002800407047890001F1804101F5314109
:109C98000A607047890001F1804101F53141086887
:109CA80070470000034AD2F8903043F40043C2F8EA
:109CB8009030704700040058034AD2F8903023F4DB
:109CC8000043C2F89030704700040058074B1A68E8
:109CD80022F040021A6040F441704FF4B852186004
:109CE8005A601A6842F040021A6070470000015832
:109CF80037B5054600284ED0837903F0FF046BB1D1
:109D0800032C0BD0254B4FF400629A612868FFF7AB
:109D1800DDFF002401232B71AC602FE000236B7161
:109D28002846F8F703FE1E4AD2F8903043F48053D1
:109D3800C2F89030002CE5D102234FF0B042AB714D
:109D4800D2F8943023F40043C2F89430154B1B68C2
:109D58001C214B43DB0C64214B430193019B93B9BA
:109D68000124AC60FFF79EFF0C4B9A6842F4006236
:109D78009A604FF400629A61002CC7D00123AB713E
:109D8800204603B030BD019B013B0193D2F89430CB
:109D98005B04E3D4E6E70124F2E700BF00040058BF
:109DA800000800582808002037B5174D2B680246D0
:109DB8001C204343DB0C6420434314480193019B5C
:109DC80093B901209060114C21732B681C214B43DF
:109DD800DB0C64214B430193019B6BB9012090601C
:109DE8000A4BDB6803B030BD019B013B01938368DC
:109DF8009C07E4D50020E6E7019B013B0193A3689B
:109E0800DB07E9D5ECE700BF28080020000001586F
:109E180037B5184D2B6802461C204343DB0C6420E1
:109E2800434315480193019BA3B901209060124C4C
:109E3800FF2323732B681C256B43DB0C64256B43C2
:109E48000193019B73B9012090600B4BDB680B7089
:109E580003B030BD019B013B019383689C07E2D5A9
:109E68000020E4E7019B013B0193A368DB07E8D5E9
:109E7800EBE700BF28080020000001580F4B13B57E
:109E88001B680F4C182253431B0D64225343014691
:109E980001936269019B02F0040223B902238B60DB
:109EA800012002B010BD019B013B0193606910F0D5
:109EB8000200F6D0002AECD11046F2E7280800206C
:109EC8000004005807B50379012B0FD10A4B1B6812
:109ED800182253431B0C0193FFF7EEFE019B013B35
:109EE8000193019B002BF9D1FFF7DCFE03B05DF86D
:109EF80004EBFFF7C3BF00BF28080020F8B51E46D3
:109F08008379012B154604460F46DAB22DD14379E1
:109F1800012B2AD0022342718371FFF7D3FF0D2151
:109F28002046FFF7C9FEFFF73FFF390A2046FFF733
:109F38003BFFF9B22046FFF737FF2E44B5420ED15A
:109F48002046FFF7AFFEFFF799FFA068012300380E
:109F5800A3714FF0000318BF01206371F8BD15F815
:109F6800011B2046FFF720FFE8E70220F6E7F8B5D7
:109F78001E468379012B154604460F46DAB22FD1C7
:109F88004379012B2CD04271FFF79CFF1D212046FD
:109F9800FFF792FEFFF708FF390A2046FFF704FF94
:109FA800F9B22046FFF700FF00212046FFF7FCFE2C
:109FB8002E44B5420ED12046FFF774FEFFF75EFF30
:109FC800A06801230038A3714FF0000318BF0120D7
:109FD8006371F8BD29462046FFF71AFF0135E8E707
:109FE8000220F6E7F8B51F468379012B154604468B
:109FF8000E46DAB22CD14379012B29D04271FFF7F2
:10A0080061FF06F0EF03A3F1840253425341237129
:10A0180031462046FFF750FEFFF7C6FE2F44AF42F9
:10A0280010D1FFF73FFE842E02D02046FFF726FF0F
:10A03800A06801230038A3714FF0000318BF012066
:10A048006371F8BD15F8011B2046FFF7ADFEE6E782
:10A058000220F6E7F8B51E468379012B154604461B
:10A068000F46DAB227D14379012B24D04271FFF78A
:10A0780029FF39462046FFF71FFEFFF795FE00210E
:10A088002046FFF791FE2E44B5420ED12046FFF739
:10A0980009FEFFF7F3FEA06801230038A3714FF013
:10A0A800000318BF01206371F8BD29462046FFF759
:10A0B800AFFE0135E8E70220F6E737B50023ADF833
:10A0C800043001AA022312210546FFF7C3FFBDF899
:10A0D8000440022364BA01AAA4B219462846FFF72D
:10A0E80081FFE20702D5284609F0F6F9A30702D551
:10A0F800284609F0F7F9600702D5284609F01CFA46
:10A10800210702D5284609F01DFAE20602D528469D
:10A1180009F01EFAA30602D5284609F007FA6006D8
:10A1280002D5284609F0E4F9210606D514F4807111
:10A1380018BF0121284609F0E1F9A20502D52846F1
:10A1480009F0ECF9630402D5284609F007FA03B0D0
:10A1580030BDF8B51E468379012B154604460F46D7
:10A16800DAB227D14379012B24D04271FFF7AAFE36
:10A178000E212046FFF7A0FDFFF716FE39462046C0
:10A18800FFF712FE2E44B5420ED12046FFF78AFD96
:10A19800FFF774FEA06801230038A3714FF0000395
:10A1A80018BF01206371F8BD15F8011B2046FFF7A1
:10A1B800FBFDE8E70220F6E7F8B51E468379012B98
:10A1C800154604460F46DAB22BD14379012B28D025
:10A1D8004271FFF777FE1E212046FFF76DFDFFF75E
:10A1E800E3FD39462046FFF7DFFD00212046FFF753
:10A1F800DBFD2E44B5420ED12046FFF753FDFFF795
:10A208003DFEA06801230038A3714FF0000318BF7A
:10A2180001206371F8BD29462046FFF7F9FD013595
:10A22800E8E70220F6E7026852E8003F23F0C0039F
:10A2380042E8003102680029F5D102F1080353E829
:10A24800003F23F4000302F1080C4CE80031002918
:10A25800F3D12023C0F888307047000010B5026899
:10A2680052E8003F23F4907342E800310268002965
:10A27800F5D10F4C02F1080353E8003F234002F1E7
:10A28800080C4CE800310029F4D1C36E012B07D12A
:10A2980052E8003F23F0100342E800310029F7D1CB
:10A2A8002023C0F88C300023C366436710BD00BF6D
:10A2B800FEFFFFEFF8B504461346D4F88850202D6A
:10A2C80032D1F1B1EAB1E06FA4F85620A4F85420D5
:10A2D80000262122C4F890602165C4F888202268ED
:10A2E80088B1124FC762124F0763124F2832C0E974
:10A2F8000D76FDF745FE30B11023C4F89030C4F850
:10A30800885001200FE0236840221A62226802F177
:10A31800080353E8003F43F0800302F1080141E8D5
:10A3280000300028F3D1F8BD0220FCE741A3000863
:10A3380089A3000895A3000808B50346806A1B682E
:10A348001B6813F0200317D1A0F85630026802F1F9
:10A35800080353E8003F23F08003083242E8003145
:10A3680002680029F2D152E8003F43F0400342E876
:10A3780000310029F7D108BDF8F78AFEFBE77047DE
:10A3880008B5806AFFF7FBFF08BD7047806A38B5DB
:10A398000468D0F88830D0F88C50A268120606D528
:10A3A800212B04D10023A0F85630FFF73CFFA36807
:10A3B8005B0606D5222D04D10023A0F85E30FFF7F6
:10A3C8004DFFD0F8903043F01003C0F89030FFF7FD
:10A3D800DCFF38BD08B5806A0023A0F85E30A0F81D
:10A3E8005630FFF7D2FF08BD704700000368D969EF
:10A3F8001A682DE9F04140F60F0631429D6804467F
:10A4080010D18E0640F1978002F0200605F08057A3
:10A418003E4300F09080436F002B00F08580BDE83C
:10A42800F0411847AB4EAC482E401040304300F086
:10A438008280CF0709D5D00507D501201862D4F846
:10A44800900040F00100C4F890008F0709D5E80794
:10A4580007D502201862D4F8900040F00400C4F830
:10A4680090004F0709D5E80707D504201862D4F8EB
:10A47800900040F00200C4F890000F070BD502F0DE
:10A488002000304307D008201862D4F8900040F02C
:10A498000800C4F890000E050AD5500108D54FF4FD
:10A4A80000601862D4F8903043F02003C4F890306C
:10A4B800D4F89030002B37D08B0609D502F0200253
:10A4C80005F080552A4303D0636F0BB120469847A7
:10A4D8002668D4F89020B36802F0280203F04003FD
:10A4E80053EA0205204621D0FFF7B8FEB3685F069D
:10A4F80017D5226802F1080353E8003F23F0400310
:10A50800083242E800310029F3D1D4F8800040B184
:10A51800724B8363FDF7ADFD30B1D4F88000836BD7
:10A528007DE72046FFF731FFBDE8F081FFF72DFFFB
:10A53800C4F89050F8E7E06E012840F08980CE0614
:10A5480040F18680D00640F1838010221A629A6812
:10A5580051064BD5D4F8802011684A6892B2002A77
:10A56800E2D0B4F85C009042DED9A4F85E200A6814
:10A5780092062FD453E8002F22F4807243E800217A
:10A588000029F7D103F1080252E8002F22F0010256
:10A5980003F1080040E800210029F3D103F1080283
:10A5A80052E8002F22F0400203F1080040E80021A1
:10A5B8000029F3D12022C4F88C20E16653E8002F4B
:10A5C80022F0100243E800210029F7D1D4F88000D6
:10A5D800FDF71AFD02232367B4F85E30B4F85C1067
:10A5E800C91A89B22046FFF7FFFE9DE7B4F85E203E
:10A5F800B4F85E00B4F85C1080B292B2002893D030
:10A60800891A89B200298FD053E8002F22F490725A
:10A6180043E800200028F7D1314D03F1080252E841
:10A62800002F2A4003F1080646E800200028F4D14C
:10A638002022C4F88C206067E06653E8002F22F0DF
:10A64800100243E800200028F7D102232367C9E756
:10A65800CF0209D56E0207D54FF4801220461A6240
:10A66800BDE8F04100F0A0BD08060BD502F080005F
:10A6780005F40005284305D0A36F002B3FF454AF21
:10A688002046CCE64F0611D556060FD553E8002FC5
:10A6980022F0400243E800210029F7D12023C4F822
:10A6A8008830A1672046F8F7F3FC3DE70D0206D590
:10A6B800500004D52046BDE8F04100F077BDCB013D
:10A6C8007FF532AF002ABFF62FAF2046BDE8F04134
:10A6D80000F06BBD0100001020010004DDA300089C
:10A6E800FEFFFFEFD0F88C20B0F86010222A08B5E2
:10A6F800036855D15B6A826D0B401370836D01331B
:10A708008365B0F85E30013B9BB2A0F85E30B0F8CC
:10A718005E309BB2002B42D1026852E8003F23F41E
:10A72800907342E8003103680029F5D103F108026B
:10A7380052E8002F22F0010203F1080C4CE8002136
:10A748000029F3D12022C0F88C20184A416793428F
:10A75800016705D1C26E012A0ED0F8F7A7FC1EE0EA
:10A768005A681102F6D553E8002F22F0806243E8B8
:10A7780000210029F7D1EDE70022C26653E8002F37
:10A7880022F0100243E800210029F7D1DA69B0F875
:10A798005C10D20644BF10221A62FFF725FE08BDDE
:10A7A8009A6942F008029A61F9E700BF0080004008
:10A7B800D0F88C20B0F86010222A08B5036852D16E
:10A7C8005A6A1140826D22F8021B8265B0F85E2039
:10A7D800013A92B2A0F85E20B0F85E2092B2002A48
:10A7E80040D153E8002F22F4907243E80021002959
:10A7F800F7D103F1080252E8002F22F0010203F119
:10A80800080C4CE800210029F3D12022C0F88C2044
:10A81800174A41679342016705D1C26E012A0ED0DB
:10A82800F8F744FC1EE05A681102F6D553E8002FE9
:10A8380022F0806243E800210029F7D1EDE70022E9
:10A84800C26653E8002F22F0100243E800210029D5
:10A85800F7D1DA69B0F85C10D20644BF10221A6248
:10A86800FFF7C2FD08BD9A6942F008029A61F9E74C
:10A87800008000402DE9F74F0368B0F86080DF6979
:10A888001A689D68D0F88C1001922229044640F07D
:10A89800B480B0F86890DFF86CA1DFF86CB10026DE
:10A8A800B9F1000F01D0BB0621D4B4F85E309BB2D9
:10A8B800D3B1B4F868209A4216D9226802F1080385
:10A8C80053E8003F23F08053083242E80031226801
:10A8D8000029F2D14D4B636752E8003F43F0200353
:10A8E80042E800310029F7D103B0BDE8F08F2368B2
:10A8F800A26D5B6A03EA08031370A36D0133A365B5
:10A90800B4F85E30013B9BB2A4F85E302368DF697F
:10A9180078072CD0F9070AD5019AD20507D5012165
:10A928001962D4F8901041F00101C4F89010B807EA
:10A9380009D5E90707D502211962D4F8901041F02A
:10A948000401C4F890107A0709D5E80707D504214F
:10A958001962D4F8903043F00203C4F89030D4F868
:10A96800903023B12046FFF710FDC4F89060B4F88A
:10A978005E309BB2002B93D1216851E8003F23F44D
:10A98800807341E8003023680028F5D103F10802FC
:10A9980052E8001F01EA0A0142E800100028F5D138
:10A9A80020215B45C4F88C10606720670AD059687D
:10A9B800090207D553E8001F21F0806143E8001021
:10A9C8000028F7D1E16E012913D1E66653E8001F8C
:10A9D80021F0100143E800100028F7D1D969CA0610
:10A9E80044BF102119622046B4F85C10FFF7FCFC44
:10A9F80056E72046F8F75AFB52E79A6942F00802F0
:10AA08009A6171E7FEFFFFEF00800040EDA60008A5
:10AA18002DE9F74F0368B0F86080DF691A689D6810
:10AA2800D0F88C1001922229044640F0B280B0F888
:10AA38006890DFF868A1DFF868B10026B9F1000F67
:10AA480001D0BB0621D4B4F85E309BB2D3B1B4F8C0
:10AA580068209A4216D9226802F1080353E8003F99
:10AA680023F08053083242E8003122680029F2D1ED
:10AA78004C4B636752E8003F43F0200342E8003143
:10AA88000029F7D103B0BDE8F08F2368A26D596A99
:10AA980008EA010122F8021BA265B4F85E20013A17
:10AAA80092B2A4F85E20DF6978072CD0F9070AD59E
:10AAB800019AD20507D501211962D4F8901041F006
:10AAC8000101C4F89010B80709D5E90707D5022194
:10AAD8001962D4F8901041F00401C4F890107A0774
:10AAE80009D5E80707D504211962D4F8903043F056
:10AAF8000203C4F89030D4F8903023B12046FFF711
:10AB080044FCC4F89060B4F85E309BB2002B95D139
:10AB1800216851E8003F23F4807341E8003023683E
:10AB28000028F5D103F1080252E8001F01EA0A01E2
:10AB380042E800100028F5D120215B45C4F88C10AC
:10AB4800606720670AD05968090207D553E8001FD3
:10AB580021F0806143E800100028F7D1E16E012957
:10AB680013D1E66653E8001F21F0100143E80010F6
:10AB78000028F7D1D969CA0644BF102119622046B6
:10AB8800B4F85C10FFF730FC58E72046F8F78EFA67
:10AB980054E79A6942F008029A6173E7FEFFFFEFF3
:10ABA80000800040B9A7000838B504460368216949
:10ABB800A2681D68C0690A4361690A437D49024366
:10ABC80029400A431A605A68E16822F440520A434D
:10ABD8005A60794AA16993421CBF226A11439A6854
:10ABE80022F06E4222F430620A439A60DA6A616A9D
:10ABF80022F00F020A43DA62704A93421CD14FF0E6
:10AC0800B043D3F8883003F0030343F44033A3F58B
:10AC18004033013B022B00F2C780694A9B5CB0F5C8
:10AC2800004F40F08980082B24D8DFE803F061C08A
:10AC38008323802323236500624A934209D14FF07E
:10AC4800B043614AD3F8883003F00C0343F440233F
:10AC5800E4E7594A93420DD14FF0B043D3F8883016
:10AC680003F44063B3F5006F1AD005D853B1B3F5B8
:10AC7800806F12D0012009E0B3F5406FFAD14FF48C
:10AC880000400EE0FEF7D2FC58B900204FF0011347
:10AC9800A3660023C4E91D3338BDFEF7CFF8F3E7F8
:10ACA8004A4865684A4B626A05EB450133F8122049
:10ACB800B0FBF2F39942DDD8B3EB053FDAD80023B5
:10ACC8001946F6F721FF090241EA10616B080002F4
:10ACD800C0182A464FF0000341F10001F6F714FFAF
:10ACE8003C4BA0F540729A42C4D82368D860CCE7A0
:10ACF800FEF79CFC0028C8D06168354B626A33F8BF
:10AD08001220B0FBF2F24B0803EB42034FF6EF724E
:10AD1800B3FBF1F3A3F110019142ABD823F00F027A
:10AD2800216892B2C3F342031343CB60ADE7FEF749
:10AD380085F8DFE72548DFE7082B9BD801A252F802
:10AD480023F000BF95AD0008A1AD0008ADAD000827
:10AD58007DAC0008A7AD00087DAC00087DAC0008FC
:10AD68007DAC000871AD00084FF400406368616A6B
:10AD7800174A32F81120B0FBF2F000EB5300B0FB99
:10AD8800F3F04FF6EF73A0F11002ACE7FEF74EFCBC
:10AD980000283FF47AAFE9E7FEF758FCF8E7FEF73A
:10ADA8004DF8F5E70948E1E7B0F5004FF4D1FEF7B3
:10ADB8004DFC9FE7F369FFCF008000400038014059
:10ADC800BC4F010800440040BF4FF5070024F400C1
:10ADD800CC4F0108FFFC0F00836ADA0710B506D5CF
:10ADE8000168C46A4A6822F4003222434A609C0718
:10ADF80006D50168046B4A6822F4803222434A600F
:10AE0800590706D50168446B4A6822F48022224318
:10AE18004A601A0706D50168846B4A6822F4004222
:10AE280022434A60DC0606D50168C46B8A6822F4AE
:10AE3800805222438A60990606D50168046C8A68A4
:10AE480022F4005222438A605A060FD50168446CE6
:10AE58004A6822F480122243B4F5801F4A6005D163
:10AE68004A68846C22F4C00222434A601B0606D555
:10AE78000268C16C536823F400230B43536010BD70
:10AE88002DE9F041DDF8188004460E4615461F46A8
:10AE98002268D36936EA03030CBF01230023AB42BF
:10AEA80001D0002027E0B8F1FF3FF2D0F7F726FEE7
:10AEB800C01B4045206802D8B8F1000F1DD150E8EA
:10AEC800003F23F4D07340E80032002AF7D100F1A4
:10AED800080353E8003F23F0010300F1080141E8AB
:10AEE8000032002AF3D12023C4F88830C4F88C300B
:10AEF80084F884200320BDE8F08103685A07C7D589
:10AF0800C3691B05C4D54FF40063036250E8003FD2
:10AF180023F4D07340E80032002AF7D100F1080387
:10AF280053E8003F23F0010300F1080141E8003233
:10AF3800002AF3D12023C4F88830C4F88C30C4F830
:10AF48009030D5E773B504460026C0F89060F7F74F
:10AF5800D5FD23681B681A07054619D423681B68A2
:10AF68005B070AD56FF07E43009300222B464FF40F
:10AF780080012046FFF784FFB0B900202023C4F8E1
:10AF8800883084F88400C4F88C30E06620670CE0D0
:10AF98006FF07E430093324603464FF4001120467B
:10AFA800FFF76EFF0028D9D0032002B070BD10B59E
:10AFB800044650B3D0F888301BB980F88430F7F7CE
:10AFC80053FF22682423C4F88830136823F0010350
:10AFD80013602046FFF7E8FD012816D0A36A13B1D5
:10AFE8002046FFF7F9FE23685A6822F490425A6017
:10AFF8009A6822F02A029A601A6842F001022046F2
:10B008001A60BDE81040FFF79DBF012010BD000089
:10B0180030B581658168A0F85C200023B1F5805FB8
:10B02800A0F85E20436735D10369002B40F2FF1377
:10B0380018BFFF23A0F860300023C0F89030222307
:10B04800C0F88C30016801F1080353E8003F43F071
:10B058000103083141E800340368002CF2D1456E41
:10B0680084680169B5F1005F34D1B0F86850954241
:10B0780030D8B4F5805F1DD1254A264C002918BF69
:10B0880022464267C1B153E8002F42F4807243E878
:10B098000021F7E729B90369002B14BF7F23FF2399
:10B0A800C8E7B1F1805FC5D10369002B0CBF7F23CE
:10B0B8003F23BFE7174AE4E703F1080252E8002FED
:10B0C80042F0805203F1080040E800210029F3D142
:10B0D800002030BDB4F5805F0FD10F4A0F4C002916
:10B0E80018BF2246426751B153E8002F42F49072CC
:10B0F80043E800210029F7D1EAE7084AF2E753E8D4
:10B10800002F42F0200243E800210029F7D1DFE7B1
:10B1180019AA00087DA80008B9A70008EDA600082C
:10B12800D0F88C30202B30B415D1B9B1B2B100238E
:10B138000468C3660A4B9C420AD063681B0207D5A1
:10B1480054E8003F43F0806344E80035002DF7D110
:10B1580030BCFFF75DBF022030BC70470120FBE721
:10B1680000800040436E30B52BB90123A0F86A3047
:10B17800A0F8683030BD0368094D9A689968094C91
:10B18800490FC2F342626B5C615CDB00B3FBF1F315
:10B19800A0F86A30AB5CA25CDB00B3FBF2F3E7E734
:10B1A800EC4F0108E44F01087047704770471FB51E
:10B1B80004AB03E9060090F88430012B04463AD02A
:10B1C800012380F884302423C0F8883003681A6883
:10B1D80022F001021A609A6822F440120A439A6027
:10B1E80071B95A68BDF80C009DF80E1022F01002D3
:10B1F80002435A605A6822F07F4242EA01625A606A
:10B208001A6842F001021A60F7F778FC6FF07E4284
:10B21800034600924FF4800100222046FFF730FEDB
:10B2280038B92023C4F88830002384F8843004B067
:10B2380010BD0320F8E70220F9E790F88430012BCD
:10B248000FD0012380F88430016851E8002F42F0C4
:10B25800020241E80023002BF6D180F8843018461A
:10B2680070470220704710B590F88430012B0446CF
:10B2780017D02423C0F8883003681A68196821F0A9
:10B288000101196042F000524FF0005141661A6006
:10B29800FFF768FF2023C0F88830002084F8840076
:10B2A80010BD0220FCE770B590F88430012B0446ED
:10B2B80017D005682423C0F888302E682B6823F03F
:10B2C80001032B60AB6823F060431943A960FFF7C3
:10B2D80049FF20232E60C0F88830002084F88400BD
:10B2E80070BD0220FCE770B590F88430012B04464D
:10B2F80017D005682423C0F888302E682B6823F0FF
:10B3080001032B60AB6823F060631943A960FFF762
:10B3180029FF20232E60C0F88830002084F884009C
:10B3280070BD0220FCE7000038B5094D002455F82F
:10B33800043B33B90134E3B2052B64B2F7D10020E2
:10B3480038BD002CF6D01B6998470028F2D0F7E7E3
:10B35800701000207FB50A2301A88DF8043003F08F
:10B36800D9F80038044B059A1A6018BF01204042EA
:10B3780007B05DF804FB00BF6810002070B50446F4
:10B388000B46144962784A700020A2780A72087045
:10B398001A884A729A788A72DB780B746368CB6071
:10B3A8000D4B1B68DA6A2AB1237803F0FB030B2BD9
:10B3B80000D09047094E002556F8043B1BB19B6A04
:10B3C8000BB1204698470135EBB2052B6DB2F3D18E
:10B3D80070BD00BF480800206C10002070100020CD
:10B3E80070B5044611480123037063784370A3784D
:10B3F8008372E368C360E37803762369437623792D
:10B4080043720B4B1B689B6A03B19847094E002592
:10B4180056F8043B1BB1DB690BB120469847013550
:10B42800EBB2052B6DB2F3D170BD00BF5C080020F4
:10B438006C1000207010002038B501F011FE0C4D82
:10B44800052455F8043B5BB15B694BB155F8043CE6
:10B458009B682BB1984718B155F8043C5B6998472D
:10B46800013C14F0FF04ECD1BDE83840FFF75CBFA5
:10B4780070100020014B1868704700BF681000204A
:10B4880000B58BB0012368468DF8003002F0BCFC93
:10B4980038B99DF80400003818BF01200BB05DF8DA
:10B4A80004FB0020FAE7000030B58BB0054601F038
:10B4B800BBFD0446002839D1FFF7E2FF012838D147
:10B4C80068468DF8004002F09FFC10B14FF0FF3045
:10B4D80004E09DF80430AB4202D100200BB030BD2F
:10B4E800012DF3D0022D11D0002DF7D1002BF4D06F
:10B4F80068468DF8045002F099FD0028E6D10E4BFD
:10B508001B681B6B002BE8D09847E6E7002BDDD1C2
:10B5180068468DF8045002F089FD0028D6D1064B04
:10B528001B681B6B002BD8D02846EDE76FF0010095
:10B53800D4E76FF00200D1E76C10002070B5324CF0
:10B54800324B94F9042094F9055090B00126022852
:10B558008DF804608DF809208DF80A500AD18DF80D
:10B568000800D871197202F09FFB01A802F0D2FFFF
:10B5780010B070BD4FF480701A715D71D880197267
:10B58800234B8DF808601B7853BB1E2306A88DF843
:10B598001C208DF8183002F049FD1F238DF8183053
:10B5A80006A823798DF81C3002F040FD21238DF880
:10B5B800183006A863798DF81C3002F037FD202377
:10B5C8008DF8183006A863798DF81C3002F02EFD2E
:10B5D80028238DF8183006A80E4B079302F026FD95
:10B5E80002F062FB012306A88DF818308DF81C3094
:10B5F80002F01CFD084B1B685B6A0BB103489847B7
:10B608006078FFF751FFB3E784100020300800206E
:10B6180064100020000300016C10002008B501F040
:10B6280003FD40B9FFF72CFF012806D0084B197A13
:10B63800D879FFF783FF012008BD064B1B68DB683C
:10B6480098470028F7D1BDE80840FFF76DBE00BF56
:10B6580030080020701000202DE9F04186B0054622
:10B668000C46164601F0E0FC002840F08D8001F001
:10B67800EDFC40B9FFF704FF012807D0444B197AC5
:10B68800D879FFF75BFF6FF002046DE0414F3B682C
:10B69800DB68984730B13A682B7812789A4201D023
:10B6A800002B6ED13C4FDFF8F4803C72003C18BF91
:10B6B800012498F8043068788DF8044069468DF8BC
:10B6C800123002F049FB002840D000238DF80430E6
:10B6D8000393ADF810306FF0060495E80300304B83
:10B6E80083E8030098F80430BB72314601A803F0E0
:10B6F80009F82C4B059A1A6011283FD801A353F872
:10B7080020F000BF6BB7000891B7000885B70008A4
:10B7180085B7000885B7000885B7000885B7000811
:10B728008FB6000885B7000885B7000885B70008F8
:10B738007FB7000885B7000885B7000891B70008EB
:10B7480091B7000891B7000879B700082B788DF8F1
:10B7580008306B78ADF810306B6803934FF0FF3406
:10B76800BBE7E31D18BF0024204606B0BDE8F08102
:10B778006FF00404F8E76FF00504F5E74FF0FF34C5
:10B78800F2E76FF00304EFE76FF00104ECE700BFA6
:10B7980030080020701000205C0800208410002071
:10B7A8006C0800206810002010B504468AB018B94B
:10B7B8004FF0FF300AB010BD002368468DF8003006
:10B7C80002F022FB0028F3D19DF804302370F1E742
:10B7D800F0B587B000220B462A498DF807200122D0
:10B7E8000A7042784A700446002A41D102790A72E6
:10B7F8001A884A729A788A72DB780B740369CB606C
:10B80800C378214D8DF80830037B8DF809308368A3
:10B8180003932B68DB6A0BB102A898472B689B6BD4
:10B8280013B1227E02B19847184E0025374656F8C4
:10B83800043B53B11A6A42B11A78E3789A4219D193
:10B8480056F8043C20461B6A98470135EBB2052B95
:10B858006DB2ECD10DF10700FFF7A6FF63793BB19C
:10B868000021012204A8ADF810100591FFF7F4FE9D
:10B8780007B0F0BD002DE8D13B68DB689847002889
:10B88800DED1E2E7480800206C100020701000208C
:10B8980010B504468AB018B94FF0FF300AB010BD91
:10B8A8001F2368468DF8003002F0AEFA0028F3D165
:10B8B800024A9DF9043023701371EFE784100020C9
:10B8C80000B58BB02223019068468DF8003002F055
:10B8D800ADFB003818BF012040420BB05DF804FBF7
:10B8E80070B5634C014618228EB0204605F066FFFD
:10B8F800F8F73AFE23784068012202FA03F1014082
:10B9080004D15C4B084607F04FFFFEE75A495B48F5
:10B918001A4602F011F818B14FF0FF300EB070BDA2
:10B92800262304A88DF8103002F080FB544E554DA4
:10B93800002870D1012333702B68DB690BB100201C
:10B948009847262304A88DF8103002F05DFA059B6D
:10B9580093F84820227093F8182193F81A316270EE
:10B96800A370454BD3E9020105F01AFE05460028ED
:10B97800D2D1454E062304A88DF8103002F044FABF
:10B98800059B736104A802F051FB022304A88DF8FB
:10B998001030059602F038FA0836032304A88DF80B
:10B9A8001030059602F030FA0F2605F0BDFE01238F
:10B9B80004A88DF814308DF8106002F037FB1023BE
:10B9C8000DEB03008DF810308DF8145002F02EFBAB
:10B9D80004238DF8103004A8A3788DF8143002F0F1
:10B9E80025FB39238DF8103004A86369059302F00C
:10B9F8001DFB02A920788DF8086003F051FF00387C
:10BA080018BF0120E0711420FFF75AFFE07903F016
:10BA180003F8284682E727238DF810302B681B6926
:10BA280043B104A802F0F0F92B6805981B694FF49C
:10BA3800EE619847262304A88DF8103002F0F6FA34
:10BA480050B9012304A88DF8103002F0DDF99DF8F3
:10BA58001430002B7FF46EAF3378002B7FF46CAF7B
:10BA6800052204A88DF81020059302F0DFFA78E784
:10BA780084100020F44F01089C100020B41000200E
:10BA8800641000206C1000204C10002037B50023F3
:10BA98000D4601930446C0B900F0D0FA0190019B0D
:10BAA800C3B10E4A0E4942F824300E4ADA620E4AF1
:10BAB8001A630E4A5A630E4A126892699A612846B6
:10BAC8005B68F2229847002006E001A900F0BCFA62
:10BAD8000028E4D04FF0FF3003B030BD70100020D4
:10BAE800580F002045B5000861B600085DB300088E
:10BAF8006C100020154B07B51860154B154A1A60D5
:10BB0800154A5A60154A9A60154ADA60154B026858
:10BB18001A6042685A6082689A60C268DA60124A9B
:10BB280001911A61114982695A610020FFF7AEFF3D
:10BB380048B901A800F086FA003818BF0120404231
:10BB480003B05DF804FB4FF0FF30F9E76C100020FC
:10BB5800B4100020E9B30008D9B70008F5BB000805
:10BB680085B300089C10002059F800083C08002004
:10BB780051B118B1012804D000207047044B0B6064
:10BB88007047044B0B60F7E74FF0FF30704700BF7A
:10BB9800000300010300010108B502F059FF002865
:10BBA80014BF6FF00100002008BD08B502F0A4F82A
:10BBB800002814BF6FF00100002008BD10B504462E
:10BBC8008AB018B94FF0FF300AB010BD202368467C
:10BBD8008DF8003002F018F90028F3D1024A9DF9D7
:10BBE800043023705371EFE7841000202DE9F041F1
:10BBF8002F4D304F00232B7043786B703B689B6A46
:10BC08008AB004460BB128469847DFF8AC80002676
:10BC180058F8043B1BB15B6A0BB1204698470136C4
:10BC2800F3B2052B76B2F3D12378052B2FD00C2B4A
:10BC380035D0012B25D1214C062368468DF80030DC
:10BC480002F0E2F80199E07905F0F0FC10B91C4B1C
:10BC5800019A5A611B48FFF71BFE1B48FFF7AEFF0E
:10BC68006B788BB9A371194B5878FFF71DFC3B68AB
:10BC78005B6A0BB1114898476B7813B9E07905F006
:10BC880065FD0AB0BDE8F081FF23A371EFE7104B13
:10BC980001225A74227A9A74627ADA74F1E7637824
:10BCA800002BEED00AB0BDE8F041FFF753BB00BF50
:10BCB8005C0800206C100020701000203008002064
:10BCC8004C10002034080020350800208410002083
:10BCD8004808002030B58BB0FFF767FF0446F0B97D
:10BCE80003F0BEFD831C1DD0F8B9134D2B685B69AA
:10BCF800DBB1262368468DF8003002F085F82B6802
:10BD080001985B694FF4EE61984703F0BBFD78B981
:10BD18002CB9094B1B68DB690BB1012098472046F9
:10BD28000BB030BD6FF00704EFE74FF0FF34ECE7DE
:10BD38004FF0FF34F3E700BF6C10002030B5064D1C
:10BD4800064C30B129B12860A160627101232370CB
:10BD580030BD00232B60FAE7F0100020C41000204B
:10BD6800014B1878704700BFC4100020024B1878A8
:10BD780000B15878704700BFC41000207047000019
:10BD8800064B1A784AB15A783AB10278012A04D196
:10BD9800027912B19A8901329A817047C410002041
:10BDA800074B1A7852B15A7842B10278052A05D160
:10BDB800017A427AD973012098731A74704700BFC8
:10BDC800C410002013B51A4C23783BB363782BB307
:10BDD800A27BA36862B10022A2730322A27105228A
:10BDE8001A70E27B5A70227C9A700122A27004E0D9
:10BDF800A278012A14D0042AF7D0E0228DF8002076
:10BE08000C48A27901938DF8012008F049F80A4BF3
:10BE18001B6B1BB1E17801226846984702B010BD40
:10BE28000222A271A2895A70110A1970E5E700BFAF
:10BE3800C4100020D810002078080020FFF7C2BFE7
:10BE480030B5794C23788DB0002B43D0437B002B41
:10BE580040D0657825B1837B13B9A3890133A381C9
:10BE6800C178E02936D1002D36D1027B042A31D1A0
:10BE78008368187801282DD1587801282AD1987814
:10BE8800012827D1DB78012B24D102206380A071FF
:10BE9800E56002A863708DF80C3021718DF80820D8
:10BEA800257402F0C3F8284602F0B6FD5F4B1B6804
:10BEB8005B6803B1984700225D4B00924FF0FF3159
:10BEC8005C4807F041FF41F288315A4808F022F8EF
:10BED800FFF778FF0DB030BD83681A78A2700A2A80
:10BEE800F8D8DFE802F0062124282A3D44658D8F22
:10BEF8009900504807F086FF00236370A3814B4CDC
:10BF080004238DF80830236802A81B788DF80C30BC
:10BF180002F08CF82368587802F07EFD23689B684D
:10BF2800002BD7D09847D5E70223A371D2E740F278
:10BF380001136380CEE70123FBE7A568037BA371A8
:10BF480004222A7062799A4228BF1A4600230133D4
:10BF5800D9B28A42BED98168C95C0131E954F6E791
:10BF680005238DF8083002A802F0D4FAB2E7314868
:10BF780007F048FF00236370A3812C4C04238DF83D
:10BF88000830236802A81B788DF80C3002F04EF8B0
:10BF98002368587802F040FD23689B6803B19847EE
:10BFA800254BDB6A002B95D001210220984791E7A9
:10BFB800027B032A0DD106228DF80820B3F8013040
:10BFC8005BBAADF80C3002A802F0A4FA0123A37002
:10BFD80080E7072AF7D18DF80820B3F8012052BA74
:10BFE800ADF80C201A79D978120242EA014259793F
:10BFF8000A4364214A4304929B798DF81430E2E79E
:10C008000A23AEE700228DF808205B788DF80C3003
:10C0180002A802F00BF85DE70D228DF808205B7886
:10C028008DF80C309FE700BFC4100020F0100020EE
:10C0380045BE0008D8100020780800200048704746
:10C0480078080020002070474FF0FF30704700004C
:10C05800044B054A93F81831022B18BF062382F8BF
:10C068008034704764180020D81F0020034BD3F891
:10C07800483313B15B6903B118477047D81F0020D4
:10C08800034A137843F002031370FFF7EFBF00BFB2
:10C09800D41F00201FB50A4B8DF8090093F87C20A7
:10C0A8008DF80A2093F88C2093F848000D3202A9E5
:10C0B8008DF8082003F0F4FBC0B205B05DF804FB6E
:10C0C8006418002010B50D4C04F57D7007F09AFE39
:10C0D80094F8103413B1012384F80F34084B93F803
:10C0E8001831022B02BF94F8813443F0100384F80E
:10C0F8008134BDE81040FFF7B9BF00BFD81F00204A
:10C108006418002010B50C4CD4F8403343F0800379
:10C11800C4F8403394F8103413B10020FFF7D2FF6D
:10C1280094F8813423F0120343F0120384F8813425
:10C13800BDE81040FFF78CBFD81F00202DE9F04163
:10C148002C4D95F81831022B07460E4602D02A4B83
:10C15800DB6A984702F01BFD044628B1022002F072
:10C168000CFD002002F00EFD95F81831012B17D1B7
:10C1780002F00FFD804630B1002002F0FFFC0020E5
:10C1880002F001FD444602F006FD48B1002002F02D
:10C19800F6FC002002F0F8FCBDE8F041FFF758BFBC
:10C1A800002CF9D1154C94F8802494F81034B2B9C5
:10C1B8000BB184F83574384602F090FEE86A07F04F
:10C1C800E7FDD4F8B4339842E6D30D4807F01AFED9
:10C1D80094F8813443F0100384F88134DCE70BB120
:10C1E80084F83564304602F079FE95F81831022B50
:10C1F800EED1D1E764180020FC560108D81F0020B2
:10C2080070230020074A10B5137843F00103137018
:10C21800FFF72CFFBDE81040034B0122002102204C
:10C2280007F0C2BAD41F00203D500108074A10B5D4
:10C23800137843F004031370FFF718FFBDE81040AC
:10C24800034B01220021022007F0AEBAD41F0020C0
:10C258004D5001082DE9F0410F4616461D4680460F
:10C2680007F08CFD0A4A0B4C1378278143F008032A
:10C27800C4E90008137066812573FFF7F7FEBDE86F
:10C28800F041054B01220021022007F08DBA00BFC2
:10C29800D41F0020E02400205D50010813B507F0EA
:10C2A8006DFD0D4B6C461860204607F0BBFC94E80A
:10C2B80003000A4A0A4B83E80300137843F010038B
:10C2C8001370FFF7D3FE074B01220021022002B0B2
:10C2D800BDE8104007F068BAF0240020D41F002001
:10C2E800102300206A5001082DE9F04192B006465B
:10C2F80002F04DFC002840F05681AC4D95F81831FD
:10C30800012B09D02B6BAA4C93B194F80431BBB123
:10C31800042B6FD0032003E002F03BFC18B10F2080
:10C3280012B0BDE8F08102F036FC0028EAD0F6E74A
:10C33800B5F81E31D4F81424013B53432B63E4E7CA
:10C348009C4803F0E4F9002840F0298194F80C3166
:10C3580023802B6B0C930DF1180895F839308DF864
:10C368003830404695F81C318DF83A3007F080FC9B
:10C37800D5F82431009302AF98E80600D5F82031AB
:10C38800384607F00CFC97E803000FAB83E803007E
:10C39800EB6A0D9300238DF844302388ADF84630BE
:10C3A80095F82C3101228DF839201BB98DF84420DD
:10C3B8008DF83930804B0093804B95F84800A3F1F5
:10C3C80073020CA903F0E1FAC0B10B28A8D1D4F884
:10C3D800841499B1002EA3D0D4F84033784843F0A0
:10C3E8002003C4F8403307F095FD754807F058FD61
:10C3F800002095E76F4803F0BEF9A4E795F8487068
:10C4080095F9693095F9392095F87D106D4E3846C3
:10C4180003F0CDFA009641B2EB6C95F850203846FF
:10C42800143603F063FA0096EB6C95F8502095F9F2
:10C43800701095F8480003F059FAD4F8C413AB6D9E
:10C44800D4F8D8230B44C4F8B033EB6D1344C4F8C4
:10C45800B43394F80431042B07D02B6E0B44C4F882
:10C46800B0336B6E1344C4F8B4330023089395F8C3
:10C478002C3183B108A802F061FC00284AD195F953
:10C48800390094F837629DF82070FFF703FE3E44A8
:10C4980080B2B0423CD300238DF8133095F8393080
:10C4A8008DF8213095F838308DF82230D5F8803065
:10C4B8000993D5F884300A93238894F81164ADF869
:10C4C8002C3095F84800404B8DF820600DF1130290
:10C4D80008A903F01FFA012384F8353495F8393098
:10C4E80084F836349DF8133084F83734D4F814348B
:10C4F800C4F84464C4F83C34C4F84C3402F04DFB2E
:10C5080050B1D4F8140402F05AFB28B1102007E700
:10C51800082005E7132003E795F81831012B01D10E
:10C5280002F04FFB02F03CFB0023059394F8043122
:10C5380095F9395094F81164BBB1042B7FF4EAAE35
:10C5480005A802F037FE60BB94F80C341BB994F8C8
:10C558000E34012B02D9059B013B0593154B059819
:10C568003246E9B202F098FE02E0124802F06CFE90
:10C57800A8B9D4F8403394F80C11218043F0020391
:10C58800C4F8403394F8103423B994F80C340133C8
:10C5980084F80C340D4B0E489B6A984728E7112005
:10C5A800BEE61220BCE60E20BAE600BF64180020E2
:10C5B800D81F0020E0200020941800205C240020D0
:10C5C8004023002090230020EC230020FC56010883
:10C5D800DA1F002073B5144C144D04F57876EB6C13
:10C5E80095F8502095F9781095F84800009603F0D2
:10C5F8007DF940F2012395F84800A4F8F23304F2DB
:10C608001C42314603F07EF958B194F81C3484F882
:10C618005E34074B00205B6B984794F8F33384F83B
:10C62800803402B070BD00BFD81F002064180020FD
:10C63800FC560108F8B5334D95F81841012C06460B
:10C648004BD0022C51D064B938B9D5E91B0105F19A
:10C65800740383E803002046F8BD01283DD0022872
:10C6680001D00324F7E7284F85F8180107F5737EF2
:10C67800BEE80F0007F5787CACE80F00DEF8003064
:10C68800CCF8003095F8E93087F8F363E3B195F812
:10C698000031022B18D1D5F804316B67C7F8E433A1
:10C6A80095F87D3095F8082187F8F03395F88C30A7
:10C6B80085F8782087F8F13397F8112487F8E02374
:10C6C80040F20133A7F8F233002387F810340F4BF8
:10C6D800DB6A9847FFF77EFFBDE702F063FA04467E
:10C6E8000028B8D185F81861B5E70028B9D1064BFC
:10C6F80085F81801062283F88024044BDB6A9847E2
:10C708003446A8E764180020D81F0020FC5601080A
:10C71800F0B5484C484EB4F8DC202287D4E92D0106
:10C7280094F8B12084F8692004F16C0282E80300CF
:10C73800D4E92F0104F1740282E80300B4F8C4209C
:10C74800A4F87C20D4F8CC20C4F884208FB0D4F886
:10C75800D020D4F8C810C4F888200025374AC4F877
:10C7680080100123A4F81E31C6F80C24C4E94E55E4
:10C7780084F82C51A56284F81B5184F83A50C4F807
:10C788003051A4F8345186F8105484F841518DF88A
:10C79800143004F5087394F84800A4F84251039340
:10C7A80003A904F52D73049303F088F8E36EC6F823
:10C7B800D03394F87D3086F8DC3394F88C3086F8E2
:10C7C800DD334FF48073A6F8DE3386F8CC5306F5D4
:10C7D80073770FCF06F578740FC43B68236040F277
:10C7E8000123A6F8F233D6F8483386F81154CDE978
:10C7F80001551BB15A685B6901920293104B06936D
:10C80800A3F144020792A3F1140208920D4A0A9276
:10C8180025330993A2F19C030B93A2F198030C937F
:10C8280001A9131D06A802F274620D9302F0A4F97F
:10C838000FB0F0BD64180020D81F002000010100CF
:10C848003424002048190020F8B50D4F0D4C0E4E29
:10C858000D4607F0D7FA3B6B984796F8480004F264
:10C868001C42294603F04EF848B194F81C3484F869
:10C878005E34706D7B6B9847EB7C84F88034F8BD30
:10C88800FC560108D81F0020641800200D4890F8B5
:10C89800113480F8B8330C4B93F8692080F8BB2327
:10C8A80093F87D2093F88C3080F8C933002380F802
:10C8B800C823A0F8CA3300F56E7100F56070FFF761
:10C8C800C3BF00BFD81F0020641800200F4890F88D
:10C8D8008034CBB190F8113480F8CC330C4BDA6E3D
:10C8E800C0F8D02393F87D2093F88C3080F8DD339E
:10C8F8004FF4807380F8DC23A0F8DE3300F5737101
:10C9080000F56670FFF7A0BF704700BFD81F002072
:10C918006418002070B5344C2421204604F064FFCC
:10C92800636A984218BF60624FF01C012F4814BF19
:10C938000125002504F058FF636C984218BF606415
:10C948004FF0FC012A4818BF45F0020504F04CFFDF
:10C95800D4F84431984218BFC4F844014FF0D401C8
:10C96800244818BF45F0040504F03EFFD4F81C32F3
:10C97800984218BFC4F81C024FF090011E4818BF17
:10C9880045F0080504F030FFD4F8B032984218BFDB
:10C99800C4F8B0024FF49461184818BF45F0100568
:10C9A80004F022FFD4F85437984218BFC4F854074B
:10C9B8004FF01401124818BF45F0200504F014FF89
:10C9C800D4F86C3798420F4B18BFC4F86C07D3F8EB
:10C9D800483318BF45F040052BB11B691BB12846E9
:10C9E800BDE87040184770BD641800208C180020FE
:10C9F800AC180020AC190020841A0020181B002055
:10CA0800BC1F0020D81F00202DE9F04F91B0002650
:10CA1800BD4F8DF81560054688469346ADF81860F9
:10CA2800B146C14502D311B0BDE8F08F15F8090031
:10CA380002F0C2F948444045F5DC15F8093009F11F
:10CA48000104023BE4B2112BEDD801A252F823F005
:10CA5800A1CA0008D1CA000891CB0008BDCB0008C4
:10CA68004DCC000871CC0008E5CC000819CD0008B1
:10CA780097CD00082FCA00082FCA0008F7CD000874
:10CA88002FCA00082FCA0008ADCE0008D3CE000870
:10CA980017CF000855CF0008052002F039FA88B1F1
:10CAA8000521002002F0F8F92B5D87F8503409F1D0
:10CAB800030409F102095FFA89F9E4B215F80930AB
:10CAC80087F85134A146ACE700238DF816308DF86D
:10CAD80017308DF81C308DF82030002E52D18B4E37
:10CAE800631E2B440D9396F81A318DF83A3096F858
:10CAF8007C308DF8393096F839308DF83B3096F81F
:10CB080038308DF83C3096F868308DF83D30D6F8DE
:10CB180028310C9308AB019307AB009396F84800B3
:10CB2800A8EB09090DF117030DF116020CA98DF8F0
:10CB3800389002F0FBFE8DF8150000F0070007287A
:10CB48000BD19DF8163086F839309DF8173086F8E5
:10CB580038309DF81C3086F8683000264FF00509FB
:10CB680006E001220DF11501032002F03BF8013621
:10CB7800F2B29DF82030B3FBF9F19142F1D8013BB4
:10CB88002344DCB201269DE72B5D604903F00F03C7
:10CB9800012281F81B3109F1020902FA03F3A1F815
:10CBA8001E315FFA89F9002206A9042002F01AF85A
:10CBB8004C4687E707238DF815302B5DC3F3021227
:10CBC80003F00F038DF8303009F10303DBB28DF861
:10CBD8003120EA5C09F10403DBB209F10504EB5CDE
:10CBE80009F102095FFA89F91B0443EA022315F8DF
:10CBF8000920DFF8189113436422534399F8480039
:10CC08000D930CA902F0A1FE00F00703072BE4B274
:10CC18008DF815000ED19DF8303089F8703089F8FC
:10CC280078300D9BC9F86C30C9F874309DF83130F4
:10CC380089F869308DF81800012206A9052001F04D
:10CC4800D1FF3FE7D7F8483363B11B6853B1984722
:10CC58000BF03F038DF818008DF81930022206A951
:10CC68000620ECE7FF20F3E703238DF815302B5D52
:10CC78008DF824300CAB089309F10303DBB209F1FA
:10CC88000604EA5C09F10403DBB208A9EB5C1B04A7
:10CC980043EA022309F10202D2B209F10509AA5CAA
:10CCA8001343642253435FFA89F90C9300230D93CD
:10CCB80015F809308DF83830144B93F8480002F015
:10CCC8004AFEC3B20028E4B28DF81530FFF6FAAE7A
:10CCD8008DF81830012206A90720B0E72B5D03F074
:10CCE8000F03012B4FF47A7238BF01235343074ACD
:10CCF80009F10209936503F57A73D3655FFA89F937
:10CD0800002206A9082051E7D81F00206418002037
:10CD18002B5D9C4CC3F340128DF81D2094F84800FD
:10CD2800C3F3001207A903F00F038DF81C208DF838
:10CD38001E3002F016FE09F1020901305FFA89F986
:10CD48003FF436AFBDF81C308F4AA4F87C309DF80C
:10CD58001E309DF81CA0D05CF4F758FE0223C4F8DE
:10CD680080000CA994F848008DF830308DF832A076
:10CD780002F096FD94F93930089040B29842B8BF55
:10CD8800184684F83900002206A909200EE7032373
:10CD98008DF815302B5D8DF8303009F10303DBB2C7
:10CDA80009F10504EA5C09F10403DBB209F102099F
:10CDB800EB5C5FFA89F91B0443EA022315F80920A2
:10CDC8001343642253430D936E4B0CA993F8480008
:10CDD80002F0CDFDC3B20028E4B28DF81530FFF69D
:10CDE80071AE8DF81830012206A90A2027E70A201B
:10CDF80002F08EF800283FF465AE0A21002002F008
:10CE08004BF80023ADF8263009F10203DBB24FF4EA
:10CE18007A71EA5C09F10303DBB20DF1300AEB5CCD
:10CE28001B0443EA02232A5D134309F10402D2B228
:10CE380009F1060409F10509AA5C5FFA89F943EAD0
:10CE4800026315F8092003934A4312125046ADF8BD
:10CE5800242006F0E7FE039B03F1965303F5A9137C
:10CE680003F5EC530893D7F83C3300930DF12009F0
:10CE780099E80600D7F838330AA806F090FE0B9B0D
:10CE880000939AE806000A9B484606F06DFE99E86A
:10CE9800030006F09FFE01F08FFE0123E4B287F83D
:10CEA80030340FE60D2002F033F800283FF40AAEC4
:10CEB8000D21002001F0F0FF97F88034043B012B8E
:10CEC8007FF600AE01F074FEFCE509F10203DBB267
:10CED8002A5DE95C09F10303DBB209F10504EB5CA7
:10CEE80009F104095FFA89F91B0415F8090043EAF6
:10CEF800012313436421594300F00F0001F059FE48
:10CF0800E4B28DF81800012206A9112097E60E2038
:10CF180001F0FEFF00283FF4D5AD0E21002001F0FE
:10CF2800BBFF09F10203DBB2184AE85C2B5D12680B
:10CF380009F1040409F103095FFA89F943EA0020B9
:10CF480015F80910E4B201F036FEBBE52A5D09F1D7
:10CF5800020309F1040409F10309DBB25FFA89F954
:10CF6800E95C15F809301B0443EA012313436420E4
:10CF7800584301F022FEE4B28DF81800012206A9F8
:10CF880013205CE66418002077500108E024002094
:10CF98000E4B93F88124920703D593F87F24012A36
:10CFA80006D90B4A92F81A1111B1916A01319162AE
:10CFB800002283F80C2483F8102483F80F24D3F874
:10CFC800402322F00202C3F840237047D81F0020F4
:10CFD8006418002010B5124C04F55A7006F012FFC0
:10CFE800D4F84033012023F02003C4F84033FFF77E
:10CFF8007BF998B10B2811D00A4B93F8393084F893
:10D008003634092094F80E3484F8393484F8350419
:10D0180001F064FFBDE81040FFF7BABF10BD00BFC4
:10D02800D81F002064180020074BD3F84023012A9A
:10D0380006D03AB993F88204013818BF0120704726
:10D048000020704701207047D81F0020034BD3F8F9
:10D058004003431E58425841704700BFD81F002064
:10D068002DE9F04FA5B0EFF3108172B6C04A002049
:10D078001368106081F31088BE4C002B00F0DA8032
:10D08800D9065FFA83FB6BD5BB4D95F81831022B97
:10D0980002D0BA4BDB6A9847EFF3108872B6B84FE4
:10D0A80006F06CFE3E68D4F8B013361A3144B54821
:10D0B80006F030FFB34806F0F3FED4F8B413B248D4
:10D0C800314406F027FFB04806F0EAFE88F31088DE
:10D0D80095F81831022B02D094F810348BB116232E
:10D0E8000EA995F848008DF8383002F0D9FBD4F82D
:10D0F800B4130C900144A54806F00CFFA34806F0B1
:10D10800CFFE3B6894F81124EB620AAF38468DF8DD
:10D118006020199306F0ACFDD5F82431009304AED5
:10D1280097E80600D5F82031304606F038FD96E835
:10D1380003001BAB83E80300D4F814341A9395F862
:10D148002C3195F84800003B18BF012318A98DF829
:10D15800613002F0AEFB94F810340BB984F8353422
:10D168001BF0080F3AD08A4B834D5F681E89B3F9CC
:10D178000A8093F90C90D5F8E420039200230793D2
:10D1880084F83834A4F81A3484F81D34C4F82034E8
:10D19800A4F8243484F82634C4F8283484F81834DD
:10D1A800C4F82C3484F83034744B94F88024DB6A47
:10D1B80084F87F24A4F87C8484F87E949847724885
:10D1C80006F020FE3146384601F0DFFC8246002892
:10D1D80000F0E680A4F8728484F874941BF0040FBD
:10D1E8001AD0654B93F81831022B02D0634BDB6AD7
:10D1F80098470220FEF72CFF84F8350401F06EFEF4
:10D2080094F8103413B1012384F80F3494F881345E
:10D2180043F0100384F881341BF0020F03D0062179
:10D228000520FEF78BFF1BF0010F03D0042103201C
:10D23800FEF784FF01F0C6FC94F88124D0065FD580
:10D24800002384F88234D4F84033190644BF23F00D
:10D258008203C4F8403312F0050F00F0C5820C2099
:10D2680001F056FE002800F0BF8294F88134DF07F1
:10D2780000F1BA825E0740F1CB82D4F8403323F044
:10D288000203C4F84033D4F8402382BB94F8815495
:10D2980015F001011EBF2B4662F3000384F88134A8
:10D2A80094F881345E0744BF6FF3820384F88134B5
:10D2B800012384F8823421B1D4F8443335481B68FB
:10D2C80098476D070BD5344801F02EFE01F05CFE3F
:10D2D80028B194F8813443F0040384F8813401F0D0
:10D2E80060FC94F881346FF3041384F881340123CB
:10D2F80084F8823494F8813443F0200384F881342C
:10D3080094F8813418070AD56FF3C303234984F8C6
:10D318008134D4F84433A1F12000DB68984794F8AD
:10D32800813499070AD56FF341031C4984F8813485
:10D33800D4F84433A1F164005B68984794F88034CA
:10D34800022B01D1FFF746F994F881349A0640F18F
:10D35800EC826FF3451384F88134D4F84033002B02
:10D3680040F0E38225B0BDE8F04FFFF7D3BA00BF25
:10D37800D41F0020D81F002064180020FC56010884
:10D38800F02400205823002070230020CC23002004
:10D39800E02400200C240020202400205424002015
:10D3A80095F81831012B0CD101F0F3FB804668B1D8
:10D3B800504601F0E3FB504601F0E5FB042384F8F6
:10D3C8007F347EB9012384F819344AE101F0E3FB84
:10D3D8000028F6D0404601F0D2FB404601F0D4FBCD
:10D3E8000523ECE73B7802935B09013B062B00F22F
:10D3F800ED81DFE813F00700EB019200EB018F00ED
:10D40800EB01DB01102EDDD995F82C310E97F6B221
:10D418008DF83C60002BD5D118A804F0F9F80EAAB5
:10D4280018A9FF2002F04CF89DF84830C3F3030315
:10D4380007468DF8203095F8480095F87D308DF82E
:10D448002130072208A902F03EFA002F5AD10028FD
:10D4580058D09DF843309DF842201199C5F8E41042
:10D468001B0443EA02239DF8412002201343C5F818
:10D47800E03004F0DBF89DF8483095F8480085F86E
:10D488002A71C3F30212C3F3030385F8703085F8D9
:10D4980078309DF8493085F86920012B38BF012381
:10D4A8004FF47A725343AB651344EB654FF00108B0
:10D4B8000DF14A03113E0CA90C9385F868808DF88C
:10D4C800346002F008FA0223404685F82C3101F056
:10D4D8001FFD18B14146384601F0DEFC94F81034BF
:10D4E800002B00F0798194F8383413B10020FEF74E
:10D4F800E9FD94F8813443F0100384F88134FEF791
:10D50800A7FD6BE6012001F003FD0028E6D001210C
:10D518000720E1E7012384F8183495F87D308DF869
:10D52800223094F81C348DF8213095F88C3095F819
:10D5380048000D3308A98DF8203002F0B1F9A6F1A2
:10D548000D031BB2069023EAE37300B283423FF750
:10D5580039AF0B2E7FF636AFA24B219318A8FF23C5
:10D5680018978DF864608DF8883002F075F8804659
:10D5780000287FF427AF9DF86C301A99C4F82C1452
:10D5880013F00F0203D09DF8800000286CD19DF89D
:10D59800880000286AD0002A7FF414AF9DF8802004
:10D5A800002A0CBF0227032700220792D5F8EC2097
:10D5B80091425DD195F8E910002959D0D5F80C11A0
:10D5C80095F8EAA00968079195F81811022902D17F
:10D5D800032184F87F14032F7FF4F4AE13F0600F57
:10D5E8007FF4F0AE03924FF00108152395F8480038
:10D5F8008DF8203008A902F053F995F82A310690E1
:10D60800BAF1000F37D0BAF1010F3ED1012B34D156
:10D618006FF009063E4106F00106C6F10206F6B2B1
:10D6280081B2BDF86E2007AB304601F0CFFD70B374
:10D63800072824D1082384F8193495F82A315BB9CE
:10D64800029B03F0E003A02B06D16A6B239B9A424E
:10D6580002D1012385F83A30079BC4F82834C4F86E
:10D668006034FEF74FFDB9E547469DE701279BE784
:10D678004FF0010AB9E70426D2E70326D0E70828C5
:10D6880003D10A2384F81934E6E70123FAE718AB33
:10D6980000930399079B3246504601F063FE20B180
:10D6A80002280CBF0B230C238DE6079BC4F82834F3
:10D6B800C4F860349DF86C3084F81904C3F340133F
:10D6C80084F8263484F8383494F87F3484F81A843B
:10D6D800012B98BFA862B8F1010FC4F8200484F8A0
:10D6E800240484F8350433D1022284F8182495F8E8
:10D6F8003A20002A3BD19DF86C20D20637D4012B62
:10D7080094F834149DF86C2005D8012901D19606A7
:10D7180001D501F001FB022F37D0032F09D09DF866
:10D728006C10012F4A4601F00F011CA831D0FFF7F9
:10D738006BF99DF8803084F81B34219BC4F82034A1
:10D748009DF8883084F82434012384F8253426E0B1
:10D75800029A02F0E002A02A11D195F82A110122BA
:10D7680085F83A2009B92399696384F8182495F84B
:10D778001821002AC3D1012284F81D24BFE7002202
:10D7880085F83A2084F81824B5E79DF88810219880
:10D798004A46FFF739F99DF8803084F81B3494F82D
:10D7A800813443F0020384F8813497E6DFF834804B
:10D7B800013EB2B2791C404604F000F80323A4F8F5
:10D7C8001834C4F8208484F82464E8E7012384F832
:10D7D8001934FEF797FC81E695F81831022B7FF48F
:10D7E80088AE83E61022002094F881345D070FD5B7
:10D7F800012001F08DFB88B3012001F05FFB08B91F
:10D8080084F80C04D4F8403323F00203C4F84033FE
:10D8180094F88114C8077FF536AD94F834340BB109
:10D82800032B26D1424B94F80C0493F868209042BD
:10D8380008D28A0750D593F818311BB194F87F3471
:10D84800002B49D13B4806F0DDFAD4F8403323F0E9
:10D858002003C4F84033FFF79BFB14E5062001F0D2
:10D8680057FB0028CED1072001F052FB0028C9D170
:10D87800CEE7012B30D194F80F24002A3FF403ADF2
:10D8880094F80E3494F80D04834204D211F0020285
:10D8980018BF94F83824264D95F82A11002941D14B
:10D8A80032BB834218D20133DBB2DF0784F80E346F
:10D8B80012D522238DF8603095F87C308DF86230CF
:10D8C80095F8480095F839308DF8613018A901F0BD
:10D8D800E7FF0E9085F8390094F8813400206FF343
:10D8E800041384F8813484F80F04FFF773FBCAE447
:10D8F80094F838648EB902238DF8683005F50873FA
:10D90800189395F8480005F52D7318A9199301F097
:10D91800D5FF84F8106484F8386494F80E3484F8D9
:10D9280039348FE7002AD7D08CE725B0BDE8F08FCF
:10D9380064180020402300202DE9F04F8A468BB060
:10D9480091460746002800F08D81002900F08A8161
:10D958000368002B00F086814368002B00F0828169
:10D968008368002B00F07E81C368002B00F07A8169
:10D97800104601F091FF002800F07681BC4CBD4DA7
:10D98800384601F03FFA4FF4EE620021204603F0DA
:10D9980029FF4FF4A1620021284603F023FFB64B6C
:10D9A800C4F8283100264FF001080F2305A948467E
:10D9B8008DF8143084F8489084F8186184F88C60E5
:10D9C80085F80E8485F80D8401F06AFF801B18BF66
:10D9D80001204FF00A0B84F81C0105A994F84800AF
:10D9E8008DF814B001F05CFF4FF0060984F8DC00F4
:10D9F80005A994F848008DF8149001F051FF102300
:10DA080084F8DD0005A994F848008DF8143001F079
:10DA180047FF1123C4F89C0005A994F848008DF825
:10DA2800143001F03DFF1223C4F8A00005A994F8B2
:10DA380048008DF8143001F033FF1323C4F8A40014
:10DA480005A994F848008DF8143001F029FF142333
:10DA58000DEB0301C4F8A80094F848008DF81430C1
:10DA680001F01EFF1723C4F8AC0005A994F848007C
:10DA78008DF8143001F014FF182384F8B10005A9BB
:10DA880094F848008DF8143001F00AFF1923C4F8FF
:10DA9800B400C4F8BC0005A994F848008DF8143007
:10DAA80001F0FEFEC0B21E2384F8B80084F8C0005E
:10DAB80005A994F848008DF8143001F0F1FE1F23F1
:10DAC80084F8C40005A994F848008DF8143001F0D2
:10DAD800E7FE202384F8C50005A994F848008DF8CE
:10DAE800143001F0DDFE2123C4F8C80005A994F81C
:10DAF80048008DF8143001F0D3FE0B23C4F8CC0095
:10DB080005A994F848008DF8143001F0C9FE0C23DB
:10DB1800A4F8D00005A994F848008DF8143001F055
:10DB2800BFFED4F89C306365D4F8A030A365D4F860
:10DB3800A430E365D4F8A8302366D4F8AC30636623
:10DB480004F5087307A90490A4F8D200079394F881
:10DB580048008DF8246004F52D73089384F8B0808C
:10DB6800C4F894B084F89890C4F84CB084F85090F5
:10DB780084F8688001F0A2FEC5F848A3FEF7C8FD46
:10DB880032463E4B00964FF0FF3105F55A70C4E916
:10DB98000B66C5F8447385F8816484F81981C5F863
:10DBA800408306F0D1F83246354B00964FF0FF31EE
:10DBB80005F5607006F0C8F83246324B00964FF013
:10DBC800FF3105F5667006F0BFF832462E4B009619
:10DBD8004FF0FF3102AE05F57D7006F0B5F830461E
:10DBE80006F046F896E8030004F5907383E803000E
:10DBF800264BC5F84C33264BC5F85433254BC5F88E
:10DC08005C33254F254BC5F85033254BC5F85833A1
:10DC180005F553703B68984704F5A47003F016FBAC
:10DC280020B1112630460BB0BDE8F08F204601F038
:10DC38009DFA0028F5D100F0C7FFB8B9194801F0DE
:10DC4800F7FA06460028ECD17B69984703F094FD63
:10DC5800BB6D94F819019847FB6A9847012385F82A
:10DC68008234DFE70326DDE70926DBE71326D9E759
:10DC780064180020D81F002000030001DDCF000831
:10DC880095C80008D5C80008CDC00008A5C200087E
:10DC98005DC2000889C00008FC56010835C20008AA
:10DCA8000DC200084C19002008B5034B0020C3F82A
:10DCB8004003FEF7CDF908BDD81F002010B5FFF7C7
:10DCC800B3F90A4C60B90A4B93F81831022B02D108
:10DCD800084BDB6A98470123C4F84033002010BD85
:10DCE800D4F84003013818BF0120F8E7D81F0020F6
:10DCF80064180020FC56010838B5134C04F55A7016
:10DD080006F080F804F5607006F07CF804F566709B
:10DD180006F078F804F57D7006F074F800F040FF1E
:10DD28000A4B0025DB6A9847C4F84053FEF7F2FD1A
:10DD3800074908484FF4EE6203F040FD0123C4F898
:10DD48004033284638BD00BFD81F0020FC560108C4
:10DD580064180020F410002030B52A4B89B005461D
:10DD680093F8DD008DF8020093F8DC009A6A8DF8CC
:10DD780003000020019202900C4600293ED0059233
:10DD8800D3F8882006921A8FD3F82811039152BA33
:10DD980093F81A11ADF81C2093F87C2093F84830BA
:10DDA8008DF810008DF811108DF81E208DF81F3099
:10DDB8000DF1030201AB0DF1020103A800F06EFEA4
:10DDC8009DF90200FEF766F9607002A800F0B6FF40
:10DDD800B0B9029A0F2A0DD863789A420AD8154426
:10DDE800AB42A3EB02012CBF002001202170C00030
:10DDF80009B030BD002323700820F9E70320F7E7B6
:10DE08001320F5E7641800201FB50446002800F029
:10DE1800FD8000783F2800F2F380DFE810F0400032
:10DE280046004B005000540058005D00F100F1001E
:10DE3800F100F100F100F100F100F1006400680068
:10DE48006C0077007E0081008400890087008B00C9
:10DE58008F009200950098009B009E00A200AA00E7
:10DE6800A600AE00B100B500BE00BA00BC00F100CB
:10DE7800C200F100F100F100F100F100F100F10041
:10DE8800F100F100F100F100F100F100F100F10002
:10DE9800CA00CE00D300D700DB00DF00E8005D4BEE
:10DEA80093F81831237104B010BD5A4B93F82C31F4
:10DEB800237102E0606803F065FB0020F3E7606807
:10DEC80003F0A6FBF9E7534B93F81A31F0E7514BEF
:10DED800D3F8E0306360F0E74E4B211D93F82C0136
:10DEE80003F0AEFBE9E74B4B93F81931E0E7494BF8
:10DEF80093F88C30DCE71D238DF80830454B02A9D8
:10DF080093F8480001F0CCFC6060D6E7424B04343B
:10DF180093E8030084E80300CFE7404B0434F7E7B5
:10DF28003F4B0434F4E73F4B0434F1E71B23E3E7AA
:10DF38001A23E1E7374B93F86830B9E7354B5B6D47
:10DF4800C8E7344B9B6DC5E7324BDB6DC2E7314BFD
:10DF58001B6EBFE72F4B5B6EBCE72E4B93F8DD3093
:10DF6800A6E72C4B93F83930A2E72A4B93F8DC301C
:10DF78009EE7284B93F838309AE7264BDB6CA9E7E5
:10DF8800244B93F8503093E7224BD3F884306360E6
:10DF980093E7204B9EE7244B9CE71E4BD3F8CC30ED
:10DFA800F5E71C4BD3F82831636001F00DFDA06044
:10DFB80083E7184BD3F890308CE7164BB3F88830CA
:10DFC800A3807AE7134BB3F88A30F9E7114BB3F81B
:10DFD800D030F5E70F4BB3F8D230F1E70D4B93F89B
:10DFE80048200AB1062A13D1B3F84C37E8E7094BA1
:10DFF80093F848200AB1062A0AD1D3F8503769E7BE
:10E00800204604B0BDE8104000F0CEBD03204AE72A
:10E01800182048E764180020D0180020181900209C
:10E02800D818002020190020F410002073B50446E9
:10E0380000285ED0A04DD5F840339A0700F15F82E2
:10E0480002783F2A00F25682DFE812F040004600CC
:10E058004E0056005A005F00640070007A007F008E
:10E06800840089008E00930098009D00A700540248
:10E07800AC00CC00DF000601280119012C013C018D
:10E088004001440148014C01500162018A017801B4
:10E098009C01A201A901AE01B30154021802540265
:10E0A80054025402540254025402540254025402B8
:10E0B80054025402540254025402540254022702D5
:10E0C8002C02310236023B0240024A02007902B0B9
:10E0D800BDE87040FEF7AEBA0379022B09D0774A43
:10E0E80082F82C31002005E0406803F03DFA002852
:10E0F800F8D0032002B070BD406803F079FAF6E763
:10E108006E4B027983F81A21ECE76C4B4268C3F82E
:10E11800E020E7E7694D416895F82C0103F086FA9D
:10E128000028E6D16368C5F8E430E3E741680029D0
:10E13800DFD0002001F0A8F90028D3D01120D9E7BA
:10E1480041680029D5D00120F4E741680029D0D0E2
:10E158000820EFE741680029CBD00920EAE74168A9
:10E168000029C6D00C20E5E741680029C1D00D2060
:10E17800E0E741680029BCD00E20DBE741680029B0
:10E18800B7D00F20D6E74E4C4C4B007983F81901D5
:10E19800A36D9847E36A9847A4E7484B027983F848
:10E1A8008C209FE7454D037A8DF8003095F848009C
:10E1B80095F87D308DF801300722694601F083FB20
:10E1C800002896D0636895F84800009300226946B5
:10E1D80001F079FB00288CD06C35D4E9010185E881
:10E1E80003007FE7354D037A8DF8003095F8480035
:10E1F80095F87D308DF801300722694601F063FB00
:10E2080000283FF476AFB435E7E72C4D037A8DF854
:10E21800003095F8480095F87D308DF801300722D8
:10E22800694601F050FB00283FF463AFD4E90101CF
:10E2380005F1740383E8030095F81831022B7FF485
:10E2480051AF95F82C31002B3FF44CAF1C4BDB6AD7
:10E258009847FEF7BFF945E7184D037A8DF8003067
:10E2680095F8480095F87D308DF801300722694609
:10E2780001F029FB00283FF43CAFBC35ADE743680B
:10E28800009301238DF804300C4B694693F848003D
:10E2980001F026FB00287FF425AF2AE743680093A6
:10E2A8000023EFE703795A1E0E2A3FF622AF034AEE
:10E2B80082F8683016E700BFD81F002064180020D5
:10E2C800FC560108904B42685A650BE78E4B426832
:10E2D8009A6507E78C4B4268DA6503E78A4B426820
:10E2E8001A66FFE6884B42685A66FBE6864C037955
:10E2F80094F848008DF800300622694601F0E3FAE8
:10E3080000283FF4F6AE9DF8003084F8DD30E9E6E9
:10E318007D4C03798DF8003094F8480094F87C30EF
:10E328008DF802300522694601F0CDFA00283FF445
:10E33800E0AE9DF8003084F83930D3E6724C0379AA
:10E3480094F848008DF800300A22694601F0BBFABB
:10E3580000283FF4CEAE9DF8003084F8DC30C1E6EA
:10E36800694C037994F848008DF800300922694611
:10E3780001F0A9FA00283FF4BCAE9DF8003084F8FB
:10E388003830AFE6604B4268C3F89420DA64A9E6F7
:10E398005D4B027983F8982083F85020A2E65A4B07
:10E3A8004268C3F884209DE6574B4268C3F8CC20E6
:10E3B80098E6012B40F0A380544C2421204603F01A
:10E3C80013FA636A984201D0172093E61C2104F1DE
:10E3D800280003F009FA636C9842F5D1FC2104F196
:10E3E800480003F001FAD4F844319842ECD1D42122
:10E3F80004F5A47003F0F8F9D4F81C329842E3D17C
:10E40800902104F5087003F0EFF9D4F8B03298427F
:10E41800DAD14FF4946104F52D7003F0E5F9D4F8DE
:10E4280054379842D0D1142104F5EB6003F0DCF99D
:10E43800D4F86C379842C7D1334E214630464FF452
:10E44800EE6203F0BBF920464FF4EE62002103F0C0
:10E45800C9F995F8113485F8E033736FC5F8E433DA
:10E4680096F87D3085F8F03340F20123A5F8F233B1
:10E47800274B96F819019B6D984733E68379012B52
:10E488003FF637AE204B42684068C3F8282100F0B9
:10E4980089FE00283FF42EAE50E61B4B4268C3F8B5
:10E4A80090201FE6184B8288A3F888201AE6164B9E
:10E4B8008288A3F88A2015E6134B8288A3F8D02017
:10E4C80010E6114B8288A3F8D2200BE60E4B93F886
:10E4D80048200AB1062A14D1A288A3F84C2701E6DD
:10E4E800094B93F848200AB1062A0AD16268C3F892
:10E4F8005027F7E502B0BDE8704000F057BB012097
:10E50800F8E51820F6E500BF64180020F410002094
:10E51800FC5601082DE9F04186B00023ADF8003023
:10E528000646002800F0E280FEF77EFD20B10124B7
:10E53800204606B0BDE8F08100F02CFD0028F6D199
:10E5480000F022FD014618B96948142203F04AF97F
:10E55800684D95F88134012243F0040385F8492475
:10E5680085F8813433788DF804300021013B8DF82B
:10E5780005208DF807100D2B00F2B080DFE803F0BE
:10E5880007AEAEAE525A7DAEAE85AEA28F9ED5F81E
:10E59800404314F02004CAD1DFF85C81574FFEF7DE
:10E5A800B7F8224696F9051098F8480001F0E5F901
:10E5B80088F83900B37988F83830204607238DF871
:10E5C8000530FEF737F8FF2307F58670A5F80C31FC
:10E5D80085F80441C5F8087103F01AF807F58A7040
:10E5E80002F0D0FF2046FDF77FFE044640B196F9C1
:10E5F800051098F84800012201F0BFF988F83900A1
:10E60800D5F884343361002C6CD000F0BDFC0028B0
:10E618008ED195F8813485F8100460F3820385F86B
:10E62800813485E700226946022000F0DBFA10B346
:10E638001324E5E795F811348DF808302E4BB2888D
:10E6480093F839108DF8091093F838108DF80A10DE
:10E65800D3F880100391D3F88410049193F84800FC
:10E66800ADF8142002A901F09DF9D5F8403343F024
:10E678000203C5F840330024C2E7214BB28896F95B
:10E688000C10B068DB6B9847EFE702A90D2000F08B
:10E6980027FB0028EFD0002269460D20C5E7164B5E
:10E6A80093F81831D3B9347904F0070000F077FAF9
:10E6B8008DF80040012269461020B6E7002269461D
:10E6C8001220B2E78DF8072000F05AFA044638B94C
:10E6D80000F053FA204600F055FA91E702248FE73C
:10E6E80001248DE701A800F0A1FB21E703241FE71F
:10E6F80020240020D81F002064180020DA1F0020E2
:10E70800FC5601082DE9F04F91B00026039105460B
:10E7180018B9032011B0BDE8F08FFEF785FC8246DA
:10E72800002840F06481B84C14220146074604F2E0
:10E73800344003F057F8012384F8353484F80E3454
:10E748002A789A4200F0B080032A00F0BF80002A9D
:10E7580040F0C98084F80D34022295F80490D5F869
:10E768000880AE8995F90EB062F347179A46A74B11
:10E77800022493F87C2093F848008DF8244009A9D6
:10E788008DF8262001F08CF8BAF1000F00F02D81E9
:10E798009E4B93F81A21B2B940B25845B8BF5846B3
:10E7A80093F87C208DF814008DF8162093F8480013
:10E7B800052205A901F087F80028AAD0934B9DF8F7
:10E7C800142083F83920198F1A8F93F82C0102919D
:10E7D800996A069152BA002800F0058193F81B0146
:10E7E80000B9186393F81801ADF83C20013893F884
:10E7F8007C208DF83E20D0F1000B93F848208DF84E
:10E808003F204BEB000B824A93F83A0093F81A41E9
:10E8180001900D914FF00100D3F88810D3F82831FA
:10E828008DF830000E910B93511C06AB0BA88DF898
:10E83800314000F033F9019B4FEA0B1B4BEA431BB5
:10E848004FF0000A4BEA801B4BEAC413D0456E4CCC
:10E85800019308BF56463246414604F59C709B46D4
:10E86800CDE907AAA4F800A084F810A402F0A6FF36
:10E87800F9B2A770C7F34217F2B2042F634E019B97
:10E8880084F8372233D0072F00F09D80022F32D032
:10E898000220029B33875C4B002283F810245A4BDA
:10E8A800D3F884342B6135E7EB7B082B28BF08238A
:10E8B80084F80D34042395F80490D5F80880AE89BF
:10E8C80095F90EB063F34717924650E784F80D3474
:10E8D800D5F804802E8995F90AB067F01F079A4683
:10E8E8004FF0000943E7D346D046D1463FE74FF003
:10E8F800010084F81004474F84F80D11042084F8AF
:10E908000401FF20D6F8E41084F80C0184F81431CF
:10E9180007A807F59B73C4F8087184F82891C4F810
:10E92800101184F83021C4F82C3100F043FC002881
:10E9380057D1079BA4F8380408A8A4F81631C4F8DE
:10E94800403400F0FBF960BB089BABB196F9390085
:10E95800FDF7A0FB94F837322BB3089B0F2B19D87F
:10E9680007F58B7208A90F2000F0F4F9C8B9089BC5
:10E9780063F3030B84F814B10398FDF7B5FC002882
:10E9880087D1069B86F83A00B36200F0B7F980B3E6
:10E99800132080E707F2864208A900F0DBF9002877
:10E9A800EAD0132075E707F286473A4608A900F02F
:10E9B800D1F90028F5D1089B84F82801C4F82C71F6
:10E9C80084F83031D8E7B8F1000FD5D0002AD3D079
:10E9D8004146E01C02F0F2FE94F8373201332380FE
:10E9E800CAE7122055E7072055E7204657E70120D8
:10E9F80090E62B7884F8343494F8813443F001039A
:10EA080084F881344BE700BFD81F00206418002029
:10EA18009C180020DA1F002037B50B4D8DF8040034
:10EA280004460F2295F8480001A900F04CFF40B1B8
:10EA3800064A85F81C4192F8813443F0200382F895
:10EA4800813403B030BD00BF64180020D81F0020F7
:10EA580010B5FFF733F90446A0B90B4805F0D2F911
:10EA68000A4805F0CFF90A4805F0CCF9094805F03D
:10EA7800C9F900F095F8FDF74BFE074BDB6A98479C
:10EA8800204610BD0124FBE7402300205823002026
:10EA980070230020CC230020FC5601082DE9F04FFC
:10EAA80090F802908BB004468A460192B9F1000FA3
:10EAB80060D14579816890F9102090F9118019602A
:10EAC800002D55D0817C8DF81610C07C4FF0020BBC
:10EAD80005A9CDE902238DF814B000F0E1FE029AF1
:10EAE80047B2BA421646B8BF3E46BA420CDC039B50
:10EAF800C3F800904D46019B8AF8006083F80080B7
:10EB080028460BB0BDE8F08FA268A189E3898A4244
:10EB18000B4434BF002501259A42ECD3082305A9EC
:10EB2800E07C8DF8143000F0BBFEE289A368B3FBEB
:10EB3800F2F102FB1133012B4FFA80F8DBD12223CB
:10EB48008DF81430E07CA37C8DF8156005A98DF84C
:10EB5800163000F0A5FE46B2B742CCD12579002D7B
:10EB6800C9D0E07C8DF824B007A900F0A7FEC1E762
:10EB78001646C0E70025C3E77047704770477047DF
:10EB8800002070477047704770470020704700208A
:10EB9800704700207047002070470020704770477A
:10EBA8007047704702207047022070470220704764
:10EBB800704700207047704770470020704700205A
:10EBC800704770477047000010B5054CFC2220467E
:10EBD800002102F007FE0020C4E9000010BD00BFBC
:10EBE800F42400202DE9F04180461546002942D042
:10EBF800244B002403F1010C1A462001103312F8AB
:10EC0800016F002E39D19A42F9D11F4F3B680BB9D9
:10EC1800C7F800C07B680BB1C3F800C03B180022DE
:10EC280001349A6083F80C800D302301AAB238446D
:10EC3800FD50C7F804C002F0C1FDB8F1050F17D0A8
:10EC4800A8F10808B8F1020F8CBF4FF000084FF088
:10EC5800010807EB041400236371D7F8F83084F82F
:10EC6800048001332B44C7F8F8303046BDE8F08102
:10EC78004FF00108EDE70126F7E701340F2CB9D171
:10EC88000226F2E7FB240020F424002010B510B37C
:10EC9800124A1368984204D103681360002304E001
:10ECA8000B4613B119688842FAD15168884208BFE7
:10ECB80053600BB101681960D2F8F8308168013BE4
:10ECC80000245B1A04602146C2F8F830102202F0D2
:10ECD80089FD204610BD0120FCE700BFF424002078
:10ECE800054B1B6813B11A798242FAD1002B0B60CD
:10ECF8000CBF032000207047F424002010B5054BFA
:10ED0800186800B910BD037B04680BB9FFF7BEFF94
:10ED18002046F6E7F424002010B5074B186800B920
:10ED280010BD03790468052B02D0083B022B01D8DB
:10ED3800FFF7ACFF2046F2E7F424002028B1044B8B
:10ED4800D3F8F8300360002070470120704700BFF7
:10ED5800F42400202DE9F04107460E4615463AB343
:10ED680031B3144B1C6800232CB93046FFF7E6FF7B
:10ED78000020BDE8F081A268F91A0132914210D34F
:10ED88002279EA54581C22895FFA80F8611D55FAE5
:10ED980080F002F013FDA368246898445FFA88F3B2
:10EDA800E2E720462468FFF771FF002CF9D1DCE781
:10EDB8000120DEE7F42400200238C0B211289ABFEF
:10EDC800014B185C002070478750010830B50B4B89
:10EDD80093F820200446084672B100211C330578B8
:10EDE800A54208D001319842CDB20CBF0448043086
:10EDF800AA42F4D8002030BD1046FCE7F0250020D8
:10EE0800FC25002010B5084C00232060142204F1D2
:10EE18000C00FF2184F82030C4E9010002F0E2FC74
:10EE2800012384F8213010BDF025002010B50E4ACA
:10EE380092F82010042915D8936804781C70447837
:10EE48005C70C078D87001310020987082F820106A
:10EE580002F11C018B4214BF043302F10C039360CE
:10EE6800012010BD0020FCE7F0250020094B93F895
:10EE7800200068B15A6803F11C018A4200F1FF3092
:10EE880014BF043203F10C0283F820005A600120F9
:10EE9800704700BFF025002010B5074B93F82020DD
:10EEA8000446084632B15968FFF790FF10B10123B4
:10EEB8004470837010BD00BFF025002008B5064BD4
:10EEC80093F820202AB15968FFF780FF08B14078ED
:10EED80008BD0120FCE700BFF025002030B50A4A34
:10EEE80092F82010536882F8210061B191680124DA
:10EEF8001C32DD78587005B99C7093420CBF034BE7
:10EF080004339942F5D130BDF0250020FC250020BE
:10EF180008B5044B5968FFF759FF003818BF01209E
:10EF280008BD00BFF02500202DE9F3410422154E4D
:10EF3800044600210DEB020096F8208002F052FCF6
:10EF48000025EBB2984502D802B0BDE8F08173689D
:10EF5800197821705A7862709F785FB133682046BB
:10EF68009B689847FFF782FF17B901A8FFF75EFF74
:10EF78000135E6E7DB788DF804108DF805208DF86B
:10EF88000730EFE7F0250020014B93F82000704789
:10EF9800F0250020034B93F82000042894BF00209C
:10EFA80001207047F02500201FB50024CDE9024458
:10EFB800C41F8DF800408DF801100C0AADF804202C
:10EFC800090C120C8DF803108DF806208DF8073007
:10EFD80002461B0A012168468DF802408DF8083068
:10EFE80002F05DFA002818BF0F2004B010BD2DE90B
:10EFF800F04188B017460D460F9A064600284DD0B6
:10F0080000240121CDE904448DF810109DF8381032
:10F018008DF81510ADF81630190CCDE900441B0E0B
:10F02800CDE902448DF81930ADF81A20130C120EF0
:10F0380007948DF818108DF81C308DF81D20E3B258
:10F048004FEA0318002D5FFA88F803DC002008B0A7
:10F05800BDE8F081013310218DF81F303A466B4628
:10F068000DEB010002F0B1F90346C8B9102DAC460A
:10F07800A8BF4FF0100CDAB2624503F1010303DBBD
:10F08800103D2DB20134DAE708EB020020326A4461
:10F09800315C12F8202C4A403254ECE70A20D6E7BB
:10F0A8000F20D4E70138032815D8DFE800F002085C
:10F0B8000C100A4B1B681B690B6000207047074B3C
:10F0C8001B685B69F8E7054B1B689B69F4E7034B12
:10F0D8001B68DB69F0E70520704700BF1426002095
:10F0E8002DE9F041C4B00C464A9E17461D4680469D
:10F0F800B8B3B1F5807F36D84FF4887200216846DE
:10F1080002F070FB492300934FF48073ADF804308C
:10F118002B0C8DF80830330CADF80650ADF80A60AA
:10F128008DF80C3022460023414604A82D0E360ED9
:10F138008DF80E308DF809508DF80D608DF80F4060
:10F1480002F03CFB04F110014B9A3B4689B2684639
:10F1580002F025F910B1012818BF0F2044B0BDE80E
:10F16800F0810A20FAE70E20F8E7000010B590B108
:10F178000A4C28220021206002F034FB2368084A48
:10F188001A6000204FF0FF32C3E90302C3E90522E9
:10F19800C3E9072210BD0920FCE700BF14260020A0
:10F1A80000010101024B1B6818600020704700BF76
:10F1B8001426002030B1044B1B68DB680133036060
:10F1C800002070470A2070471426002073B50E46A9
:10F1D800002101911D4633B301A9FFF763FFD0B9A0
:10F1E800019C631C04D0A3B2D31A002B10DDE218D3
:10F1F8000E4B2A601B689B786BB9121B63EB0303E9
:10F20800B24273F10003ACBF01200020C00002E04D
:10F2180003D12C60072002B070BD230C1B0403F53A
:10F2280080331A44E4E70A20F5E700BF14260020DB
:10F2380028B1044B1B681C334362002070470A2026
:10F24800704700BF142600201FB50446F0B1002304
:10F2580003A8039302F07AF90E4ABDF80C3012683D
:10F2680020469380E38200F052FA60B904F1180353
:10F27800009321680123132202F088F840B9204640
:10F2880000F045FA00B1112004B010BD0A20FBE7D8
:10F298000F20F9E714260020F0B5054687B01C4674
:10F2A8003BB32F4E3368DB68834257D894F820204D
:10F2B800002A14BF09220822834205D3204600F001
:10F2C8005AFA70B111200AE0002301900093A36854
:10F2D80094F82810606AFFF78AFE0028EED007B07D
:10F2E800F0BD23792168B4F808C0A768043B9AB236
:10F2F80009B90A20F3E7B2F5807F2DD8ADF80EC022
:10F308008DF817304FEA174C04F12C033F0E8DF897
:10F31800117000932F0C08234FF0490EADF80C0024
:10F328008DF814708DF816002F0E0DEB0300CDF834
:10F3380008E08DF810C0ADF812508DF8157002F085
:10F3480025F808B10F20CAE7204600F014FA002873
:10F35800B8D13368DD60C2E70E20C0E70620BEE7FB
:10F36800142600202DE9FF410A9D80460F461646C7
:10F378001C46002D5AD0002303A910460393FFF71B
:10F3880091FE18B1062004B0BDE8F081039B9C42B1
:10F3980001D80133F6D1284600F05EF9002847D19C
:10F3A800264B1A78424503D01A79424542D10120AA
:10F3B800AA68BA4240D103EB8002EB6A92F8018056
:10F3C8002979CDE900430439927828683B4689B207
:10F3D800FFF786FE0028D6D195F820300194002B3F
:10F3E8004FF00103009314BF4246082295F82810F5
:10F3F800686A3B46FFF7FBFD0028C4D1013E032E97
:10F40800C1D8DFE806F002070B0F0D4B1B681C6123
:10F418001C62B8E70A4B1B685C61F9E7084B1B687C
:10F428009C61F5E7064B1B68DC61ACE70A20AAE79C
:10F438001020A8E70C20A6E70220A4E7B4080020C3
:10F44800142600201FB50A460B2A4FF00001CDE90B
:10F458000011CDE9021107D00C2A13D00A2A0FD0C7
:10F468000B2005B05DF804FB012802D120238DF89C
:10F478000030684602F013F8002818BF0F20F0E7A4
:10F488003023F4E70B21F4E738B5054602F002F81B
:10F49800044678B97DB9094B1B680B219878FFF7AA
:10F4A800D1FF38B90C21FFF7CDFF18B90A21FFF7B2
:10F4B800C9FF00B10F24204638BD00BF1426002024
:10F4C8002DE9F04380468FB00C461746002A6BD0D2
:10F4D800002969D0002529461D2206A8059504F0B3
:10F4E800A3FE8DF81350344D2B680DF114099E8836
:10F4F800CDF804900DF1130302933B7900933B6818
:10F5080032462146404601F0E6FF00284ED13868D1
:10F518003A79494602F052F9384600F04FF8002887
:10F5280046D13C7AFA79BB79240444EA02241C4384
:10F538002B689A6894423DD99C609DF813000B2172
:10F54800FFF780FF034658BB0C21FFF77BFF0346FC
:10F5580030BB0A21FFF776FF034608BB7B7ABA7AED
:10F56800FF7A3F0447EA02271F433A4633462146BB
:10F578000920FFF719FD034690B933463A4621465C
:10F588000820FFF711FD034650B92A689DF81310AB
:10F5980091700021D1604FF0FF31C2E904119161EF
:10F5A80018460FB0BDE8F0830A23F9E70F23F7E701
:10F5B8001023F5E70323F3E71426002010B50446CB
:10F5C800002845D00168002942D011F8013B437159
:10F5D8000322063002F0F2F82046032250F8091BF5
:10F5E800043102F0EBF82168CB79E3600A7A43EA48
:10F5F8000223E3604A7A43EA0243E3608A7A43EAF1
:10F608000263E360CB7A23740B7B63742379212B29
:10F618001AD110220D3104F1120002F0CFF81D2288
:10F628002168501C8B5C6362085C43EA0023901CD1
:10F638006362085C033243EA004363628A5C43EA1C
:10F6480002636362002010BD112B03DC0D22E7E783
:10F658000220F8E70120F6E710B50446002854D048
:10F668000168002951D00B7843714B7883608A7800
:10F6780043EA02238360CA7843EA024383600A7933
:10F6880043EA026383604B7903738B79C381CA7938
:10F6980043EA0223027BC38102F00F0208311030D3
:10F6A80002F08CF8237B002203F00F0384F820205B
:10F6B80084F82820227903F10800111A04290DDDA5
:10F6C80021680933043AD21A085C84F82000D2B2BF
:10F6D800606A84F82820194402F070F823792268B7
:10F6E8001A44002012F8043CE36212F8031C43EAAF
:10F6F8000123E36212F8021C43EA0143E36212F8B1
:10F70800012C43EA0263E36210BD0220FCE710B556
:10F71800044660B3036853B30279162A29D942799B
:10F728001A700146082251F8060B013002F050F811
:10F738002146082251F80E0B093002F049F82368D7
:10F74800E28A5A74E38A22681B0A93742368A269BE
:10F75800DA74A36922681B0A13752368628B5A75C9
:10F768002368E27E9A7517232371002010BD0120BB
:10F77800FCE70220FAE738B50446002863D00168A0
:10F78800002960D0037B90F8282003F00F03002A9B
:10F7980057D10833207904321344984255D36379FA
:10F7A8000B702368A2685A70A36822681B0A9370BA
:10F7B80023686289DA702368E27A1A712368227BE7
:10F7C8005A712368E2899A71E38922681B0A2146E3
:10F7D800D371227B51F8100B02F00F02083001F0B0
:10F7E800EDFF237B94F8282003F00F0303F10805AD
:10F7F8002AB1226894F82010515503F109052068B0
:10F8080094F82820616A284401F0D8FF94F8283039
:10F818002268E16A2B44D1545A1CE16A206892B2EA
:10F82800090A81549A1C2168E08D92B28854DA1C26
:10F83800216894F82F0092B2043388542371002071
:10F8480038BD0933A6E70120FAE70220F8E70000EF
:10F85800024B1A8810431880704700BF18260020F2
:10F8680008B5074B1B883BB1FEF728FA00280CBFE8
:10F8780000206FF0020008BD6FF00100FBE700BF39
:10F888001826002010B5034B00241C80FEF70CFA44
:10F89800204610BD18260020B0FA80F040097047B5
:10F8A80082B018B9084602B000F0D0B8002002B003
:10F8B800704710B9084600F083B9704710B9084678
:10F8C80000F09AB970470346084611460BB900F094
:10F8D800E7B90020704710B9084600F045BD7047E9
:10F8E80010B9084600F008BA0020704710B4044662
:10F8F800084611461A46019B14B910BC00F01ABA02
:10F9080010BC70470346084611460BB900F044BACC
:10F918000020704710B40446084611461A4614B928
:10F9280010BC00F0B1BA002010BC704730B40546D6
:10F93800084611461A46DDE902341DB9029430BC66
:10F9480000F02EBB002030BC704710B9084600F00C
:10F95800DFBB0020704710B9084600F043BD002007
:10F96800704710B9084600F0EEBB0020704710B988
:10F97800084600F0EBBB00207047034608461146D6
:10F988000BB900F005BC0020704710B404460846C7
:10F9980011461A46019B14B910BC00F0FBBB0920A4
:10F9A80010BC704710B9084600F03CBD704710B451
:10F9B8000446084611461A4614B910BC00F05CBD4E
:10F9C800C8B210BC7047000000487047030001012E
:10F9D800064B10B51B6A0446984730B10448054BDE
:10F9E800204498428CBF0020012010BDFC5601081D
:10F9F800403576C9405DC600F0B5114B85B00C4660
:10FA080010491F56054601F045F80F4BE4B25E6AEF
:10FA1800072D4FF00103CDE9024301460AD1052223
:10FA28000023CDE900234FF47A727A431846B04791
:10FA380005B0F0BD08220020CDE900203A46F5E7E0
:10FA4800C35001089C500108FC5601081FB500234B
:10FA580000930378013B382B00F28580DFE803F040
:10FA68001D2383838320838383834042444B8353B2
:10FA780056595C5F6265836D206F74797B7E7E80EA
:10FA88008725838383838383838383838383838992
:10FA98008B908383899083929600C378002B62D0E1
:10FAA800022300935FE08378F8E743788DF8043009
:10FAB80007238DF805308378003B18BF01235B00CE
:10FAC8008DF8063010238DF80730334B1B6801A8DA
:10FAD80003F59062CDE9022300F0BCFF009042E0FC
:10FAE8004023DEE72023DCE7827890F9013042B931
:10FAF8002A4AD35CD5E7827890F901300AB9284AB6
:10FB0800F7E7284AF5E740F6B833CAE74FF47A73BF
:10FB1800C7E74FF4FA63C4E741F28833C1E741F21B
:10FB28007073BEE74FF48043BBE71F484FF47A7108
:10FB380001F028FE00F5FA60D0E71C4BB1E7164B40
:10FB48001B6803F59063ACE7134B1B6803F28C4307
:10FB5800A7E71023A5E7104B1B68A2E70123A0E73E
:10FB68004FF083430093009805B05DF804FB104BF9
:10FB7800F8E7104B95E740F21123ADF80030F2E7B3
:10FB880003238EE790F901300B4AB2E70B4990F94D
:10FB9800010000F07FFFA1E720260020D3500108D4
:10FBA800E3500108DB50010818FCFFFF00EA0637A4
:10FBB8009A99094040F70937C35001089C50010839
:10FBC80037B50B4B02781B680C2101FB02335B7ABB
:10FBD80003EB4304074B1D6803690093C36842782D
:10FBE800816805EBC40000F0D5FC03B030BD00BF50
:10FBF800202600201C26002030B587B0027A642316
:10FC0800ADF80030012A4FF00003CDE90133CDE90A
:10FC1800033301468DF802308DF8143027D0022ABC
:10FC28002ED012BB006800B34B68F3B1194A1A4CC6
:10FC3800106069461822236001F0C0FD174B246844
:10FC480093E807000C3384E8070093E8070004F101
:10FC58000C05032385E80700A4F88C34012204F27C
:10FC68008C4104F5906000F086FC07B030BD0A496D
:10FC780008684360036100F28C4100F59060F2E788
:10FC8800054B1B68B3F88024B3F88C140A43A3F817
:10FC98008024EAE71C26002020260020EC430108E7
:10FCA80008B503460A2924D8DFE801F006232323F0
:10FCB800230B161B23212100BDE808400068FFF72D
:10FCC80087BE90F900009978072271B900F013FCFB
:10FCD800003818BF012008BD052293F90000002153
:10FCE800F4E790F900005978EEE70221EEE70722E1
:10FCF800F3E70020EFE7000010B504791CB1012CF0
:10FD08000BD0002010BD0A4B01681B68012203F5C7
:10FD1800906000F030FC0120F4E7054B01681B6897
:10FD2800224603F28C4000F026FC2046EAE700BF9A
:10FD380020260020F7B50728144D1C46A8BF072029
:10FD480058700E462946174600F0A4FE94F9013073
:10FD5800A070072B13D1322000F09CFD0C4BDB6DFB
:10FD68000546984704F10C020834034601920094B2
:10FD78003A463146284600F092FD03B0F0BD054AE8
:10FD880055F82310D05C00F07DFDE7E79C50010892
:10FD9800FC560108C35001082DE9F04F344F90F983
:10FDA80001607B68D0F804908BB004468846984779
:10FDB8000546002859D1E37C73B92E4A2378126886
:10FDC80003EB4303990002EB8303D3F80490B9F1E2
:10FDD800000F01D152F80190274B484613F906B09D
:10FDE800FB689847A37CD7F818A022890993072EA7
:10FDF80028D100230121CDE90223204A0693CDE929
:10FE08000431CDE907330521CDE900214FF47A7299
:10FE180002FB0BF24CF250311846D047637C13B307
:10FE2800174B995D7B6D0D31C9B228469847E07C28
:10FE38003246494600F040FE88F8006001200BB0C9
:10FE4800BDE8F08F002101250823CDE90013CDE995
:10FE58000715CDE90511CDE903110292A1782B46CA
:10FE68005A462846D9E7074BDBE70020E7E700BFFB
:10FE7800FC56010820260020C350010885450100D2
:10FE8800E3500108D35001082DE9F04F8DB090F9E7
:10FE98000130DFF8F8A0DFF8F890CDE90A123D4A02
:10FEA800017812F903B0DAF800203B4B0C2505FB6A
:10FEB80001221B68527A182101FB0233044693F988
:10FEC800021090F9020000F0E0FD3449064694F96A
:10FED800010000F0DFFDA26861688046304600F04E
:10FEE80006FD2178DAF80020D9F80C306943074676
:10FEF80050589847D9F81C309C4694F90130002591
:10FF0800072B4FF47A63CDE90753CDE905552DD179
:10FF18000123CDE903530523CDE901534FF47A7347
:10FF280003FB0BF300933946434646F2A8122846D2
:10FF38006746B8472378DAF800200C214B4394F938
:10FF48000110D05800F0DAFDA18994F90100FFF7FB
:10FF580053FD0B9B217B1860D9F8543028469847ED
:10FF68000A9B01201E700DB0BDE8F08F0120082308
:10FF7800CDE90350CDE901032A46CDF800B0654626
:10FF880043463946A84701200546D3E720260020E6
:10FF9800FC560108C35001081C2600209C5001088B
:10FFA8002DE9F04F8FB0002405468A4691469846C1
:10FFB8000494ADF81440ADF8024007264FF0010B49
:10FFC8002B7AA34206D9686804A9204400F0F4FB00
:10FFD80000285DD102238DF8083002A86B7A8DF8CD
:10FFE8000A30FFF733FDAB7A8DF81D309DF81130DC
:08FFF8008DF81E309DF8123057
:020000040801F1
:100000008DF81F309DF810308DF82030EB7A8DF888
:1000100021302B7B8DF822306B7B8DF82330102321
:100020008DF81C608DF824303A4E8DF82C000DF1BF
:1000300002030A93072332688DF82D30ADF834306F
:100040002B680C9206930DF1120204AB0DF1110115
:1000500006A800F0CFFB072805460BD130680C221C
:10006000002100F5906001F0C1FB3368BDF802206B
:10007000A3F880249DF811308AF800309DF81230E2
:1000800089F800309DF8103088F80030189B284619
:100090001C700FB0BDE8F08F9DF81330BDF81470E0
:1000A000ADF802702044C4B2F3B917B3194A002066
:1000B0001168072602464FF00C0C062B1BD10CFBD7
:1000C00000FE51F80EE0BEF1000F04D00BFA00F272
:1000D0003A4397B2012201301028EED1002A3FF4B2
:1000E00073AFADF802706FE75A1E042A01D9062BD0
:1000F000DCD0062668E747FA00FE1EF0010FEAD0C2
:100100000CFB00FE51F80EE0BEF1000F08BF062602
:10011000E1E700BF2026002038B505464068FFF71C
:100120005BFC0722841D002195F90000E4B200F079
:10013000E6F908B904F0FD0495F901000722002151
:1001400000F0DDF908B904F0FB04204638BD0020BA
:100150007047000010B503780F2B044618D840688C
:10016000FFF73AFC22780B4902EB42020968831C34
:1001700001EB820051F82220DBB21AB903F0FD0333
:1001800058B210BD032B06BF626842600223F7E736
:100190000020F6E720260020022070472DE9F041DC
:1001A0003A4D0446286896B00E46904600211F46F8
:1001B0000122032300F59060CDE90411CDE9061179
:1001C0008DF80C108DF80D10ADF80E3000F0B9F967
:1001D00030B92A68B2F8803443F00303A2F88034BF
:1001E0002A68637A8DF8203002F59061CDE9091212
:1001F000274A94F9083012680B921022ADF830208B
:100200000DF10E020D9222680E9262680F92D4E9EF
:100210000301A27A8DF8402001228DF8412011AA15
:1002200082E80300227DE18A8DF8213018468DF89E
:100230004C20FFF7E5FB08AB15930DF10D0314906F
:100240000093CDF8048003AB04AA39460EA800F051
:10025000C1FB044678B99DF80C10013901F096FAFB
:1002600000F158030DEB030010F8483C33702046B2
:1002700016B0BDE8F0810C2801BF2A68B2F88034BE
:1002800043F00303A2F88034F1E700BF20260020EA
:100290001C260020F8B50679012E054601D8062057
:1002A000F8BD0F2E2BD80368187A40F303000722FD
:1002B000002140B200F023F92B680446187A40F37D
:1002C00003100722002140B200F019F9A8B1B4FAD6
:1002D00084F4640929680B7A086843F3030243F342
:1002E000031352B25BB29A42C8BF0124FFF774FBFA
:1002F00048B9002CD3D10420D2E70124EAE7032037
:10030000CEE70520CCE7002CFBD10C4F29683B68D9
:1003100006EB460003EB80000C2201F053FA3A682A
:100320000C2303FB062320465C72B2F880140123E1
:10033000B3400B43A2F88034B2E700BF2026002070
:1003400010B4017801290ED9084B18680C234B43CF
:10035000C4180022C250C4E9012200F5906010BC0C
:10036000102200F0D5B8002010BC704720260020D5
:100370002DE9F04186B050238DF814300379102B0D
:10038000074630D10368DD7B6DBB0224A846642696
:10039000062C14D83A68535D03932A44517843EAF3
:1003A00001230393927843EA02437343CDE9033870
:1003B00063B968468DF80040FFF7C2FF0DE0CDF845
:1003C0000C808DF81480CDF81080F2E703AB01A803
:1003D00001938DF80840FFF75DFF0134E4B2102C63
:1003E00005F10305D4D106B0BDE8F0811FB5026860
:1003F0000379116851B901A88DF80430FFF7A0FF07
:1004000078B9002040B205B05DF804FB02A8029262
:100410008DF80C30FFF73EFF0628F2D8024B185C2F
:10042000F0E70320EEE700BFBC50010870B5114EA5
:1004300001783268104B0C2505FB01221B68527AAB
:10044000182101FB0233044693F9021090F90200CF
:1004500000F01FFB2378326861686B43D558A268AF
:1004600000F049FA054BA289DB6B01462846BDE83E
:1004700070401847202600201C260020FC5601084A
:10048000074B9B56C91A431E5842584140008842A8
:10049000B8BF08460528A8BF0520C0B2704700BFF6
:1004A000CB500108F0B59A42069D03DB9DF914304C
:1004B0009A4220DD0020F0BD03EB430331F814C065
:1004C00005EB830300264CFA06F7FF0707D51F7AD2
:1004D00007F00F0E724502DBB2EB171F0DDD013680
:1004E000102E03F10C03EED10134E4B22301DBB290
:1004F0009842E1D8DEE70024F8E70120DBE78842F4
:1005000004DB9042CCBF00200120704700207047E0
:1005100010B51409B4EB111F03464FEA11100ED3A6
:1005200091420CD202B201F00F0133F812400120C7
:1005300000FA01F124EA010123F8121010BD002095
:10054000FCE7F0B528B100EB4105012700209142FE
:1005500000D3F0BD002435F802CB234607FA04F699
:1005600036EA0C0608BF013304F1010408BFDBB210
:10057000102CF3D118440131C0B2C9B2E7E710B56D
:1005800000B149B910BD31F8134020F813400133D0
:10059000DCB2A242F7D8F5E70023F9E782B030B524
:1005A000048804936AB9B3F5616F18D349F6AF258F
:1005B00042F21072AB4298BF4FF47A72944238BF45
:1005C0001446012C38BF01246143BDE83040C368A4
:1005D0008B428CBF5B1A0023C36002B07047642259
:1005E000ECE700002DE9F04F91B01546DDF86C8086
:1005F00004939DF8683009930C46064603F0C2FB4D
:10060000684ADFF8A4B10590A8F5F633303BB3FB98
:10061000F2F3534303F5F63203F5A83303F5C07341
:100620000393182313FB05433032069208930025E9
:100630004FF0FF3A089BA34207D1002D14BF50464C
:100640004FF0FF3011B0BDE8F08FBDF97030ADF85C
:100650002C300B99CDF86C804046CDF8288003F003
:1006600021FBB4F800906EB9B8F5616F5BD349F621
:10067000AF2242F21073904598BF4FF47A739945B8
:1006800038BF99464B46012B38BF01230793002EF4
:1006900052D1B9F1640F48D1A0605F46A1680EA89D
:1006A00003F022FB0F9B0093DDE90A120E9B0CA8BE
:1006B00003F079FA049B0C9A0BB9099B2BB12369BF
:1006C000BB4202D1394B9A420DD9394BE76098456C
:1006D00009D90023ADF83430069B0D990C931846C8
:1006E00003F0E0FAA060606800B9E760276126B116
:1006F00003F052FBE3680344E360D4E9033293421E
:10070000059B1D996360079B88BFE2604B43E168CE
:10071000994202D20498A8B9A6B101231D442375B9
:10072000EDB2183486E76423A9E7B9F57A7F0ABFEA
:10073000204F214FA060B1E7049B0BB9C4F80CB067
:100740005F46D0E700209342207506D85B1A9A4591
:1007500005F1010528BF9A46EDB2002EE1D1B9F1AD
:10076000640F164AADF8346019D049F6B023B9F5D4
:100770007A7F18BF1346904584BF039A9B180C9349
:100780001C9B00930CAF97E806001B9B384603F0B8
:100790000AFA97E8030003F085FA8246C1E74FF4AE
:1007A0006163E8E78051010040771B007F51010041
:1007B0002FEC010080A81201002E930230EC010002
:1007C0000378032B14D1437803F00F021B098A70BE
:1007D0004B7083788B80C27843EA02238B80037945
:1007E000C3F3021203F00F03CA700B7005207047A9
:1007F000002070472DE9F34798464379057990F931
:1008000007609146044690F906208A4683B190F924
:10081000087075B30F2A12D194F909200F2E1ED13A
:1008200094F90A60072D24D1002F08BF012720E08A
:1008300090F90B7090F9092090F90A60E9E7A36933
:10084000019394F915300093216994F91430207BB9
:10085000FFF728FE0028E1D105F0FD05DEE794F959
:100860001D30B3420FDC94F91C30B342DADA05F0E4
:10087000FB0528468AF8002089F8006088F8007097
:1008800002B0BDE8F0871E46CCE70000024B03FA39
:1008900000F0B0FBF1F0704740420F004FF4FA5304
:1008A000B3FBF0F0704730B54FF47A750C1F6A4314
:1008B00000FB042252001EBF00F1FF341219B2FBEC
:1008C000F0F2914238BF1146039A1160820048430A
:1008D0001CBF013040084FF47A71121A01FB132338
:1008E000002BCABF03F2E73393FBF1F1B3FBF1F145
:1008F000049B196030BD38B5400014460D46F1F731
:1009000089F801462846F0F7D3FF2146F0F7D0FFDB
:10091000F0F7C2FE03F0D8FCF0F79EFF40B238BDFE
:100920002DE9F74F019300231F469C461C01058AC1
:100930005FFA84FE04F0F004A54206D8019B82F819
:1009400000C01F7003B0BDE8F08F0EEB4E054FEAFC
:100950004309AD000024466836F809602641F607D1
:1009600027D5866806EB050A765916B3067836B998
:10097000466926B136F809602641F60719D59AF876
:10098000086090F901B046F303084FFA88F8D8459B
:100990000FDC46F3031676B25E450ADB9AF809606F
:1009A00006EB4608C66806EBC806367D4EB9013729
:1009B000FFB20134102C05F10C05CCD10133DBB2B0
:1009C000B4E70CF101060EEB040801F80C805FFAA5
:1009D00086FCEEE72DE9FF4704464068DDE90C6739
:1009E0001D468A46914603F0D7F923681B1A3B60DF
:1009F0004FF000080123337085F80080636813B15D
:100A00002368834224D8CAF80080D4F81CC0A369A4
:100A10009CF800E00393D4E9030101AB83E80300F1
:100A2000237D0093DCF80C10237A627A7046FFF77E
:100A3000D9FD334638602A46E0694946FFF770FF22
:100A40002B782BB1C7F80080002004B0BDE8F087F8
:100A50003378002B14BF0B200C20F6E737B590F944
:100A6000002090F90250954204460FD0013A52B24C
:100A700095420BD0A368019394F90130009361680B
:100A8000E0782B46FFF70EFD0028EFD0104603B0AC
:100A900030BD8842B8BF08467047000051F82000BA
:100AA000054B984205D0054BC31A584258414000A7
:100AB00070470120704700BF90D0030020A10700BD
:100AC00005281FB50ED80C4B53F820300093CDE904
:100AD00001120A4B01220021022002F069FE05B03A
:100AE0005DF804FBCDE90012054B01220021022034
:100AF00002F05EFEF3E700BF54510108EB5001081D
:100B00000A51010807B5054BCDE90001012200217A
:100B1000022002F04DFE03B05DF804FB26510108EF
:100B200010B5102204460021F13000F05FFE0021D4
:100B3000C4F814112046F022BDE8104000F056BE63
:100B400002460846102100F0A5B92DE9F0430446FD
:100B5000D0F8140185B00E46154604F2011988B389
:100B6000C0F110089045474628BF1746BAB248441E
:100B700000F028FED4F814313B440F2BC4F8143194
:100B80002DD9A8452BD204F1F00304F5807113F898
:100B9000012F187C8B4282EA00021A70F7D104F10F
:100BA000F10810224146684600F00CFE22466946D4
:100BB000684600F0E9F910226946404600F002FE5E
:100BC0003E44ED1B04F5807804F1F107102D09D89F
:100BD000AAB23146484600F0F5FDC4F8145105B0FC
:100BE000BDE8F08304F1F003711E13F8012F11F832
:100BF000010F434582EA00021A70F6D110223946ED
:100C0000684600F0DFFD22466946684600F0BCF900
:100C100010226946384600F0D5FD1036103DD5E764
:100C2000F0B589B00C46102200210546684600F058
:100C3000DDFD22466946684600F0A6F99DF90030C0
:100C4000002B6A464FF0000143DA137812F8010FC7
:100C500001315B0043EAD0130F2902F8013CF4D1C3
:100C60009DF80F305B0083F08703D4F81401DBB2EA
:100C700010288DF80F303BD104F58073694604F5D8
:100C8000887013F8016F11F8012B984282EA06026E
:100C90001A70F6D104F1F00304F5807113F8012FF6
:100CA000187C8B4282EA00021A70F7D110220DEBF9
:100CB000020004F1F10100F085FD2246294604A856
:100CC00000F062F910220021684600F08FFD09B0A3
:100CD000F0BD137812F8010F01315B0043EAD01325
:100CE0000F2902F8013CF4D19DF80F305B00BCE7FE
:100CF0009DF90030002B6A464FF0000137DA137877
:100D000012F8016F01315B0043EAD6130F2902F894
:100D1000013CF4D19DF80F305B0083F08703471C42
:100D2000DBB28DF80F30102F04EB0003C0F10F067B
:100D30004FF0800288BF002600F5817083F8012102
:100D40000021324620443E4403F072FAC4F8146194
:100D500004F58073694604F5887013F8016F11F883
:100D6000012B984282EA06021A70F6D192E71378B4
:100D700012F8016F01315B0043EAD6130F2902F824
:100D8000013CF4D19DF80F305B00C8E70A78037886
:100D9000534003704A784378534043708A7883788D
:100DA00053408370CA78C3785340C3700A7903797B
:100DB000534003714A794379534043718A79837967
:100DC00053408371CA79C3795340C3710A7A037A55
:100DD000534003724A7A437A534043728A7A837A41
:100DE00053408372CA7AC37A5340C3720A7B037B2F
:100DF000534003734A7B437B534043738A7B837B1B
:100E000053408373CA7BC37B5340C373704710B591
:100E10000B7814786340037054784B7863404370C8
:100E200094788B7863408370D478CB786340C370B8
:100E300014790B796340037154794B7963404371A2
:100E400094798B7963408371D479CB796340C37192
:100E5000147A0B7A63400372547A4B7A634043727C
:100E60008B7A947A63408372D47ACB7A6340C3726C
:100E7000147B0B7B63400373547B4B7B6340437356
:100E8000947B8B7B63408373CB7BD27B5340C37358
:100E900010BD0000A1F11003DBB2102B2DE9F047CB
:100EA00004D8374C24FA03F3DB0705D4002382F877
:100EB000F030FF20BDE8F087531E4418A0424ED109
:100EC00001F11C039B005FFA83F9C3F30313013B99
:100ED0002C4D82F8F03001240B46D618B3FBF1F00C
:100EE00001FB103010F0FF0016F804AC16F803EC0C
:100EF00016F802CC16F8017C36D115F80E8015F8DC
:100F00000CE015F807C015F80A70E00900EB400086
:100F100084EA080800EBC0006400C0B2E4B24440B8
:100F2000C246581AC0B212F800808AEA080A02F8CB
:100F300003A01044043390F801808EEA080E86F86E
:100F400001E090F802E08CEA0E0C86F802C0C0784E
:100F5000DBB247409945F770BFD80020AAE710F8E8
:100F6000015B03F8015FA9E71829DAD9102801BF4E
:100F700015F80AA015F80EE015F80CC0EF5DD0E7E3
:100F8000010101006C5301082DE9F04FA3B092F864
:100F9000F0301D911B920193002B00F0538101460C
:100FA0001EA8FFF734FF1B9BA74CA84DA84E10337B
:100FB0000293002303939DF87C0004909DF8860023
:100FC0000590205C06909DF87B000790205C0890BF
:100FD00004989DF881C0205C099014F80C000A90D8
:100FE0009DF880000B909DF885009DF878809DF815
:100FF0007DE09DF882A09DF887900C909DF87A0086
:10100000029B1C9314F80A2014F8093014F80810F5
:1010100014F80E700D90205C0E909DF87F000F90DC
:10102000205C10900B98205C11900C98205C129022
:101030009DF8840013909DF8790014909DF87E002F
:101040001590205C16909DF883001790205C1890F6
:101050001398205C19901498205C1A900398013022
:1010600003900298DDF804B0103002909DF80C0057
:10107000834536D88DF878108DF87A2009990E9A24
:101080008DF87C108DF882201199069A8DF88010C9
:101090008DF87E201999169A8DF884108DF8862087
:1010A0000A99189A8DF87D108DF887201299109A58
:1010B0008DF87B301B9B8DF881108DF883201A9959
:1010C000089A1D988DF885108DF87F201EA903EBD6
:1010D0000B128DF87970FFF79AFE002023B0BDE85F
:1010E000F08F15F808B082EA03008BEA000016F8CA
:1010F0000EB080EA0B008DF8780015F80E004B401A
:10110000434016F80A0043408DF8793081EA07031E
:1011100015F80A10594016F80930594016F80830E9
:101120008DF87A107A40534015F8092053408DF815
:101130007B30089A069B5340049AAA5C534016F8E9
:101140000C2053408DF87C30DDE908325A4015F808
:101150000C305340059AB25C53408DF87D30DDE988
:1011600009325A40059BEB5C5340079AB25C5340EE
:101170008DF87E30069B0A9A5340049AB25C5A401E
:10118000079BEB5C5A408DF87F200E9B109A5340D2
:101190000B9AAA5C53400C9AB25C53408DF8803095
:1011A000DDE910325A400C9BEB5C53400D9AB25C67
:1011B00053408DF88130DDE911325A400D9BEB5CD4
:1011C00053400F9AB25C53408DF88230129A0E9BB6
:1011D00053400B9AB25C5A400F9BEB5C1C995A40EF
:1011E0008DF88320169B189A5340139AAA5C53409B
:1011F000149AB25C53408DF88430DDE918325A40BD
:10120000149BEB5C5340159AB25C53408DF88530CB
:10121000DDE919325A40159BEB5C5340179AB25CDA
:1012200053408DF886301A9A169B5340139AB25C3D
:101230005340179AAA5C1EA853408DF88730FFF7D9
:10124000A5FDB8E6FF2049E76C5301086C51010881
:101250006C52010808B538B1044A05491060D8221B
:1012600000F0B0FA002008BD0220FCE72426002090
:101270009C5801080A4B1A6870B5002302F1180542
:1012800003EB03142E5D864204D1183422440A6015
:10129000002070BD01330B2BF2D10320F9E700BF12
:1012A000242600202DE9F041CCB00646DDF8488127
:1012B00017461C460D4631B3B8F1000F23D006A8DF
:1012C000FFF72EFC204601A9FFF7D4FF0446B0B972
:1012D000019906A80131FFF733FC26B110223146EF
:1012E00006A8FFF732FC3A46294606A8FFF72DFC70
:1012F00006A902A8FFF794FC029BC8F8003020461C
:101300004CB0BDE8F0810224F9E7000030B595B09B
:1013100013A90446FFF7AEFF002830D11B490C2368
:1013200003FB00F2555CA5422BD1139B187C109057
:10133000D87B0F90987B0E90587B0D90187B0C906B
:10134000D87A0B90987A0A90587A0990187A08906F
:10135000D879079098790690587905901879049073
:10136000D8780390987802900A445B780193936848
:1013700000930022064B1146022002F019FA15B024
:1013800030BD01300B28CBD1F9E700BFE45501088F
:101390006C5401080B2B10B402D810BCFFF782BFAD
:1013A000032010BC704730B50D4685B01446014689
:1013B00068B103AA002000922A460390FFF772FF4B
:1013C00018B90398001B18BF012005B030BD0220DA
:1013D000FBE72DE9F0430D46BFB014469946804621
:1013E00020B31BB311F00F0122D1F02201A800F0AD
:1013F000FDF920466946FFF73DFF044648B90098CD
:1014000001AA10210130FFF745FD2E46AF1BFFB2A8
:101410001EB920463FB0BDE8F08301AA09EB0701E1
:1014200008EB0700FFF7B0FD103EEFE70224F0E7FE
:101430000524EEE7F0B5184E3468024685B008463C
:10144000002304F1180103EB03154F5D97421ED1F1
:101450000D2A05F1190513D10023CDE90033CDE99B
:1014600002330C2210216B46FFF7B3FF04463068AD
:1014700010226946284400F0A5F9204605B0F0BDC9
:1014800001461022601900F09DF90024F5E70133B0
:101490000B2BD8D10324F0E72426002009B1FFF755
:1014A000C9BF022070471FB51446A0B10C2A01D154
:1014B0000B2912D10023CDE90033CDE902330A46CE
:1014C0006B461021FFF785FF18B969462046FFF7E4
:1014D000B1FF04B010BD0220FBE70320F9E7F8B527
:1014E0001E46DDE907479DF818505BB354B34FB370
:1014F000212D29D819462A46204600F063F90122F9
:10150000631C691EB018FFF764FFF8B9E37ADB09C2
:101510003B70EBB96319204613F8012C13F8021C39
:10152000120642EA014213F8041C0A4313F8031C92
:10153000012342EA0122291FFFF735FF003818BFB7
:101540000120F8BD0220FCE70520FAE70720F8E7B4
:101550000420F6E710B5044628B1044B5B699847B0
:101560002060002010BD0220FCE700BFFC560108EF
:1015700008B5014630B1044B0822186800F022F982
:10158000002008BD0220FCE72426002008B530B169
:10159000044B0822196800F015F9002008BD02204C
:1015A000FCE700BF242600207FB5124E002304462E
:1015B00002A801930D46FFF7E9FF33685B690193C9
:1015C0006CB102AA082312F8011B41B9013B13F0C8
:1015D000FF03F8D102A8A04702A8FFF7C9FF35B161
:1015E000019B23B901A8A8473368019A5A610020DA
:1015F00004B070BD2426002008B5014638B1054B63
:1016000018680822104400F0DDF8002008BD022010
:10161000FCE700BF2426002008B538B1044B196848
:101620000822114400F0CEF8002008BD0220FCE79B
:1016300024260020034B1B6802280CBF1961596146
:10164000002070472426002041B1054B1B6802286A
:101650000CBF1B695B690B6000207047022070475C
:101660002426002030B58FB0002405460CA809942C
:10167000FFF78CFF9DF8373007939DF836300693BF
:101680009DF8353005939DF8343004939DF8333040
:1016900003939DF8323002939DF8313001939DF809
:1016A00030300093224621461E4B022002F080F883
:1016B0000AA8FFF7B1FF9DF82F3007939DF82E3051
:1016C00006939DF82D3005939DF82C3004939DF8DA
:1016D0002B3003939DF82A3002939DF82930019313
:1016E0009DF82830009322460F4B2146022002F03D
:1016F0005FF809A92846FFF7A7FF9DF82430039358
:101700009DF8253002939DF8263001939DF82730EF
:1017100000932246054B2146022002F049F80FB003
:1017200030BD00BFC85401080655010844550108E2
:1017300008B50020FFF7EAFD0120FFF7E7FD0920CB
:10174000FFF7E4FD0820FFF7E1FD0020FFF78AFF27
:10175000002008BD10B504460B20FFF7D7FD0C2074
:10176000FFF7D4FD0920FFF7D1FD0820FFF7CEFDDC
:101770000A20FFF7CBFD2046FFF774FF002010BDC5
:10178000014B1860704700BFBC0800200B4A30B501
:1017900014680B4D43F2390305FB04331360091A37
:1017A0006FF00042B3FBF2F2C2EBC27201319B1A3E
:1017B00093FBF1F201FB1233184430BDBC0800204A
:1017C0006D4EC64101380A44914200D1704711F86C
:1017D000013B00F8013FF7E710440A44914200D171
:1017E000704711F8013B00F8013DF7E702F020BD1A
:1017F00030B530B10A4D01444FF0FF33814201D181
:10180000D84330BD10F8012B5340082243F30004A5
:10181000013A2C4092B284EA5303002AF6D1EDE754
:101820002083B8ED01207047054B4FF400529A62B7
:10183000044B1B6813B15B6803B11847704700BFC6
:101840000004004828270020054B4FF480529A627C
:10185000044B1B6813B1DB6803B11847704700BF26
:10186000000400482827002001207047012070470D
:1018700001F048B901F036B910B501F019FE0E219A
:10188000044640F61F1001F02DF92046012101F019
:10189000F9FDBDE8104001F0D7BA000070B50C4E5C
:1018A00001EB40030D46B3654FF6FF71002304467C
:1018B0001A46084601F05EFB96F85600002101F03A
:1018C000E1FD29462046BDE8704001F095BA00BF11
:1018D0004427002010B5044601F0AAFE01281CD1BF
:1018E00001F0AEFE34B11248214602F017FB104859
:1018F00002F0DAFA0F4C104B00214FF48052A16530
:101900009A6194F8560001F0BDFD63786BB16FF0F9
:101910007F40BDE8104001F053BA002340F262213D
:101920001A46084601F026FBDCE7A0688001F0E7D4
:101930002C2700204427002000040048002001F04C
:10194000BFB9000008B501F0C7F80438C0B20328D9
:1019500096BF024B0020185C08BD00BFF856010876
:1019600008B501F0BAFD033008BD01F049B901F036
:1019700009B908B501F000FD00B208BD38B50D4643
:10198000144601F05DFB284601F092FD0E2105464C
:1019900040F61F1001F0A6F828460121074D01F07E
:1019A00071FD01F051FA4FF47A716143284602F05B
:1019B000B5FA2846BDE8384002F076BAA0270020E4
:1019C00001F03EBB08B5084B002193F8560001F02A
:1019D00059FD00234FF4C0711A46084601F0CAFAB7
:1019E000BDE8084001F024BA4427002010B50446A1
:1019F00001F01EFE01281CD101F022FE34B1124874
:101A0000214602F08BFA104802F04EFA0F4C104BB0
:101A100000214FF48052A1659A6194F8560001F0BC
:101A200031FD63786BB16FF07F40BDE8104001F08D
:101A30007DB9002340F262211A46084601F09AFA65
:101A4000DCE7A0688001F0E72C2700204427002075
:101A50000004004808B54FF0040001F017F9BDE894
:101A600008400220F1F756B808B500231A46194677
:101A7000184601F07FFABDE8084001F06DB900009A
:101A80001D4B73B51D4D186000241D486C70C5E9D1
:101A90000144AC6501F098FAAC8101F003FA2146EB
:101AA000204601F04BFC21460422012001F0FCFA03
:101AB000144E154D4FF6FF7123462246084601F09D
:101AC00059FAFFF7C7FF2246104B00944FF0FF3141
:101AD000304602F03DF90E4B009422464FF0FF31A4
:101AE000284602F035F9304602F090F9284602B057
:101AF000BDE8704002F08AB9282700204427002062
:101B0000C92A0108A02700202C2700202918010835
:101B1000491801080128084805D1084BC1771970F8
:101B20000E3001F0A7BB437D012B03D1034B817520
:101B30001970F5E7704700BF44270020C008002057
:101B40000D4B10B5044618735873012000F016F8B9
:101B50005CB134214FF4E86000F0C4FF4421BDE8DB
:101B6000104040F2417000F0BDBF14214FF4E86016
:101B700000F0B8FF2421F2E74427002038B5114CCB
:101B80000546207001F061FD052D04D8DFE805F061
:101B9000090B03171709032001F070FA0023637380
:101BA00038BD0020F8E7012001F068FA207B637B54
:101BB0008342F5D06073BDE83840FFF7C1BF022013
:101BC000EAE700BF442700202DE9F0431E4687B016
:101BD00000230546CDE901330C46174601F027FDE9
:101BE000032D61D8DFE815F07B00C3000E0104006F
:101BF000A27C082A04D94FF0FF3007B0BDE8F0837B
